
LEDs_Animation.elf:     file format elf32-littlearm

Sections:
Idx Name          Size      VMA       LMA       File off  Algn
  0 .isr_vector   000001ac  08000000  08000000  00010000  2**0
                  CONTENTS, ALLOC, LOAD, READONLY, DATA
  1 .text         0000194c  080001ac  080001ac  000101ac  2**2
                  CONTENTS, ALLOC, LOAD, READONLY, CODE
  2 .rodata       00000010  08001af8  08001af8  00011af8  2**2
                  CONTENTS, ALLOC, LOAD, READONLY, DATA
  3 .ARM.extab    00000000  08001b08  08001b08  0002000c  2**0
                  CONTENTS
  4 .ARM          00000008  08001b08  08001b08  00011b08  2**2
                  CONTENTS, ALLOC, LOAD, READONLY, DATA
  5 .preinit_array 00000000  08001b10  08001b10  0002000c  2**0
                  CONTENTS, ALLOC, LOAD, DATA
  6 .init_array   00000004  08001b10  08001b10  00011b10  2**2
                  CONTENTS, ALLOC, LOAD, DATA
  7 .fini_array   00000004  08001b14  08001b14  00011b14  2**2
                  CONTENTS, ALLOC, LOAD, DATA
  8 .data         0000000c  20000000  08001b18  00020000  2**2
                  CONTENTS, ALLOC, LOAD, DATA
  9 .ccmram       00000000  10000000  10000000  0002000c  2**0
                  CONTENTS
 10 .bss          00000024  2000000c  2000000c  0002000c  2**2
                  ALLOC
 11 ._user_heap_stack 00000600  20000030  20000030  0002000c  2**0
                  ALLOC
 12 .ARM.attributes 00000030  00000000  00000000  0002000c  2**0
                  CONTENTS, READONLY
 13 .debug_info   00003a26  00000000  00000000  0002003c  2**0
                  CONTENTS, READONLY, DEBUGGING, OCTETS
 14 .debug_abbrev 00000e2f  00000000  00000000  00023a62  2**0
                  CONTENTS, READONLY, DEBUGGING, OCTETS
 15 .debug_aranges 00000400  00000000  00000000  00024898  2**3
                  CONTENTS, READONLY, DEBUGGING, OCTETS
 16 .debug_ranges 00000378  00000000  00000000  00024c98  2**3
                  CONTENTS, READONLY, DEBUGGING, OCTETS
 17 .debug_macro  0002151f  00000000  00000000  00025010  2**0
                  CONTENTS, READONLY, DEBUGGING, OCTETS
 18 .debug_line   00004a10  00000000  00000000  0004652f  2**0
                  CONTENTS, READONLY, DEBUGGING, OCTETS
 19 .debug_str    000caf04  00000000  00000000  0004af3f  2**0
                  CONTENTS, READONLY, DEBUGGING, OCTETS
 20 .comment      00000050  00000000  00000000  00115e43  2**0
                  CONTENTS, READONLY
 21 .debug_frame  00000e54  00000000  00000000  00115e94  2**2
                  CONTENTS, READONLY, DEBUGGING, OCTETS

Disassembly of section .text:

080001ac <__do_global_dtors_aux>:
 80001ac:	b510      	push	{r4, lr}
 80001ae:	4c05      	ldr	r4, [pc, #20]	; (80001c4 <__do_global_dtors_aux+0x18>)
 80001b0:	7823      	ldrb	r3, [r4, #0]
 80001b2:	b933      	cbnz	r3, 80001c2 <__do_global_dtors_aux+0x16>
 80001b4:	4b04      	ldr	r3, [pc, #16]	; (80001c8 <__do_global_dtors_aux+0x1c>)
 80001b6:	b113      	cbz	r3, 80001be <__do_global_dtors_aux+0x12>
 80001b8:	4804      	ldr	r0, [pc, #16]	; (80001cc <__do_global_dtors_aux+0x20>)
 80001ba:	f3af 8000 	nop.w
 80001be:	2301      	movs	r3, #1
 80001c0:	7023      	strb	r3, [r4, #0]
 80001c2:	bd10      	pop	{r4, pc}
 80001c4:	2000000c 	.word	0x2000000c
 80001c8:	00000000 	.word	0x00000000
 80001cc:	08001ae0 	.word	0x08001ae0

080001d0 <frame_dummy>:
 80001d0:	b508      	push	{r3, lr}
 80001d2:	4b03      	ldr	r3, [pc, #12]	; (80001e0 <frame_dummy+0x10>)
 80001d4:	b11b      	cbz	r3, 80001de <frame_dummy+0xe>
 80001d6:	4903      	ldr	r1, [pc, #12]	; (80001e4 <frame_dummy+0x14>)
 80001d8:	4803      	ldr	r0, [pc, #12]	; (80001e8 <frame_dummy+0x18>)
 80001da:	f3af 8000 	nop.w
 80001de:	bd08      	pop	{r3, pc}
 80001e0:	00000000 	.word	0x00000000
 80001e4:	20000010 	.word	0x20000010
 80001e8:	08001ae0 	.word	0x08001ae0

080001ec <__aeabi_uldivmod>:
 80001ec:	b953      	cbnz	r3, 8000204 <__aeabi_uldivmod+0x18>
 80001ee:	b94a      	cbnz	r2, 8000204 <__aeabi_uldivmod+0x18>
 80001f0:	2900      	cmp	r1, #0
 80001f2:	bf08      	it	eq
 80001f4:	2800      	cmpeq	r0, #0
 80001f6:	bf1c      	itt	ne
 80001f8:	f04f 31ff 	movne.w	r1, #4294967295
 80001fc:	f04f 30ff 	movne.w	r0, #4294967295
 8000200:	f000 b974 	b.w	80004ec <__aeabi_idiv0>
 8000204:	f1ad 0c08 	sub.w	ip, sp, #8
 8000208:	e96d ce04 	strd	ip, lr, [sp, #-16]!
 800020c:	f000 f806 	bl	800021c <__udivmoddi4>
 8000210:	f8dd e004 	ldr.w	lr, [sp, #4]
 8000214:	e9dd 2302 	ldrd	r2, r3, [sp, #8]
 8000218:	b004      	add	sp, #16
 800021a:	4770      	bx	lr

0800021c <__udivmoddi4>:
 800021c:	e92d 47f0 	stmdb	sp!, {r4, r5, r6, r7, r8, r9, sl, lr}
 8000220:	9d08      	ldr	r5, [sp, #32]
 8000222:	4604      	mov	r4, r0
 8000224:	468e      	mov	lr, r1
 8000226:	2b00      	cmp	r3, #0
 8000228:	d14d      	bne.n	80002c6 <__udivmoddi4+0xaa>
 800022a:	428a      	cmp	r2, r1
 800022c:	4694      	mov	ip, r2
 800022e:	d969      	bls.n	8000304 <__udivmoddi4+0xe8>
 8000230:	fab2 f282 	clz	r2, r2
 8000234:	b152      	cbz	r2, 800024c <__udivmoddi4+0x30>
 8000236:	fa01 f302 	lsl.w	r3, r1, r2
 800023a:	f1c2 0120 	rsb	r1, r2, #32
 800023e:	fa20 f101 	lsr.w	r1, r0, r1
 8000242:	fa0c fc02 	lsl.w	ip, ip, r2
 8000246:	ea41 0e03 	orr.w	lr, r1, r3
 800024a:	4094      	lsls	r4, r2
 800024c:	ea4f 481c 	mov.w	r8, ip, lsr #16
 8000250:	0c21      	lsrs	r1, r4, #16
 8000252:	fbbe f6f8 	udiv	r6, lr, r8
 8000256:	fa1f f78c 	uxth.w	r7, ip
 800025a:	fb08 e316 	mls	r3, r8, r6, lr
 800025e:	ea41 4303 	orr.w	r3, r1, r3, lsl #16
 8000262:	fb06 f107 	mul.w	r1, r6, r7
 8000266:	4299      	cmp	r1, r3
 8000268:	d90a      	bls.n	8000280 <__udivmoddi4+0x64>
 800026a:	eb1c 0303 	adds.w	r3, ip, r3
 800026e:	f106 30ff 	add.w	r0, r6, #4294967295
 8000272:	f080 811f 	bcs.w	80004b4 <__udivmoddi4+0x298>
 8000276:	4299      	cmp	r1, r3
 8000278:	f240 811c 	bls.w	80004b4 <__udivmoddi4+0x298>
 800027c:	3e02      	subs	r6, #2
 800027e:	4463      	add	r3, ip
 8000280:	1a5b      	subs	r3, r3, r1
 8000282:	b2a4      	uxth	r4, r4
 8000284:	fbb3 f0f8 	udiv	r0, r3, r8
 8000288:	fb08 3310 	mls	r3, r8, r0, r3
 800028c:	ea44 4403 	orr.w	r4, r4, r3, lsl #16
 8000290:	fb00 f707 	mul.w	r7, r0, r7
 8000294:	42a7      	cmp	r7, r4
 8000296:	d90a      	bls.n	80002ae <__udivmoddi4+0x92>
 8000298:	eb1c 0404 	adds.w	r4, ip, r4
 800029c:	f100 33ff 	add.w	r3, r0, #4294967295
 80002a0:	f080 810a 	bcs.w	80004b8 <__udivmoddi4+0x29c>
 80002a4:	42a7      	cmp	r7, r4
 80002a6:	f240 8107 	bls.w	80004b8 <__udivmoddi4+0x29c>
 80002aa:	4464      	add	r4, ip
 80002ac:	3802      	subs	r0, #2
 80002ae:	ea40 4006 	orr.w	r0, r0, r6, lsl #16
 80002b2:	1be4      	subs	r4, r4, r7
 80002b4:	2600      	movs	r6, #0
 80002b6:	b11d      	cbz	r5, 80002c0 <__udivmoddi4+0xa4>
 80002b8:	40d4      	lsrs	r4, r2
 80002ba:	2300      	movs	r3, #0
 80002bc:	e9c5 4300 	strd	r4, r3, [r5]
 80002c0:	4631      	mov	r1, r6
 80002c2:	e8bd 87f0 	ldmia.w	sp!, {r4, r5, r6, r7, r8, r9, sl, pc}
 80002c6:	428b      	cmp	r3, r1
 80002c8:	d909      	bls.n	80002de <__udivmoddi4+0xc2>
 80002ca:	2d00      	cmp	r5, #0
 80002cc:	f000 80ef 	beq.w	80004ae <__udivmoddi4+0x292>
 80002d0:	2600      	movs	r6, #0
 80002d2:	e9c5 0100 	strd	r0, r1, [r5]
 80002d6:	4630      	mov	r0, r6
 80002d8:	4631      	mov	r1, r6
 80002da:	e8bd 87f0 	ldmia.w	sp!, {r4, r5, r6, r7, r8, r9, sl, pc}
 80002de:	fab3 f683 	clz	r6, r3
 80002e2:	2e00      	cmp	r6, #0
 80002e4:	d14a      	bne.n	800037c <__udivmoddi4+0x160>
 80002e6:	428b      	cmp	r3, r1
 80002e8:	d302      	bcc.n	80002f0 <__udivmoddi4+0xd4>
 80002ea:	4282      	cmp	r2, r0
 80002ec:	f200 80f9 	bhi.w	80004e2 <__udivmoddi4+0x2c6>
 80002f0:	1a84      	subs	r4, r0, r2
 80002f2:	eb61 0303 	sbc.w	r3, r1, r3
 80002f6:	2001      	movs	r0, #1
 80002f8:	469e      	mov	lr, r3
 80002fa:	2d00      	cmp	r5, #0
 80002fc:	d0e0      	beq.n	80002c0 <__udivmoddi4+0xa4>
 80002fe:	e9c5 4e00 	strd	r4, lr, [r5]
 8000302:	e7dd      	b.n	80002c0 <__udivmoddi4+0xa4>
 8000304:	b902      	cbnz	r2, 8000308 <__udivmoddi4+0xec>
 8000306:	deff      	udf	#255	; 0xff
 8000308:	fab2 f282 	clz	r2, r2
 800030c:	2a00      	cmp	r2, #0
 800030e:	f040 8092 	bne.w	8000436 <__udivmoddi4+0x21a>
 8000312:	eba1 010c 	sub.w	r1, r1, ip
 8000316:	ea4f 471c 	mov.w	r7, ip, lsr #16
 800031a:	fa1f fe8c 	uxth.w	lr, ip
 800031e:	2601      	movs	r6, #1
 8000320:	0c20      	lsrs	r0, r4, #16
 8000322:	fbb1 f3f7 	udiv	r3, r1, r7
 8000326:	fb07 1113 	mls	r1, r7, r3, r1
 800032a:	ea40 4101 	orr.w	r1, r0, r1, lsl #16
 800032e:	fb0e f003 	mul.w	r0, lr, r3
 8000332:	4288      	cmp	r0, r1
 8000334:	d908      	bls.n	8000348 <__udivmoddi4+0x12c>
 8000336:	eb1c 0101 	adds.w	r1, ip, r1
 800033a:	f103 38ff 	add.w	r8, r3, #4294967295
 800033e:	d202      	bcs.n	8000346 <__udivmoddi4+0x12a>
 8000340:	4288      	cmp	r0, r1
 8000342:	f200 80cb 	bhi.w	80004dc <__udivmoddi4+0x2c0>
 8000346:	4643      	mov	r3, r8
 8000348:	1a09      	subs	r1, r1, r0
 800034a:	b2a4      	uxth	r4, r4
 800034c:	fbb1 f0f7 	udiv	r0, r1, r7
 8000350:	fb07 1110 	mls	r1, r7, r0, r1
 8000354:	ea44 4401 	orr.w	r4, r4, r1, lsl #16
 8000358:	fb0e fe00 	mul.w	lr, lr, r0
 800035c:	45a6      	cmp	lr, r4
 800035e:	d908      	bls.n	8000372 <__udivmoddi4+0x156>
 8000360:	eb1c 0404 	adds.w	r4, ip, r4
 8000364:	f100 31ff 	add.w	r1, r0, #4294967295
 8000368:	d202      	bcs.n	8000370 <__udivmoddi4+0x154>
 800036a:	45a6      	cmp	lr, r4
 800036c:	f200 80bb 	bhi.w	80004e6 <__udivmoddi4+0x2ca>
 8000370:	4608      	mov	r0, r1
 8000372:	eba4 040e 	sub.w	r4, r4, lr
 8000376:	ea40 4003 	orr.w	r0, r0, r3, lsl #16
 800037a:	e79c      	b.n	80002b6 <__udivmoddi4+0x9a>
 800037c:	f1c6 0720 	rsb	r7, r6, #32
 8000380:	40b3      	lsls	r3, r6
 8000382:	fa22 fc07 	lsr.w	ip, r2, r7
 8000386:	ea4c 0c03 	orr.w	ip, ip, r3
 800038a:	fa20 f407 	lsr.w	r4, r0, r7
 800038e:	fa01 f306 	lsl.w	r3, r1, r6
 8000392:	431c      	orrs	r4, r3
 8000394:	40f9      	lsrs	r1, r7
 8000396:	ea4f 491c 	mov.w	r9, ip, lsr #16
 800039a:	fa00 f306 	lsl.w	r3, r0, r6
 800039e:	fbb1 f8f9 	udiv	r8, r1, r9
 80003a2:	0c20      	lsrs	r0, r4, #16
 80003a4:	fa1f fe8c 	uxth.w	lr, ip
 80003a8:	fb09 1118 	mls	r1, r9, r8, r1
 80003ac:	ea40 4101 	orr.w	r1, r0, r1, lsl #16
 80003b0:	fb08 f00e 	mul.w	r0, r8, lr
 80003b4:	4288      	cmp	r0, r1
 80003b6:	fa02 f206 	lsl.w	r2, r2, r6
 80003ba:	d90b      	bls.n	80003d4 <__udivmoddi4+0x1b8>
 80003bc:	eb1c 0101 	adds.w	r1, ip, r1
 80003c0:	f108 3aff 	add.w	sl, r8, #4294967295
 80003c4:	f080 8088 	bcs.w	80004d8 <__udivmoddi4+0x2bc>
 80003c8:	4288      	cmp	r0, r1
 80003ca:	f240 8085 	bls.w	80004d8 <__udivmoddi4+0x2bc>
 80003ce:	f1a8 0802 	sub.w	r8, r8, #2
 80003d2:	4461      	add	r1, ip
 80003d4:	1a09      	subs	r1, r1, r0
 80003d6:	b2a4      	uxth	r4, r4
 80003d8:	fbb1 f0f9 	udiv	r0, r1, r9
 80003dc:	fb09 1110 	mls	r1, r9, r0, r1
 80003e0:	ea44 4101 	orr.w	r1, r4, r1, lsl #16
 80003e4:	fb00 fe0e 	mul.w	lr, r0, lr
 80003e8:	458e      	cmp	lr, r1
 80003ea:	d908      	bls.n	80003fe <__udivmoddi4+0x1e2>
 80003ec:	eb1c 0101 	adds.w	r1, ip, r1
 80003f0:	f100 34ff 	add.w	r4, r0, #4294967295
 80003f4:	d26c      	bcs.n	80004d0 <__udivmoddi4+0x2b4>
 80003f6:	458e      	cmp	lr, r1
 80003f8:	d96a      	bls.n	80004d0 <__udivmoddi4+0x2b4>
 80003fa:	3802      	subs	r0, #2
 80003fc:	4461      	add	r1, ip
 80003fe:	ea40 4008 	orr.w	r0, r0, r8, lsl #16
 8000402:	fba0 9402 	umull	r9, r4, r0, r2
 8000406:	eba1 010e 	sub.w	r1, r1, lr
 800040a:	42a1      	cmp	r1, r4
 800040c:	46c8      	mov	r8, r9
 800040e:	46a6      	mov	lr, r4
 8000410:	d356      	bcc.n	80004c0 <__udivmoddi4+0x2a4>
 8000412:	d053      	beq.n	80004bc <__udivmoddi4+0x2a0>
 8000414:	b15d      	cbz	r5, 800042e <__udivmoddi4+0x212>
 8000416:	ebb3 0208 	subs.w	r2, r3, r8
 800041a:	eb61 010e 	sbc.w	r1, r1, lr
 800041e:	fa01 f707 	lsl.w	r7, r1, r7
 8000422:	fa22 f306 	lsr.w	r3, r2, r6
 8000426:	40f1      	lsrs	r1, r6
 8000428:	431f      	orrs	r7, r3
 800042a:	e9c5 7100 	strd	r7, r1, [r5]
 800042e:	2600      	movs	r6, #0
 8000430:	4631      	mov	r1, r6
 8000432:	e8bd 87f0 	ldmia.w	sp!, {r4, r5, r6, r7, r8, r9, sl, pc}
 8000436:	f1c2 0320 	rsb	r3, r2, #32
 800043a:	40d8      	lsrs	r0, r3
 800043c:	fa0c fc02 	lsl.w	ip, ip, r2
 8000440:	fa21 f303 	lsr.w	r3, r1, r3
 8000444:	4091      	lsls	r1, r2
 8000446:	4301      	orrs	r1, r0
 8000448:	ea4f 471c 	mov.w	r7, ip, lsr #16
 800044c:	fa1f fe8c 	uxth.w	lr, ip
 8000450:	fbb3 f0f7 	udiv	r0, r3, r7
 8000454:	fb07 3610 	mls	r6, r7, r0, r3
 8000458:	0c0b      	lsrs	r3, r1, #16
 800045a:	ea43 4306 	orr.w	r3, r3, r6, lsl #16
 800045e:	fb00 f60e 	mul.w	r6, r0, lr
 8000462:	429e      	cmp	r6, r3
 8000464:	fa04 f402 	lsl.w	r4, r4, r2
 8000468:	d908      	bls.n	800047c <__udivmoddi4+0x260>
 800046a:	eb1c 0303 	adds.w	r3, ip, r3
 800046e:	f100 38ff 	add.w	r8, r0, #4294967295
 8000472:	d22f      	bcs.n	80004d4 <__udivmoddi4+0x2b8>
 8000474:	429e      	cmp	r6, r3
 8000476:	d92d      	bls.n	80004d4 <__udivmoddi4+0x2b8>
 8000478:	3802      	subs	r0, #2
 800047a:	4463      	add	r3, ip
 800047c:	1b9b      	subs	r3, r3, r6
 800047e:	b289      	uxth	r1, r1
 8000480:	fbb3 f6f7 	udiv	r6, r3, r7
 8000484:	fb07 3316 	mls	r3, r7, r6, r3
 8000488:	ea41 4103 	orr.w	r1, r1, r3, lsl #16
 800048c:	fb06 f30e 	mul.w	r3, r6, lr
 8000490:	428b      	cmp	r3, r1
 8000492:	d908      	bls.n	80004a6 <__udivmoddi4+0x28a>
 8000494:	eb1c 0101 	adds.w	r1, ip, r1
 8000498:	f106 38ff 	add.w	r8, r6, #4294967295
 800049c:	d216      	bcs.n	80004cc <__udivmoddi4+0x2b0>
 800049e:	428b      	cmp	r3, r1
 80004a0:	d914      	bls.n	80004cc <__udivmoddi4+0x2b0>
 80004a2:	3e02      	subs	r6, #2
 80004a4:	4461      	add	r1, ip
 80004a6:	1ac9      	subs	r1, r1, r3
 80004a8:	ea46 4600 	orr.w	r6, r6, r0, lsl #16
 80004ac:	e738      	b.n	8000320 <__udivmoddi4+0x104>
 80004ae:	462e      	mov	r6, r5
 80004b0:	4628      	mov	r0, r5
 80004b2:	e705      	b.n	80002c0 <__udivmoddi4+0xa4>
 80004b4:	4606      	mov	r6, r0
 80004b6:	e6e3      	b.n	8000280 <__udivmoddi4+0x64>
 80004b8:	4618      	mov	r0, r3
 80004ba:	e6f8      	b.n	80002ae <__udivmoddi4+0x92>
 80004bc:	454b      	cmp	r3, r9
 80004be:	d2a9      	bcs.n	8000414 <__udivmoddi4+0x1f8>
 80004c0:	ebb9 0802 	subs.w	r8, r9, r2
 80004c4:	eb64 0e0c 	sbc.w	lr, r4, ip
 80004c8:	3801      	subs	r0, #1
 80004ca:	e7a3      	b.n	8000414 <__udivmoddi4+0x1f8>
 80004cc:	4646      	mov	r6, r8
 80004ce:	e7ea      	b.n	80004a6 <__udivmoddi4+0x28a>
 80004d0:	4620      	mov	r0, r4
 80004d2:	e794      	b.n	80003fe <__udivmoddi4+0x1e2>
 80004d4:	4640      	mov	r0, r8
 80004d6:	e7d1      	b.n	800047c <__udivmoddi4+0x260>
 80004d8:	46d0      	mov	r8, sl
 80004da:	e77b      	b.n	80003d4 <__udivmoddi4+0x1b8>
 80004dc:	3b02      	subs	r3, #2
 80004de:	4461      	add	r1, ip
 80004e0:	e732      	b.n	8000348 <__udivmoddi4+0x12c>
 80004e2:	4630      	mov	r0, r6
 80004e4:	e709      	b.n	80002fa <__udivmoddi4+0xde>
 80004e6:	4464      	add	r4, ip
 80004e8:	3802      	subs	r0, #2
 80004ea:	e742      	b.n	8000372 <__udivmoddi4+0x156>

080004ec <__aeabi_idiv0>:
 80004ec:	4770      	bx	lr
 80004ee:	bf00      	nop

080004f0 <main>:
static void MX_GPIO_Init(void);

char state=0;

int main(void)
{
 80004f0:	b580      	push	{r7, lr}
 80004f2:	af00      	add	r7, sp, #0


  /* Reset of all peripherals, Initializes the Flash interface and the Systick. */
  HAL_Init();
 80004f4:	f000 fb0a 	bl	8000b0c <HAL_Init>

  /* Configure the system clock */
  SystemClock_Config();
 80004f8:	f000 f984 	bl	8000804 <SystemClock_Config>

  /* Initialize all configured peripherals */
  MX_GPIO_Init();
 80004fc:	f000 f9ee 	bl	80008dc <MX_GPIO_Init>

  /* Infinite loop */
  while (1)
  {
	  while(HAL_GPIO_ReadPin(User_Button_GPIO_Port, User_Button_Pin) != GPIO_PIN_SET);
 8000500:	bf00      	nop
 8000502:	2101      	movs	r1, #1
 8000504:	48bb      	ldr	r0, [pc, #748]	; (80007f4 <main+0x304>)
 8000506:	f000 fe29 	bl	800115c <HAL_GPIO_ReadPin>
 800050a:	4603      	mov	r3, r0
 800050c:	2b01      	cmp	r3, #1
 800050e:	d1f8      	bne.n	8000502 <main+0x12>
	  while(HAL_GPIO_ReadPin(User_Button_GPIO_Port, User_Button_Pin) != GPIO_PIN_RESET);
 8000510:	bf00      	nop
 8000512:	2101      	movs	r1, #1
 8000514:	48b7      	ldr	r0, [pc, #732]	; (80007f4 <main+0x304>)
 8000516:	f000 fe21 	bl	800115c <HAL_GPIO_ReadPin>
 800051a:	4603      	mov	r3, r0
 800051c:	2b00      	cmp	r3, #0
 800051e:	d1f8      	bne.n	8000512 <main+0x22>
	  state ++;
 8000520:	4bb5      	ldr	r3, [pc, #724]	; (80007f8 <main+0x308>)
 8000522:	781b      	ldrb	r3, [r3, #0]
 8000524:	3301      	adds	r3, #1
 8000526:	b2da      	uxtb	r2, r3
 8000528:	4bb3      	ldr	r3, [pc, #716]	; (80007f8 <main+0x308>)
 800052a:	701a      	strb	r2, [r3, #0]

  	  switch (state)
 800052c:	4bb2      	ldr	r3, [pc, #712]	; (80007f8 <main+0x308>)
 800052e:	781b      	ldrb	r3, [r3, #0]
 8000530:	2b03      	cmp	r3, #3
 8000532:	f000 80f1 	beq.w	8000718 <main+0x228>
 8000536:	2b03      	cmp	r3, #3
 8000538:	dce2      	bgt.n	8000500 <main+0x10>
 800053a:	2b01      	cmp	r3, #1
 800053c:	d002      	beq.n	8000544 <main+0x54>
 800053e:	2b02      	cmp	r3, #2
 8000540:	d075      	beq.n	800062e <main+0x13e>
 8000542:	e155      	b.n	80007f0 <main+0x300>
  	  {
  	  	  case 1:
  	  		  HAL_GPIO_WritePin(LED_0_GPIO_Port, LED_0_Pin, GPIO_PIN_SET);
 8000544:	2201      	movs	r2, #1
 8000546:	2140      	movs	r1, #64	; 0x40
 8000548:	48ac      	ldr	r0, [pc, #688]	; (80007fc <main+0x30c>)
 800054a:	f000 fe1f 	bl	800118c <HAL_GPIO_WritePin>
  	  		  HAL_Delay(1000);
 800054e:	f44f 707a 	mov.w	r0, #1000	; 0x3e8
 8000552:	f000 fb4d 	bl	8000bf0 <HAL_Delay>
  	  		  HAL_GPIO_WritePin(LED_0_GPIO_Port, LED_0_Pin, GPIO_PIN_RESET);
 8000556:	2200      	movs	r2, #0
 8000558:	2140      	movs	r1, #64	; 0x40
 800055a:	48a8      	ldr	r0, [pc, #672]	; (80007fc <main+0x30c>)
 800055c:	f000 fe16 	bl	800118c <HAL_GPIO_WritePin>
  	  		  HAL_Delay(1000);
 8000560:	f44f 707a 	mov.w	r0, #1000	; 0x3e8
 8000564:	f000 fb44 	bl	8000bf0 <HAL_Delay>

  	  		  HAL_GPIO_WritePin(LED_1_GPIO_Port, LED_1_Pin, GPIO_PIN_SET);
 8000568:	2201      	movs	r2, #1
 800056a:	2180      	movs	r1, #128	; 0x80
 800056c:	48a3      	ldr	r0, [pc, #652]	; (80007fc <main+0x30c>)
 800056e:	f000 fe0d 	bl	800118c <HAL_GPIO_WritePin>
  	  		  HAL_Delay(1000);
 8000572:	f44f 707a 	mov.w	r0, #1000	; 0x3e8
 8000576:	f000 fb3b 	bl	8000bf0 <HAL_Delay>
  	  		  HAL_GPIO_WritePin(LED_1_GPIO_Port, LED_1_Pin, GPIO_PIN_RESET);
 800057a:	2200      	movs	r2, #0
 800057c:	2180      	movs	r1, #128	; 0x80
 800057e:	489f      	ldr	r0, [pc, #636]	; (80007fc <main+0x30c>)
 8000580:	f000 fe04 	bl	800118c <HAL_GPIO_WritePin>
  	  		  HAL_Delay(1000);
 8000584:	f44f 707a 	mov.w	r0, #1000	; 0x3e8
 8000588:	f000 fb32 	bl	8000bf0 <HAL_Delay>

  	  		  HAL_GPIO_WritePin(LED_2_GPIO_Port, LED_2_Pin, GPIO_PIN_SET);
 800058c:	2201      	movs	r2, #1
 800058e:	f44f 7100 	mov.w	r1, #512	; 0x200
 8000592:	489b      	ldr	r0, [pc, #620]	; (8000800 <main+0x310>)
 8000594:	f000 fdfa 	bl	800118c <HAL_GPIO_WritePin>
  	  		  HAL_Delay(1000);
 8000598:	f44f 707a 	mov.w	r0, #1000	; 0x3e8
 800059c:	f000 fb28 	bl	8000bf0 <HAL_Delay>
  	  		  HAL_GPIO_WritePin(LED_2_GPIO_Port, LED_2_Pin, GPIO_PIN_RESET);
 80005a0:	2200      	movs	r2, #0
 80005a2:	f44f 7100 	mov.w	r1, #512	; 0x200
 80005a6:	4896      	ldr	r0, [pc, #600]	; (8000800 <main+0x310>)
 80005a8:	f000 fdf0 	bl	800118c <HAL_GPIO_WritePin>
  	  		  HAL_Delay(1000);
 80005ac:	f44f 707a 	mov.w	r0, #1000	; 0x3e8
 80005b0:	f000 fb1e 	bl	8000bf0 <HAL_Delay>

  	  		  HAL_GPIO_WritePin(LED_3_GPIO_Port, LED_3_Pin, GPIO_PIN_SET);
 80005b4:	2201      	movs	r2, #1
 80005b6:	f44f 6180 	mov.w	r1, #1024	; 0x400
 80005ba:	4891      	ldr	r0, [pc, #580]	; (8000800 <main+0x310>)
 80005bc:	f000 fde6 	bl	800118c <HAL_GPIO_WritePin>
  	  		  HAL_Delay(1000);
 80005c0:	f44f 707a 	mov.w	r0, #1000	; 0x3e8
 80005c4:	f000 fb14 	bl	8000bf0 <HAL_Delay>
  	  		  HAL_GPIO_WritePin(LED_3_GPIO_Port, LED_3_Pin, GPIO_PIN_RESET);
 80005c8:	2200      	movs	r2, #0
 80005ca:	f44f 6180 	mov.w	r1, #1024	; 0x400
 80005ce:	488c      	ldr	r0, [pc, #560]	; (8000800 <main+0x310>)
 80005d0:	f000 fddc 	bl	800118c <HAL_GPIO_WritePin>
  	  		  HAL_Delay(1000);
 80005d4:	f44f 707a 	mov.w	r0, #1000	; 0x3e8
 80005d8:	f000 fb0a 	bl	8000bf0 <HAL_Delay>

  	  		  HAL_GPIO_WritePin(LED_4_GPIO_Port, LED_4_Pin, GPIO_PIN_SET);
 80005dc:	2201      	movs	r2, #1
 80005de:	f44f 6100 	mov.w	r1, #2048	; 0x800
 80005e2:	4887      	ldr	r0, [pc, #540]	; (8000800 <main+0x310>)
 80005e4:	f000 fdd2 	bl	800118c <HAL_GPIO_WritePin>
  	  		  HAL_Delay(1000);
 80005e8:	f44f 707a 	mov.w	r0, #1000	; 0x3e8
 80005ec:	f000 fb00 	bl	8000bf0 <HAL_Delay>
  	  		  HAL_GPIO_WritePin(LED_4_GPIO_Port, LED_4_Pin, GPIO_PIN_RESET);
 80005f0:	2200      	movs	r2, #0
 80005f2:	f44f 6100 	mov.w	r1, #2048	; 0x800
 80005f6:	4882      	ldr	r0, [pc, #520]	; (8000800 <main+0x310>)
 80005f8:	f000 fdc8 	bl	800118c <HAL_GPIO_WritePin>
  	  		  HAL_Delay(1000);
 80005fc:	f44f 707a 	mov.w	r0, #1000	; 0x3e8
 8000600:	f000 faf6 	bl	8000bf0 <HAL_Delay>

  	  		  HAL_GPIO_WritePin(LED_5_GPIO_Port, LED_5_Pin, GPIO_PIN_SET);
 8000604:	2201      	movs	r2, #1
 8000606:	f44f 5180 	mov.w	r1, #4096	; 0x1000
 800060a:	487d      	ldr	r0, [pc, #500]	; (8000800 <main+0x310>)
 800060c:	f000 fdbe 	bl	800118c <HAL_GPIO_WritePin>
  	  		  HAL_Delay(1000);
 8000610:	f44f 707a 	mov.w	r0, #1000	; 0x3e8
 8000614:	f000 faec 	bl	8000bf0 <HAL_Delay>
  	  	  	  HAL_GPIO_WritePin(LED_5_GPIO_Port, LED_5_Pin, GPIO_PIN_RESET);
 8000618:	2200      	movs	r2, #0
 800061a:	f44f 5180 	mov.w	r1, #4096	; 0x1000
 800061e:	4878      	ldr	r0, [pc, #480]	; (8000800 <main+0x310>)
 8000620:	f000 fdb4 	bl	800118c <HAL_GPIO_WritePin>
  	  	  	  HAL_Delay(1000);
 8000624:	f44f 707a 	mov.w	r0, #1000	; 0x3e8
 8000628:	f000 fae2 	bl	8000bf0 <HAL_Delay>
  	  	  	 break;
 800062c:	e0e0      	b.n	80007f0 <main+0x300>

  	  	  case 2:
		  		  HAL_GPIO_WritePin(LED_0_GPIO_Port, LED_0_Pin, GPIO_PIN_SET);
 800062e:	2201      	movs	r2, #1
 8000630:	2140      	movs	r1, #64	; 0x40
 8000632:	4872      	ldr	r0, [pc, #456]	; (80007fc <main+0x30c>)
 8000634:	f000 fdaa 	bl	800118c <HAL_GPIO_WritePin>
		  		  HAL_Delay(500);
 8000638:	f44f 70fa 	mov.w	r0, #500	; 0x1f4
 800063c:	f000 fad8 	bl	8000bf0 <HAL_Delay>
		  		  HAL_GPIO_WritePin(LED_0_GPIO_Port, LED_0_Pin, GPIO_PIN_RESET);
 8000640:	2200      	movs	r2, #0
 8000642:	2140      	movs	r1, #64	; 0x40
 8000644:	486d      	ldr	r0, [pc, #436]	; (80007fc <main+0x30c>)
 8000646:	f000 fda1 	bl	800118c <HAL_GPIO_WritePin>
		  		  HAL_Delay(500);
 800064a:	f44f 70fa 	mov.w	r0, #500	; 0x1f4
 800064e:	f000 facf 	bl	8000bf0 <HAL_Delay>

		  		  HAL_GPIO_WritePin(LED_1_GPIO_Port, LED_1_Pin, GPIO_PIN_SET);
 8000652:	2201      	movs	r2, #1
 8000654:	2180      	movs	r1, #128	; 0x80
 8000656:	4869      	ldr	r0, [pc, #420]	; (80007fc <main+0x30c>)
 8000658:	f000 fd98 	bl	800118c <HAL_GPIO_WritePin>
		  		  HAL_Delay(500);
 800065c:	f44f 70fa 	mov.w	r0, #500	; 0x1f4
 8000660:	f000 fac6 	bl	8000bf0 <HAL_Delay>
		  		  HAL_GPIO_WritePin(LED_1_GPIO_Port, LED_1_Pin, GPIO_PIN_RESET);
 8000664:	2200      	movs	r2, #0
 8000666:	2180      	movs	r1, #128	; 0x80
 8000668:	4864      	ldr	r0, [pc, #400]	; (80007fc <main+0x30c>)
 800066a:	f000 fd8f 	bl	800118c <HAL_GPIO_WritePin>
		  		  HAL_Delay(500);
 800066e:	f44f 70fa 	mov.w	r0, #500	; 0x1f4
 8000672:	f000 fabd 	bl	8000bf0 <HAL_Delay>

		  		  HAL_GPIO_WritePin(LED_2_GPIO_Port, LED_2_Pin, GPIO_PIN_SET);
 8000676:	2201      	movs	r2, #1
 8000678:	f44f 7100 	mov.w	r1, #512	; 0x200
 800067c:	4860      	ldr	r0, [pc, #384]	; (8000800 <main+0x310>)
 800067e:	f000 fd85 	bl	800118c <HAL_GPIO_WritePin>
		  		  HAL_Delay(500);
 8000682:	f44f 70fa 	mov.w	r0, #500	; 0x1f4
 8000686:	f000 fab3 	bl	8000bf0 <HAL_Delay>
		  		  HAL_GPIO_WritePin(LED_2_GPIO_Port, LED_2_Pin, GPIO_PIN_RESET);
 800068a:	2200      	movs	r2, #0
 800068c:	f44f 7100 	mov.w	r1, #512	; 0x200
 8000690:	485b      	ldr	r0, [pc, #364]	; (8000800 <main+0x310>)
 8000692:	f000 fd7b 	bl	800118c <HAL_GPIO_WritePin>
		  		  HAL_Delay(500);
 8000696:	f44f 70fa 	mov.w	r0, #500	; 0x1f4
 800069a:	f000 faa9 	bl	8000bf0 <HAL_Delay>

		  		  HAL_GPIO_WritePin(LED_3_GPIO_Port, LED_3_Pin, GPIO_PIN_SET);
 800069e:	2201      	movs	r2, #1
 80006a0:	f44f 6180 	mov.w	r1, #1024	; 0x400
 80006a4:	4856      	ldr	r0, [pc, #344]	; (8000800 <main+0x310>)
 80006a6:	f000 fd71 	bl	800118c <HAL_GPIO_WritePin>
		  		  HAL_Delay(500);
 80006aa:	f44f 70fa 	mov.w	r0, #500	; 0x1f4
 80006ae:	f000 fa9f 	bl	8000bf0 <HAL_Delay>
		  		  HAL_GPIO_WritePin(LED_3_GPIO_Port, LED_3_Pin, GPIO_PIN_RESET);
 80006b2:	2200      	movs	r2, #0
 80006b4:	f44f 6180 	mov.w	r1, #1024	; 0x400
 80006b8:	4851      	ldr	r0, [pc, #324]	; (8000800 <main+0x310>)
 80006ba:	f000 fd67 	bl	800118c <HAL_GPIO_WritePin>
		  		  HAL_Delay(500);
 80006be:	f44f 70fa 	mov.w	r0, #500	; 0x1f4
 80006c2:	f000 fa95 	bl	8000bf0 <HAL_Delay>

		  		  HAL_GPIO_WritePin(LED_4_GPIO_Port, LED_4_Pin, GPIO_PIN_SET);
 80006c6:	2201      	movs	r2, #1
 80006c8:	f44f 6100 	mov.w	r1, #2048	; 0x800
 80006cc:	484c      	ldr	r0, [pc, #304]	; (8000800 <main+0x310>)
 80006ce:	f000 fd5d 	bl	800118c <HAL_GPIO_WritePin>
		  		  HAL_Delay(500);
 80006d2:	f44f 70fa 	mov.w	r0, #500	; 0x1f4
 80006d6:	f000 fa8b 	bl	8000bf0 <HAL_Delay>
		  		  HAL_GPIO_WritePin(LED_4_GPIO_Port, LED_4_Pin, GPIO_PIN_RESET);
 80006da:	2200      	movs	r2, #0
 80006dc:	f44f 6100 	mov.w	r1, #2048	; 0x800
 80006e0:	4847      	ldr	r0, [pc, #284]	; (8000800 <main+0x310>)
 80006e2:	f000 fd53 	bl	800118c <HAL_GPIO_WritePin>
		  		  HAL_Delay(500);
 80006e6:	f44f 70fa 	mov.w	r0, #500	; 0x1f4
 80006ea:	f000 fa81 	bl	8000bf0 <HAL_Delay>

		  		  HAL_GPIO_WritePin(LED_5_GPIO_Port, LED_5_Pin, GPIO_PIN_SET);
 80006ee:	2201      	movs	r2, #1
 80006f0:	f44f 5180 	mov.w	r1, #4096	; 0x1000
 80006f4:	4842      	ldr	r0, [pc, #264]	; (8000800 <main+0x310>)
 80006f6:	f000 fd49 	bl	800118c <HAL_GPIO_WritePin>
		  		  HAL_Delay(500);
 80006fa:	f44f 70fa 	mov.w	r0, #500	; 0x1f4
 80006fe:	f000 fa77 	bl	8000bf0 <HAL_Delay>
		  		  HAL_GPIO_WritePin(LED_5_GPIO_Port, LED_5_Pin, GPIO_PIN_RESET);
 8000702:	2200      	movs	r2, #0
 8000704:	f44f 5180 	mov.w	r1, #4096	; 0x1000
 8000708:	483d      	ldr	r0, [pc, #244]	; (8000800 <main+0x310>)
 800070a:	f000 fd3f 	bl	800118c <HAL_GPIO_WritePin>
		  		  HAL_Delay(500);
 800070e:	f44f 70fa 	mov.w	r0, #500	; 0x1f4
 8000712:	f000 fa6d 	bl	8000bf0 <HAL_Delay>

  	  		  break;
 8000716:	e06b      	b.n	80007f0 <main+0x300>
  	  	  case 3:
  	  		HAL_GPIO_WritePin(LED_0_GPIO_Port, LED_0_Pin, GPIO_PIN_SET);
 8000718:	2201      	movs	r2, #1
 800071a:	2140      	movs	r1, #64	; 0x40
 800071c:	4837      	ldr	r0, [pc, #220]	; (80007fc <main+0x30c>)
 800071e:	f000 fd35 	bl	800118c <HAL_GPIO_WritePin>
  	  		HAL_Delay(100);
 8000722:	2064      	movs	r0, #100	; 0x64
 8000724:	f000 fa64 	bl	8000bf0 <HAL_Delay>
  	  		HAL_GPIO_WritePin(LED_0_GPIO_Port, LED_0_Pin, GPIO_PIN_RESET);
 8000728:	2200      	movs	r2, #0
 800072a:	2140      	movs	r1, #64	; 0x40
 800072c:	4833      	ldr	r0, [pc, #204]	; (80007fc <main+0x30c>)
 800072e:	f000 fd2d 	bl	800118c <HAL_GPIO_WritePin>
  	  		HAL_Delay(100);
 8000732:	2064      	movs	r0, #100	; 0x64
 8000734:	f000 fa5c 	bl	8000bf0 <HAL_Delay>

  	  		HAL_GPIO_WritePin(LED_1_GPIO_Port, LED_1_Pin, GPIO_PIN_SET);
 8000738:	2201      	movs	r2, #1
 800073a:	2180      	movs	r1, #128	; 0x80
 800073c:	482f      	ldr	r0, [pc, #188]	; (80007fc <main+0x30c>)
 800073e:	f000 fd25 	bl	800118c <HAL_GPIO_WritePin>
  	  		HAL_Delay(100);
 8000742:	2064      	movs	r0, #100	; 0x64
 8000744:	f000 fa54 	bl	8000bf0 <HAL_Delay>
  	  		HAL_GPIO_WritePin(LED_1_GPIO_Port, LED_1_Pin, GPIO_PIN_RESET);
 8000748:	2200      	movs	r2, #0
 800074a:	2180      	movs	r1, #128	; 0x80
 800074c:	482b      	ldr	r0, [pc, #172]	; (80007fc <main+0x30c>)
 800074e:	f000 fd1d 	bl	800118c <HAL_GPIO_WritePin>
  	  		HAL_Delay(100);
 8000752:	2064      	movs	r0, #100	; 0x64
 8000754:	f000 fa4c 	bl	8000bf0 <HAL_Delay>

  	  		HAL_GPIO_WritePin(LED_2_GPIO_Port, LED_2_Pin, GPIO_PIN_SET);
 8000758:	2201      	movs	r2, #1
 800075a:	f44f 7100 	mov.w	r1, #512	; 0x200
 800075e:	4828      	ldr	r0, [pc, #160]	; (8000800 <main+0x310>)
 8000760:	f000 fd14 	bl	800118c <HAL_GPIO_WritePin>
  	  		HAL_Delay(100);
 8000764:	2064      	movs	r0, #100	; 0x64
 8000766:	f000 fa43 	bl	8000bf0 <HAL_Delay>
  	  		HAL_GPIO_WritePin(LED_2_GPIO_Port, LED_2_Pin, GPIO_PIN_RESET);
 800076a:	2200      	movs	r2, #0
 800076c:	f44f 7100 	mov.w	r1, #512	; 0x200
 8000770:	4823      	ldr	r0, [pc, #140]	; (8000800 <main+0x310>)
 8000772:	f000 fd0b 	bl	800118c <HAL_GPIO_WritePin>
  	  		HAL_Delay(100);
 8000776:	2064      	movs	r0, #100	; 0x64
 8000778:	f000 fa3a 	bl	8000bf0 <HAL_Delay>

  	  		HAL_GPIO_WritePin(LED_3_GPIO_Port, LED_3_Pin, GPIO_PIN_SET);
 800077c:	2201      	movs	r2, #1
 800077e:	f44f 6180 	mov.w	r1, #1024	; 0x400
 8000782:	481f      	ldr	r0, [pc, #124]	; (8000800 <main+0x310>)
 8000784:	f000 fd02 	bl	800118c <HAL_GPIO_WritePin>
  	  		HAL_Delay(100);
 8000788:	2064      	movs	r0, #100	; 0x64
 800078a:	f000 fa31 	bl	8000bf0 <HAL_Delay>
  	  		HAL_GPIO_WritePin(LED_3_GPIO_Port, LED_3_Pin, GPIO_PIN_RESET);
 800078e:	2200      	movs	r2, #0
 8000790:	f44f 6180 	mov.w	r1, #1024	; 0x400
 8000794:	481a      	ldr	r0, [pc, #104]	; (8000800 <main+0x310>)
 8000796:	f000 fcf9 	bl	800118c <HAL_GPIO_WritePin>
  	  		HAL_Delay(100);
 800079a:	2064      	movs	r0, #100	; 0x64
 800079c:	f000 fa28 	bl	8000bf0 <HAL_Delay>

  	  		HAL_GPIO_WritePin(LED_4_GPIO_Port, LED_4_Pin, GPIO_PIN_SET);
 80007a0:	2201      	movs	r2, #1
 80007a2:	f44f 6100 	mov.w	r1, #2048	; 0x800
 80007a6:	4816      	ldr	r0, [pc, #88]	; (8000800 <main+0x310>)
 80007a8:	f000 fcf0 	bl	800118c <HAL_GPIO_WritePin>
  	  		HAL_Delay(100);
 80007ac:	2064      	movs	r0, #100	; 0x64
 80007ae:	f000 fa1f 	bl	8000bf0 <HAL_Delay>
  	  		HAL_GPIO_WritePin(LED_4_GPIO_Port, LED_4_Pin, GPIO_PIN_RESET);
 80007b2:	2200      	movs	r2, #0
 80007b4:	f44f 6100 	mov.w	r1, #2048	; 0x800
 80007b8:	4811      	ldr	r0, [pc, #68]	; (8000800 <main+0x310>)
 80007ba:	f000 fce7 	bl	800118c <HAL_GPIO_WritePin>
  	  		HAL_Delay(100);
 80007be:	2064      	movs	r0, #100	; 0x64
 80007c0:	f000 fa16 	bl	8000bf0 <HAL_Delay>

  	  		HAL_GPIO_WritePin(LED_5_GPIO_Port, LED_5_Pin, GPIO_PIN_SET);
 80007c4:	2201      	movs	r2, #1
 80007c6:	f44f 5180 	mov.w	r1, #4096	; 0x1000
 80007ca:	480d      	ldr	r0, [pc, #52]	; (8000800 <main+0x310>)
 80007cc:	f000 fcde 	bl	800118c <HAL_GPIO_WritePin>
  	  		HAL_Delay(100);
 80007d0:	2064      	movs	r0, #100	; 0x64
 80007d2:	f000 fa0d 	bl	8000bf0 <HAL_Delay>
  	  		HAL_GPIO_WritePin(LED_5_GPIO_Port, LED_5_Pin, GPIO_PIN_RESET);
 80007d6:	2200      	movs	r2, #0
 80007d8:	f44f 5180 	mov.w	r1, #4096	; 0x1000
 80007dc:	4808      	ldr	r0, [pc, #32]	; (8000800 <main+0x310>)
 80007de:	f000 fcd5 	bl	800118c <HAL_GPIO_WritePin>
  	  		HAL_Delay(100);
 80007e2:	2064      	movs	r0, #100	; 0x64
 80007e4:	f000 fa04 	bl	8000bf0 <HAL_Delay>

  	  		state = 0;
 80007e8:	4b03      	ldr	r3, [pc, #12]	; (80007f8 <main+0x308>)
 80007ea:	2200      	movs	r2, #0
 80007ec:	701a      	strb	r2, [r3, #0]
  	  		 break;
 80007ee:	bf00      	nop
	  while(HAL_GPIO_ReadPin(User_Button_GPIO_Port, User_Button_Pin) != GPIO_PIN_SET);
 80007f0:	e686      	b.n	8000500 <main+0x10>
 80007f2:	bf00      	nop
 80007f4:	40020000 	.word	0x40020000
 80007f8:	20000028 	.word	0x20000028
 80007fc:	40020c00 	.word	0x40020c00
 8000800:	40021800 	.word	0x40021800

08000804 <SystemClock_Config>:
/**
  * @brief System Clock Configuration
  * @retval None
  */
void SystemClock_Config(void)
{
 8000804:	b580      	push	{r7, lr}
 8000806:	b094      	sub	sp, #80	; 0x50
 8000808:	af00      	add	r7, sp, #0
  RCC_OscInitTypeDef RCC_OscInitStruct = {0};
 800080a:	f107 0320 	add.w	r3, r7, #32
 800080e:	2230      	movs	r2, #48	; 0x30
 8000810:	2100      	movs	r1, #0
 8000812:	4618      	mov	r0, r3
 8000814:	f001 f95c 	bl	8001ad0 <memset>
  RCC_ClkInitTypeDef RCC_ClkInitStruct = {0};
 8000818:	f107 030c 	add.w	r3, r7, #12
 800081c:	2200      	movs	r2, #0
 800081e:	601a      	str	r2, [r3, #0]
 8000820:	605a      	str	r2, [r3, #4]
 8000822:	609a      	str	r2, [r3, #8]
 8000824:	60da      	str	r2, [r3, #12]
 8000826:	611a      	str	r2, [r3, #16]

  /** Configure the main internal regulator output voltage
  */
  __HAL_RCC_PWR_CLK_ENABLE();
 8000828:	2300      	movs	r3, #0
 800082a:	60bb      	str	r3, [r7, #8]
 800082c:	4b29      	ldr	r3, [pc, #164]	; (80008d4 <SystemClock_Config+0xd0>)
 800082e:	6c1b      	ldr	r3, [r3, #64]	; 0x40
 8000830:	4a28      	ldr	r2, [pc, #160]	; (80008d4 <SystemClock_Config+0xd0>)
 8000832:	f043 5380 	orr.w	r3, r3, #268435456	; 0x10000000
 8000836:	6413      	str	r3, [r2, #64]	; 0x40
 8000838:	4b26      	ldr	r3, [pc, #152]	; (80008d4 <SystemClock_Config+0xd0>)
 800083a:	6c1b      	ldr	r3, [r3, #64]	; 0x40
 800083c:	f003 5380 	and.w	r3, r3, #268435456	; 0x10000000
 8000840:	60bb      	str	r3, [r7, #8]
 8000842:	68bb      	ldr	r3, [r7, #8]
  __HAL_PWR_VOLTAGESCALING_CONFIG(PWR_REGULATOR_VOLTAGE_SCALE3);
 8000844:	2300      	movs	r3, #0
 8000846:	607b      	str	r3, [r7, #4]
 8000848:	4b23      	ldr	r3, [pc, #140]	; (80008d8 <SystemClock_Config+0xd4>)
 800084a:	681b      	ldr	r3, [r3, #0]
 800084c:	f423 4340 	bic.w	r3, r3, #49152	; 0xc000
 8000850:	4a21      	ldr	r2, [pc, #132]	; (80008d8 <SystemClock_Config+0xd4>)
 8000852:	f443 4380 	orr.w	r3, r3, #16384	; 0x4000
 8000856:	6013      	str	r3, [r2, #0]
 8000858:	4b1f      	ldr	r3, [pc, #124]	; (80008d8 <SystemClock_Config+0xd4>)
 800085a:	681b      	ldr	r3, [r3, #0]
 800085c:	f403 4340 	and.w	r3, r3, #49152	; 0xc000
 8000860:	607b      	str	r3, [r7, #4]
 8000862:	687b      	ldr	r3, [r7, #4]

  /** Initializes the RCC Oscillators according to the specified parameters
  * in the RCC_OscInitTypeDef structure.
  */
  RCC_OscInitStruct.OscillatorType = RCC_OSCILLATORTYPE_HSI;
 8000864:	2302      	movs	r3, #2
 8000866:	623b      	str	r3, [r7, #32]
  RCC_OscInitStruct.HSIState = RCC_HSI_ON;
 8000868:	2301      	movs	r3, #1
 800086a:	62fb      	str	r3, [r7, #44]	; 0x2c
  RCC_OscInitStruct.HSICalibrationValue = RCC_HSICALIBRATION_DEFAULT;
 800086c:	2310      	movs	r3, #16
 800086e:	633b      	str	r3, [r7, #48]	; 0x30
  RCC_OscInitStruct.PLL.PLLState = RCC_PLL_ON;
 8000870:	2302      	movs	r3, #2
 8000872:	63bb      	str	r3, [r7, #56]	; 0x38
  RCC_OscInitStruct.PLL.PLLSource = RCC_PLLSOURCE_HSI;
 8000874:	2300      	movs	r3, #0
 8000876:	63fb      	str	r3, [r7, #60]	; 0x3c
  RCC_OscInitStruct.PLL.PLLM = 8;
 8000878:	2308      	movs	r3, #8
 800087a:	643b      	str	r3, [r7, #64]	; 0x40
  RCC_OscInitStruct.PLL.PLLN = 96;
 800087c:	2360      	movs	r3, #96	; 0x60
 800087e:	647b      	str	r3, [r7, #68]	; 0x44
  RCC_OscInitStruct.PLL.PLLP = RCC_PLLP_DIV2;
 8000880:	2302      	movs	r3, #2
 8000882:	64bb      	str	r3, [r7, #72]	; 0x48
  RCC_OscInitStruct.PLL.PLLQ = 7;
 8000884:	2307      	movs	r3, #7
 8000886:	64fb      	str	r3, [r7, #76]	; 0x4c
  if (HAL_RCC_OscConfig(&RCC_OscInitStruct) != HAL_OK)
 8000888:	f107 0320 	add.w	r3, r7, #32
 800088c:	4618      	mov	r0, r3
 800088e:	f000 fc97 	bl	80011c0 <HAL_RCC_OscConfig>
 8000892:	4603      	mov	r3, r0
 8000894:	2b00      	cmp	r3, #0
 8000896:	d001      	beq.n	800089c <SystemClock_Config+0x98>
  {
    Error_Handler();
 8000898:	f000 f8a4 	bl	80009e4 <Error_Handler>
  }

  /** Initializes the CPU, AHB and APB buses clocks
  */
  RCC_ClkInitStruct.ClockType = RCC_CLOCKTYPE_HCLK|RCC_CLOCKTYPE_SYSCLK
 800089c:	230f      	movs	r3, #15
 800089e:	60fb      	str	r3, [r7, #12]
                              |RCC_CLOCKTYPE_PCLK1|RCC_CLOCKTYPE_PCLK2;
  RCC_ClkInitStruct.SYSCLKSource = RCC_SYSCLKSOURCE_PLLCLK;
 80008a0:	2302      	movs	r3, #2
 80008a2:	613b      	str	r3, [r7, #16]
  RCC_ClkInitStruct.AHBCLKDivider = RCC_SYSCLK_DIV2;
 80008a4:	2380      	movs	r3, #128	; 0x80
 80008a6:	617b      	str	r3, [r7, #20]
  RCC_ClkInitStruct.APB1CLKDivider = RCC_HCLK_DIV2;
 80008a8:	f44f 5380 	mov.w	r3, #4096	; 0x1000
 80008ac:	61bb      	str	r3, [r7, #24]
  RCC_ClkInitStruct.APB2CLKDivider = RCC_HCLK_DIV4;
 80008ae:	f44f 53a0 	mov.w	r3, #5120	; 0x1400
 80008b2:	61fb      	str	r3, [r7, #28]

  if (HAL_RCC_ClockConfig(&RCC_ClkInitStruct, FLASH_LATENCY_1) != HAL_OK)
 80008b4:	f107 030c 	add.w	r3, r7, #12
 80008b8:	2101      	movs	r1, #1
 80008ba:	4618      	mov	r0, r3
 80008bc:	f000 fef8 	bl	80016b0 <HAL_RCC_ClockConfig>
 80008c0:	4603      	mov	r3, r0
 80008c2:	2b00      	cmp	r3, #0
 80008c4:	d001      	beq.n	80008ca <SystemClock_Config+0xc6>
  {
    Error_Handler();
 80008c6:	f000 f88d 	bl	80009e4 <Error_Handler>
  }
}
 80008ca:	bf00      	nop
 80008cc:	3750      	adds	r7, #80	; 0x50
 80008ce:	46bd      	mov	sp, r7
 80008d0:	bd80      	pop	{r7, pc}
 80008d2:	bf00      	nop
 80008d4:	40023800 	.word	0x40023800
 80008d8:	40007000 	.word	0x40007000

080008dc <MX_GPIO_Init>:
  * @brief GPIO Initialization Function
  * @param None
  * @retval None
  */
static void MX_GPIO_Init(void)
{
 80008dc:	b580      	push	{r7, lr}
 80008de:	b08a      	sub	sp, #40	; 0x28
 80008e0:	af00      	add	r7, sp, #0
  GPIO_InitTypeDef GPIO_InitStruct = {0};
 80008e2:	f107 0314 	add.w	r3, r7, #20
 80008e6:	2200      	movs	r2, #0
 80008e8:	601a      	str	r2, [r3, #0]
 80008ea:	605a      	str	r2, [r3, #4]
 80008ec:	609a      	str	r2, [r3, #8]
 80008ee:	60da      	str	r2, [r3, #12]
 80008f0:	611a      	str	r2, [r3, #16]

  /* GPIO Ports Clock Enable */
  __HAL_RCC_GPIOH_CLK_ENABLE();
 80008f2:	2300      	movs	r3, #0
 80008f4:	613b      	str	r3, [r7, #16]
 80008f6:	4b37      	ldr	r3, [pc, #220]	; (80009d4 <MX_GPIO_Init+0xf8>)
 80008f8:	6b1b      	ldr	r3, [r3, #48]	; 0x30
 80008fa:	4a36      	ldr	r2, [pc, #216]	; (80009d4 <MX_GPIO_Init+0xf8>)
 80008fc:	f043 0380 	orr.w	r3, r3, #128	; 0x80
 8000900:	6313      	str	r3, [r2, #48]	; 0x30
 8000902:	4b34      	ldr	r3, [pc, #208]	; (80009d4 <MX_GPIO_Init+0xf8>)
 8000904:	6b1b      	ldr	r3, [r3, #48]	; 0x30
 8000906:	f003 0380 	and.w	r3, r3, #128	; 0x80
 800090a:	613b      	str	r3, [r7, #16]
 800090c:	693b      	ldr	r3, [r7, #16]
  __HAL_RCC_GPIOA_CLK_ENABLE();
 800090e:	2300      	movs	r3, #0
 8000910:	60fb      	str	r3, [r7, #12]
 8000912:	4b30      	ldr	r3, [pc, #192]	; (80009d4 <MX_GPIO_Init+0xf8>)
 8000914:	6b1b      	ldr	r3, [r3, #48]	; 0x30
 8000916:	4a2f      	ldr	r2, [pc, #188]	; (80009d4 <MX_GPIO_Init+0xf8>)
 8000918:	f043 0301 	orr.w	r3, r3, #1
 800091c:	6313      	str	r3, [r2, #48]	; 0x30
 800091e:	4b2d      	ldr	r3, [pc, #180]	; (80009d4 <MX_GPIO_Init+0xf8>)
 8000920:	6b1b      	ldr	r3, [r3, #48]	; 0x30
 8000922:	f003 0301 	and.w	r3, r3, #1
 8000926:	60fb      	str	r3, [r7, #12]
 8000928:	68fb      	ldr	r3, [r7, #12]
  __HAL_RCC_GPIOD_CLK_ENABLE();
 800092a:	2300      	movs	r3, #0
 800092c:	60bb      	str	r3, [r7, #8]
 800092e:	4b29      	ldr	r3, [pc, #164]	; (80009d4 <MX_GPIO_Init+0xf8>)
 8000930:	6b1b      	ldr	r3, [r3, #48]	; 0x30
 8000932:	4a28      	ldr	r2, [pc, #160]	; (80009d4 <MX_GPIO_Init+0xf8>)
 8000934:	f043 0308 	orr.w	r3, r3, #8
 8000938:	6313      	str	r3, [r2, #48]	; 0x30
 800093a:	4b26      	ldr	r3, [pc, #152]	; (80009d4 <MX_GPIO_Init+0xf8>)
 800093c:	6b1b      	ldr	r3, [r3, #48]	; 0x30
 800093e:	f003 0308 	and.w	r3, r3, #8
 8000942:	60bb      	str	r3, [r7, #8]
 8000944:	68bb      	ldr	r3, [r7, #8]
  __HAL_RCC_GPIOG_CLK_ENABLE();
 8000946:	2300      	movs	r3, #0
 8000948:	607b      	str	r3, [r7, #4]
 800094a:	4b22      	ldr	r3, [pc, #136]	; (80009d4 <MX_GPIO_Init+0xf8>)
 800094c:	6b1b      	ldr	r3, [r3, #48]	; 0x30
 800094e:	4a21      	ldr	r2, [pc, #132]	; (80009d4 <MX_GPIO_Init+0xf8>)
 8000950:	f043 0340 	orr.w	r3, r3, #64	; 0x40
 8000954:	6313      	str	r3, [r2, #48]	; 0x30
 8000956:	4b1f      	ldr	r3, [pc, #124]	; (80009d4 <MX_GPIO_Init+0xf8>)
 8000958:	6b1b      	ldr	r3, [r3, #48]	; 0x30
 800095a:	f003 0340 	and.w	r3, r3, #64	; 0x40
 800095e:	607b      	str	r3, [r7, #4]
 8000960:	687b      	ldr	r3, [r7, #4]

  /*Configure GPIO pin Output Level */
  HAL_GPIO_WritePin(GPIOD, LED_0_Pin|LED_1_Pin, GPIO_PIN_RESET);
 8000962:	2200      	movs	r2, #0
 8000964:	21c0      	movs	r1, #192	; 0xc0
 8000966:	481c      	ldr	r0, [pc, #112]	; (80009d8 <MX_GPIO_Init+0xfc>)
 8000968:	f000 fc10 	bl	800118c <HAL_GPIO_WritePin>

  /*Configure GPIO pin Output Level */
  HAL_GPIO_WritePin(GPIOG, LED_2_Pin|LED_3_Pin|LED_4_Pin|LED_5_Pin, GPIO_PIN_RESET);
 800096c:	2200      	movs	r2, #0
 800096e:	f44f 51f0 	mov.w	r1, #7680	; 0x1e00
 8000972:	481a      	ldr	r0, [pc, #104]	; (80009dc <MX_GPIO_Init+0x100>)
 8000974:	f000 fc0a 	bl	800118c <HAL_GPIO_WritePin>

  /*Configure GPIO pin : User_Button_Pin */
  GPIO_InitStruct.Pin = User_Button_Pin;
 8000978:	2301      	movs	r3, #1
 800097a:	617b      	str	r3, [r7, #20]
  GPIO_InitStruct.Mode = GPIO_MODE_INPUT;
 800097c:	2300      	movs	r3, #0
 800097e:	61bb      	str	r3, [r7, #24]
  GPIO_InitStruct.Pull = GPIO_NOPULL;
 8000980:	2300      	movs	r3, #0
 8000982:	61fb      	str	r3, [r7, #28]
  HAL_GPIO_Init(User_Button_GPIO_Port, &GPIO_InitStruct);
 8000984:	f107 0314 	add.w	r3, r7, #20
 8000988:	4619      	mov	r1, r3
 800098a:	4815      	ldr	r0, [pc, #84]	; (80009e0 <MX_GPIO_Init+0x104>)
 800098c:	f000 fa3a 	bl	8000e04 <HAL_GPIO_Init>

  /*Configure GPIO pins : LED_0_Pin LED_1_Pin */
  GPIO_InitStruct.Pin = LED_0_Pin|LED_1_Pin;
 8000990:	23c0      	movs	r3, #192	; 0xc0
 8000992:	617b      	str	r3, [r7, #20]
  GPIO_InitStruct.Mode = GPIO_MODE_OUTPUT_PP;
 8000994:	2301      	movs	r3, #1
 8000996:	61bb      	str	r3, [r7, #24]
  GPIO_InitStruct.Pull = GPIO_NOPULL;
 8000998:	2300      	movs	r3, #0
 800099a:	61fb      	str	r3, [r7, #28]
  GPIO_InitStruct.Speed = GPIO_SPEED_FREQ_LOW;
 800099c:	2300      	movs	r3, #0
 800099e:	623b      	str	r3, [r7, #32]
  HAL_GPIO_Init(GPIOD, &GPIO_InitStruct);
 80009a0:	f107 0314 	add.w	r3, r7, #20
 80009a4:	4619      	mov	r1, r3
 80009a6:	480c      	ldr	r0, [pc, #48]	; (80009d8 <MX_GPIO_Init+0xfc>)
 80009a8:	f000 fa2c 	bl	8000e04 <HAL_GPIO_Init>

  /*Configure GPIO pins : LED_2_Pin LED_3_Pin LED_4_Pin LED_5_Pin */
  GPIO_InitStruct.Pin = LED_2_Pin|LED_3_Pin|LED_4_Pin|LED_5_Pin;
 80009ac:	f44f 53f0 	mov.w	r3, #7680	; 0x1e00
 80009b0:	617b      	str	r3, [r7, #20]
  GPIO_InitStruct.Mode = GPIO_MODE_OUTPUT_PP;
 80009b2:	2301      	movs	r3, #1
 80009b4:	61bb      	str	r3, [r7, #24]
  GPIO_InitStruct.Pull = GPIO_NOPULL;
 80009b6:	2300      	movs	r3, #0
 80009b8:	61fb      	str	r3, [r7, #28]
  GPIO_InitStruct.Speed = GPIO_SPEED_FREQ_LOW;
 80009ba:	2300      	movs	r3, #0
 80009bc:	623b      	str	r3, [r7, #32]
  HAL_GPIO_Init(GPIOG, &GPIO_InitStruct);
 80009be:	f107 0314 	add.w	r3, r7, #20
 80009c2:	4619      	mov	r1, r3
 80009c4:	4805      	ldr	r0, [pc, #20]	; (80009dc <MX_GPIO_Init+0x100>)
 80009c6:	f000 fa1d 	bl	8000e04 <HAL_GPIO_Init>

}
 80009ca:	bf00      	nop
 80009cc:	3728      	adds	r7, #40	; 0x28
 80009ce:	46bd      	mov	sp, r7
 80009d0:	bd80      	pop	{r7, pc}
 80009d2:	bf00      	nop
 80009d4:	40023800 	.word	0x40023800
 80009d8:	40020c00 	.word	0x40020c00
 80009dc:	40021800 	.word	0x40021800
 80009e0:	40020000 	.word	0x40020000

080009e4 <Error_Handler>:
/**
  * @brief  This function is executed in case of error occurrence.
  * @retval None
  */
void Error_Handler(void)
{
 80009e4:	b480      	push	{r7}
 80009e6:	af00      	add	r7, sp, #0
  \details Disables IRQ interrupts by setting the I-bit in the CPSR.
           Can only be executed in Privileged modes.
 */
__STATIC_FORCEINLINE void __disable_irq(void)
{
  __ASM volatile ("cpsid i" : : : "memory");
 80009e8:	b672      	cpsid	i
}
 80009ea:	bf00      	nop
  /* USER CODE BEGIN Error_Handler_Debug */
  /* User can add his own implementation to report the HAL error return state */
  __disable_irq();
  while (1)
 80009ec:	e7fe      	b.n	80009ec <Error_Handler+0x8>
	...

080009f0 <HAL_MspInit>:
/* USER CODE END 0 */
/**
  * Initializes the Global MSP.
  */
void HAL_MspInit(void)
{
 80009f0:	b580      	push	{r7, lr}
 80009f2:	b082      	sub	sp, #8
 80009f4:	af00      	add	r7, sp, #0
  /* USER CODE BEGIN MspInit 0 */

  /* USER CODE END MspInit 0 */

  __HAL_RCC_SYSCFG_CLK_ENABLE();
 80009f6:	2300      	movs	r3, #0
 80009f8:	607b      	str	r3, [r7, #4]
 80009fa:	4b10      	ldr	r3, [pc, #64]	; (8000a3c <HAL_MspInit+0x4c>)
 80009fc:	6c5b      	ldr	r3, [r3, #68]	; 0x44
 80009fe:	4a0f      	ldr	r2, [pc, #60]	; (8000a3c <HAL_MspInit+0x4c>)
 8000a00:	f443 4380 	orr.w	r3, r3, #16384	; 0x4000
 8000a04:	6453      	str	r3, [r2, #68]	; 0x44
 8000a06:	4b0d      	ldr	r3, [pc, #52]	; (8000a3c <HAL_MspInit+0x4c>)
 8000a08:	6c5b      	ldr	r3, [r3, #68]	; 0x44
 8000a0a:	f403 4380 	and.w	r3, r3, #16384	; 0x4000
 8000a0e:	607b      	str	r3, [r7, #4]
 8000a10:	687b      	ldr	r3, [r7, #4]
  __HAL_RCC_PWR_CLK_ENABLE();
 8000a12:	2300      	movs	r3, #0
 8000a14:	603b      	str	r3, [r7, #0]
 8000a16:	4b09      	ldr	r3, [pc, #36]	; (8000a3c <HAL_MspInit+0x4c>)
 8000a18:	6c1b      	ldr	r3, [r3, #64]	; 0x40
 8000a1a:	4a08      	ldr	r2, [pc, #32]	; (8000a3c <HAL_MspInit+0x4c>)
 8000a1c:	f043 5380 	orr.w	r3, r3, #268435456	; 0x10000000
 8000a20:	6413      	str	r3, [r2, #64]	; 0x40
 8000a22:	4b06      	ldr	r3, [pc, #24]	; (8000a3c <HAL_MspInit+0x4c>)
 8000a24:	6c1b      	ldr	r3, [r3, #64]	; 0x40
 8000a26:	f003 5380 	and.w	r3, r3, #268435456	; 0x10000000
 8000a2a:	603b      	str	r3, [r7, #0]
 8000a2c:	683b      	ldr	r3, [r7, #0]

  HAL_NVIC_SetPriorityGrouping(NVIC_PRIORITYGROUP_0);
 8000a2e:	2007      	movs	r0, #7
 8000a30:	f000 f9b4 	bl	8000d9c <HAL_NVIC_SetPriorityGrouping>
  /* System interrupt init*/

  /* USER CODE BEGIN MspInit 1 */

  /* USER CODE END MspInit 1 */
}
 8000a34:	bf00      	nop
 8000a36:	3708      	adds	r7, #8
 8000a38:	46bd      	mov	sp, r7
 8000a3a:	bd80      	pop	{r7, pc}
 8000a3c:	40023800 	.word	0x40023800

08000a40 <NMI_Handler>:
/******************************************************************************/
/**
  * @brief This function handles Non maskable interrupt.
  */
void NMI_Handler(void)
{
 8000a40:	b480      	push	{r7}
 8000a42:	af00      	add	r7, sp, #0
  /* USER CODE BEGIN NonMaskableInt_IRQn 0 */

  /* USER CODE END NonMaskableInt_IRQn 0 */
  /* USER CODE BEGIN NonMaskableInt_IRQn 1 */
  while (1)
 8000a44:	e7fe      	b.n	8000a44 <NMI_Handler+0x4>

08000a46 <HardFault_Handler>:

/**
  * @brief This function handles Hard fault interrupt.
  */
void HardFault_Handler(void)
{
 8000a46:	b480      	push	{r7}
 8000a48:	af00      	add	r7, sp, #0
  /* USER CODE BEGIN HardFault_IRQn 0 */

  /* USER CODE END HardFault_IRQn 0 */
  while (1)
 8000a4a:	e7fe      	b.n	8000a4a <HardFault_Handler+0x4>

08000a4c <MemManage_Handler>:

/**
  * @brief This function handles Memory management fault.
  */
void MemManage_Handler(void)
{
 8000a4c:	b480      	push	{r7}
 8000a4e:	af00      	add	r7, sp, #0
  /* USER CODE BEGIN MemoryManagement_IRQn 0 */

  /* USER CODE END MemoryManagement_IRQn 0 */
  while (1)
 8000a50:	e7fe      	b.n	8000a50 <MemManage_Handler+0x4>

08000a52 <BusFault_Handler>:

/**
  * @brief This function handles Pre-fetch fault, memory access fault.
  */
void BusFault_Handler(void)
{
 8000a52:	b480      	push	{r7}
 8000a54:	af00      	add	r7, sp, #0
  /* USER CODE BEGIN BusFault_IRQn 0 */

  /* USER CODE END BusFault_IRQn 0 */
  while (1)
 8000a56:	e7fe      	b.n	8000a56 <BusFault_Handler+0x4>

08000a58 <UsageFault_Handler>:

/**
  * @brief This function handles Undefined instruction or illegal state.
  */
void UsageFault_Handler(void)
{
 8000a58:	b480      	push	{r7}
 8000a5a:	af00      	add	r7, sp, #0
  /* USER CODE BEGIN UsageFault_IRQn 0 */

  /* USER CODE END UsageFault_IRQn 0 */
  while (1)
 8000a5c:	e7fe      	b.n	8000a5c <UsageFault_Handler+0x4>

08000a5e <SVC_Handler>:

/**
  * @brief This function handles System service call via SWI instruction.
  */
void SVC_Handler(void)
{
 8000a5e:	b480      	push	{r7}
 8000a60:	af00      	add	r7, sp, #0

  /* USER CODE END SVCall_IRQn 0 */
  /* USER CODE BEGIN SVCall_IRQn 1 */

  /* USER CODE END SVCall_IRQn 1 */
}
 8000a62:	bf00      	nop
 8000a64:	46bd      	mov	sp, r7
 8000a66:	f85d 7b04 	ldr.w	r7, [sp], #4
 8000a6a:	4770      	bx	lr

08000a6c <DebugMon_Handler>:

/**
  * @brief This function handles Debug monitor.
  */
void DebugMon_Handler(void)
{
 8000a6c:	b480      	push	{r7}
 8000a6e:	af00      	add	r7, sp, #0

  /* USER CODE END DebugMonitor_IRQn 0 */
  /* USER CODE BEGIN DebugMonitor_IRQn 1 */

  /* USER CODE END DebugMonitor_IRQn 1 */
}
 8000a70:	bf00      	nop
 8000a72:	46bd      	mov	sp, r7
 8000a74:	f85d 7b04 	ldr.w	r7, [sp], #4
 8000a78:	4770      	bx	lr

08000a7a <PendSV_Handler>:

/**
  * @brief This function handles Pendable request for system service.
  */
void PendSV_Handler(void)
{
 8000a7a:	b480      	push	{r7}
 8000a7c:	af00      	add	r7, sp, #0

  /* USER CODE END PendSV_IRQn 0 */
  /* USER CODE BEGIN PendSV_IRQn 1 */

  /* USER CODE END PendSV_IRQn 1 */
}
 8000a7e:	bf00      	nop
 8000a80:	46bd      	mov	sp, r7
 8000a82:	f85d 7b04 	ldr.w	r7, [sp], #4
 8000a86:	4770      	bx	lr

08000a88 <SysTick_Handler>:

/**
  * @brief This function handles System tick timer.
  */
void SysTick_Handler(void)
{
 8000a88:	b580      	push	{r7, lr}
 8000a8a:	af00      	add	r7, sp, #0
  /* USER CODE BEGIN SysTick_IRQn 0 */

  /* USER CODE END SysTick_IRQn 0 */
  HAL_IncTick();
 8000a8c:	f000 f890 	bl	8000bb0 <HAL_IncTick>
  /* USER CODE BEGIN SysTick_IRQn 1 */

  /* USER CODE END SysTick_IRQn 1 */
}
 8000a90:	bf00      	nop
 8000a92:	bd80      	pop	{r7, pc}

08000a94 <SystemInit>:
  *         configuration.
  * @param  None
  * @retval None
  */
void SystemInit(void)
{
 8000a94:	b480      	push	{r7}
 8000a96:	af00      	add	r7, sp, #0
  /* FPU settings ------------------------------------------------------------*/
  #if (__FPU_PRESENT == 1) && (__FPU_USED == 1)
    SCB->CPACR |= ((3UL << 10*2)|(3UL << 11*2));  /* set CP10 and CP11 Full Access */
 8000a98:	4b06      	ldr	r3, [pc, #24]	; (8000ab4 <SystemInit+0x20>)
 8000a9a:	f8d3 3088 	ldr.w	r3, [r3, #136]	; 0x88
 8000a9e:	4a05      	ldr	r2, [pc, #20]	; (8000ab4 <SystemInit+0x20>)
 8000aa0:	f443 0370 	orr.w	r3, r3, #15728640	; 0xf00000
 8000aa4:	f8c2 3088 	str.w	r3, [r2, #136]	; 0x88

  /* Configure the Vector Table location -------------------------------------*/
#if defined(USER_VECT_TAB_ADDRESS)
  SCB->VTOR = VECT_TAB_BASE_ADDRESS | VECT_TAB_OFFSET; /* Vector Table Relocation in Internal SRAM */
#endif /* USER_VECT_TAB_ADDRESS */
}
 8000aa8:	bf00      	nop
 8000aaa:	46bd      	mov	sp, r7
 8000aac:	f85d 7b04 	ldr.w	r7, [sp], #4
 8000ab0:	4770      	bx	lr
 8000ab2:	bf00      	nop
 8000ab4:	e000ed00 	.word	0xe000ed00

08000ab8 <Reset_Handler>:

    .section  .text.Reset_Handler
  .weak  Reset_Handler
  .type  Reset_Handler, %function
Reset_Handler: 
  ldr   sp, =_estack       /* set stack pointer */
 8000ab8:	f8df d034 	ldr.w	sp, [pc, #52]	; 8000af0 <LoopFillZerobss+0x12>
 
/* Copy the data segment initializers from flash to SRAM */  
  ldr r0, =_sdata
 8000abc:	480d      	ldr	r0, [pc, #52]	; (8000af4 <LoopFillZerobss+0x16>)
  ldr r1, =_edata
 8000abe:	490e      	ldr	r1, [pc, #56]	; (8000af8 <LoopFillZerobss+0x1a>)
  ldr r2, =_sidata
 8000ac0:	4a0e      	ldr	r2, [pc, #56]	; (8000afc <LoopFillZerobss+0x1e>)
  movs r3, #0
 8000ac2:	2300      	movs	r3, #0
  b LoopCopyDataInit
 8000ac4:	e002      	b.n	8000acc <LoopCopyDataInit>

08000ac6 <CopyDataInit>:

CopyDataInit:
  ldr r4, [r2, r3]
 8000ac6:	58d4      	ldr	r4, [r2, r3]
  str r4, [r0, r3]
 8000ac8:	50c4      	str	r4, [r0, r3]
  adds r3, r3, #4
 8000aca:	3304      	adds	r3, #4

08000acc <LoopCopyDataInit>:

LoopCopyDataInit:
  adds r4, r0, r3
 8000acc:	18c4      	adds	r4, r0, r3
  cmp r4, r1
 8000ace:	428c      	cmp	r4, r1
  bcc CopyDataInit
 8000ad0:	d3f9      	bcc.n	8000ac6 <CopyDataInit>
  
/* Zero fill the bss segment. */
  ldr r2, =_sbss
 8000ad2:	4a0b      	ldr	r2, [pc, #44]	; (8000b00 <LoopFillZerobss+0x22>)
  ldr r4, =_ebss
 8000ad4:	4c0b      	ldr	r4, [pc, #44]	; (8000b04 <LoopFillZerobss+0x26>)
  movs r3, #0
 8000ad6:	2300      	movs	r3, #0
  b LoopFillZerobss
 8000ad8:	e001      	b.n	8000ade <LoopFillZerobss>

08000ada <FillZerobss>:

FillZerobss:
  str  r3, [r2]
 8000ada:	6013      	str	r3, [r2, #0]
  adds r2, r2, #4
 8000adc:	3204      	adds	r2, #4

08000ade <LoopFillZerobss>:

LoopFillZerobss:
  cmp r2, r4
 8000ade:	42a2      	cmp	r2, r4
  bcc FillZerobss
 8000ae0:	d3fb      	bcc.n	8000ada <FillZerobss>

/* Call the clock system initialization function.*/
  bl  SystemInit   
 8000ae2:	f7ff ffd7 	bl	8000a94 <SystemInit>
/* Call static constructors */
    bl __libc_init_array
 8000ae6:	f000 ffcf 	bl	8001a88 <__libc_init_array>
/* Call the application's entry point.*/
  bl  main
 8000aea:	f7ff fd01 	bl	80004f0 <main>
  bx  lr    
 8000aee:	4770      	bx	lr
  ldr   sp, =_estack       /* set stack pointer */
 8000af0:	20030000 	.word	0x20030000
  ldr r0, =_sdata
 8000af4:	20000000 	.word	0x20000000
  ldr r1, =_edata
 8000af8:	2000000c 	.word	0x2000000c
  ldr r2, =_sidata
 8000afc:	08001b18 	.word	0x08001b18
  ldr r2, =_sbss
 8000b00:	2000000c 	.word	0x2000000c
  ldr r4, =_ebss
 8000b04:	20000030 	.word	0x20000030

08000b08 <ADC_IRQHandler>:
 * @retval None       
*/
    .section  .text.Default_Handler,"ax",%progbits
Default_Handler:
Infinite_Loop:
  b  Infinite_Loop
 8000b08:	e7fe      	b.n	8000b08 <ADC_IRQHandler>
	...

08000b0c <HAL_Init>:
  *         need to ensure that the SysTick time base is always set to 1 millisecond
  *         to have correct HAL operation.
  * @retval HAL status
  */
HAL_StatusTypeDef HAL_Init(void)
{
 8000b0c:	b580      	push	{r7, lr}
 8000b0e:	af00      	add	r7, sp, #0
  /* Configure Flash prefetch, Instruction cache, Data cache */ 
#if (INSTRUCTION_CACHE_ENABLE != 0U)
  __HAL_FLASH_INSTRUCTION_CACHE_ENABLE();
 8000b10:	4b0e      	ldr	r3, [pc, #56]	; (8000b4c <HAL_Init+0x40>)
 8000b12:	681b      	ldr	r3, [r3, #0]
 8000b14:	4a0d      	ldr	r2, [pc, #52]	; (8000b4c <HAL_Init+0x40>)
 8000b16:	f443 7300 	orr.w	r3, r3, #512	; 0x200
 8000b1a:	6013      	str	r3, [r2, #0]
#endif /* INSTRUCTION_CACHE_ENABLE */

#if (DATA_CACHE_ENABLE != 0U)
  __HAL_FLASH_DATA_CACHE_ENABLE();
 8000b1c:	4b0b      	ldr	r3, [pc, #44]	; (8000b4c <HAL_Init+0x40>)
 8000b1e:	681b      	ldr	r3, [r3, #0]
 8000b20:	4a0a      	ldr	r2, [pc, #40]	; (8000b4c <HAL_Init+0x40>)
 8000b22:	f443 6380 	orr.w	r3, r3, #1024	; 0x400
 8000b26:	6013      	str	r3, [r2, #0]
#endif /* DATA_CACHE_ENABLE */

#if (PREFETCH_ENABLE != 0U)
  __HAL_FLASH_PREFETCH_BUFFER_ENABLE();
 8000b28:	4b08      	ldr	r3, [pc, #32]	; (8000b4c <HAL_Init+0x40>)
 8000b2a:	681b      	ldr	r3, [r3, #0]
 8000b2c:	4a07      	ldr	r2, [pc, #28]	; (8000b4c <HAL_Init+0x40>)
 8000b2e:	f443 7380 	orr.w	r3, r3, #256	; 0x100
 8000b32:	6013      	str	r3, [r2, #0]
#endif /* PREFETCH_ENABLE */

  /* Set Interrupt Group Priority */
  HAL_NVIC_SetPriorityGrouping(NVIC_PRIORITYGROUP_4);
 8000b34:	2003      	movs	r0, #3
 8000b36:	f000 f931 	bl	8000d9c <HAL_NVIC_SetPriorityGrouping>

  /* Use systick as time base source and configure 1ms tick (default clock after Reset is HSI) */
  HAL_InitTick(TICK_INT_PRIORITY);
 8000b3a:	2000      	movs	r0, #0
 8000b3c:	f000 f808 	bl	8000b50 <HAL_InitTick>

  /* Init the low level hardware */
  HAL_MspInit();
 8000b40:	f7ff ff56 	bl	80009f0 <HAL_MspInit>

  /* Return function status */
  return HAL_OK;
 8000b44:	2300      	movs	r3, #0
}
 8000b46:	4618      	mov	r0, r3
 8000b48:	bd80      	pop	{r7, pc}
 8000b4a:	bf00      	nop
 8000b4c:	40023c00 	.word	0x40023c00

08000b50 <HAL_InitTick>:
  *       implementation  in user file.
  * @param TickPriority Tick interrupt priority.
  * @retval HAL status
  */
__weak HAL_StatusTypeDef HAL_InitTick(uint32_t TickPriority)
{
 8000b50:	b580      	push	{r7, lr}
 8000b52:	b082      	sub	sp, #8
 8000b54:	af00      	add	r7, sp, #0
 8000b56:	6078      	str	r0, [r7, #4]
  /* Configure the SysTick to have interrupt in 1ms time basis*/
  if (HAL_SYSTICK_Config(SystemCoreClock / (1000U / uwTickFreq)) > 0U)
 8000b58:	4b12      	ldr	r3, [pc, #72]	; (8000ba4 <HAL_InitTick+0x54>)
 8000b5a:	681a      	ldr	r2, [r3, #0]
 8000b5c:	4b12      	ldr	r3, [pc, #72]	; (8000ba8 <HAL_InitTick+0x58>)
 8000b5e:	781b      	ldrb	r3, [r3, #0]
 8000b60:	4619      	mov	r1, r3
 8000b62:	f44f 737a 	mov.w	r3, #1000	; 0x3e8
 8000b66:	fbb3 f3f1 	udiv	r3, r3, r1
 8000b6a:	fbb2 f3f3 	udiv	r3, r2, r3
 8000b6e:	4618      	mov	r0, r3
 8000b70:	f000 f93b 	bl	8000dea <HAL_SYSTICK_Config>
 8000b74:	4603      	mov	r3, r0
 8000b76:	2b00      	cmp	r3, #0
 8000b78:	d001      	beq.n	8000b7e <HAL_InitTick+0x2e>
  {
    return HAL_ERROR;
 8000b7a:	2301      	movs	r3, #1
 8000b7c:	e00e      	b.n	8000b9c <HAL_InitTick+0x4c>
  }

  /* Configure the SysTick IRQ priority */
  if (TickPriority < (1UL << __NVIC_PRIO_BITS))
 8000b7e:	687b      	ldr	r3, [r7, #4]
 8000b80:	2b0f      	cmp	r3, #15
 8000b82:	d80a      	bhi.n	8000b9a <HAL_InitTick+0x4a>
  {
    HAL_NVIC_SetPriority(SysTick_IRQn, TickPriority, 0U);
 8000b84:	2200      	movs	r2, #0
 8000b86:	6879      	ldr	r1, [r7, #4]
 8000b88:	f04f 30ff 	mov.w	r0, #4294967295
 8000b8c:	f000 f911 	bl	8000db2 <HAL_NVIC_SetPriority>
    uwTickPrio = TickPriority;
 8000b90:	4a06      	ldr	r2, [pc, #24]	; (8000bac <HAL_InitTick+0x5c>)
 8000b92:	687b      	ldr	r3, [r7, #4]
 8000b94:	6013      	str	r3, [r2, #0]
  {
    return HAL_ERROR;
  }

  /* Return function status */
  return HAL_OK;
 8000b96:	2300      	movs	r3, #0
 8000b98:	e000      	b.n	8000b9c <HAL_InitTick+0x4c>
    return HAL_ERROR;
 8000b9a:	2301      	movs	r3, #1
}
 8000b9c:	4618      	mov	r0, r3
 8000b9e:	3708      	adds	r7, #8
 8000ba0:	46bd      	mov	sp, r7
 8000ba2:	bd80      	pop	{r7, pc}
 8000ba4:	20000000 	.word	0x20000000
 8000ba8:	20000008 	.word	0x20000008
 8000bac:	20000004 	.word	0x20000004

08000bb0 <HAL_IncTick>:
 * @note This function is declared as __weak to be overwritten in case of other 
  *      implementations in user file.
  * @retval None
  */
__weak void HAL_IncTick(void)
{
 8000bb0:	b480      	push	{r7}
 8000bb2:	af00      	add	r7, sp, #0
  uwTick += uwTickFreq;
 8000bb4:	4b06      	ldr	r3, [pc, #24]	; (8000bd0 <HAL_IncTick+0x20>)
 8000bb6:	781b      	ldrb	r3, [r3, #0]
 8000bb8:	461a      	mov	r2, r3
 8000bba:	4b06      	ldr	r3, [pc, #24]	; (8000bd4 <HAL_IncTick+0x24>)
 8000bbc:	681b      	ldr	r3, [r3, #0]
 8000bbe:	4413      	add	r3, r2
 8000bc0:	4a04      	ldr	r2, [pc, #16]	; (8000bd4 <HAL_IncTick+0x24>)
 8000bc2:	6013      	str	r3, [r2, #0]
}
 8000bc4:	bf00      	nop
 8000bc6:	46bd      	mov	sp, r7
 8000bc8:	f85d 7b04 	ldr.w	r7, [sp], #4
 8000bcc:	4770      	bx	lr
 8000bce:	bf00      	nop
 8000bd0:	20000008 	.word	0x20000008
 8000bd4:	2000002c 	.word	0x2000002c

08000bd8 <HAL_GetTick>:
  * @note This function is declared as __weak to be overwritten in case of other 
  *       implementations in user file.
  * @retval tick value
  */
__weak uint32_t HAL_GetTick(void)
{
 8000bd8:	b480      	push	{r7}
 8000bda:	af00      	add	r7, sp, #0
  return uwTick;
 8000bdc:	4b03      	ldr	r3, [pc, #12]	; (8000bec <HAL_GetTick+0x14>)
 8000bde:	681b      	ldr	r3, [r3, #0]
}
 8000be0:	4618      	mov	r0, r3
 8000be2:	46bd      	mov	sp, r7
 8000be4:	f85d 7b04 	ldr.w	r7, [sp], #4
 8000be8:	4770      	bx	lr
 8000bea:	bf00      	nop
 8000bec:	2000002c 	.word	0x2000002c

08000bf0 <HAL_Delay>:
  *       implementations in user file.
  * @param Delay specifies the delay time length, in milliseconds.
  * @retval None
  */
__weak void HAL_Delay(uint32_t Delay)
{
 8000bf0:	b580      	push	{r7, lr}
 8000bf2:	b084      	sub	sp, #16
 8000bf4:	af00      	add	r7, sp, #0
 8000bf6:	6078      	str	r0, [r7, #4]
  uint32_t tickstart = HAL_GetTick();
 8000bf8:	f7ff ffee 	bl	8000bd8 <HAL_GetTick>
 8000bfc:	60b8      	str	r0, [r7, #8]
  uint32_t wait = Delay;
 8000bfe:	687b      	ldr	r3, [r7, #4]
 8000c00:	60fb      	str	r3, [r7, #12]

  /* Add a freq to guarantee minimum wait */
  if (wait < HAL_MAX_DELAY)
 8000c02:	68fb      	ldr	r3, [r7, #12]
 8000c04:	f1b3 3fff 	cmp.w	r3, #4294967295
 8000c08:	d005      	beq.n	8000c16 <HAL_Delay+0x26>
  {
    wait += (uint32_t)(uwTickFreq);
 8000c0a:	4b0a      	ldr	r3, [pc, #40]	; (8000c34 <HAL_Delay+0x44>)
 8000c0c:	781b      	ldrb	r3, [r3, #0]
 8000c0e:	461a      	mov	r2, r3
 8000c10:	68fb      	ldr	r3, [r7, #12]
 8000c12:	4413      	add	r3, r2
 8000c14:	60fb      	str	r3, [r7, #12]
  }

  while((HAL_GetTick() - tickstart) < wait)
 8000c16:	bf00      	nop
 8000c18:	f7ff ffde 	bl	8000bd8 <HAL_GetTick>
 8000c1c:	4602      	mov	r2, r0
 8000c1e:	68bb      	ldr	r3, [r7, #8]
 8000c20:	1ad3      	subs	r3, r2, r3
 8000c22:	68fa      	ldr	r2, [r7, #12]
 8000c24:	429a      	cmp	r2, r3
 8000c26:	d8f7      	bhi.n	8000c18 <HAL_Delay+0x28>
  {
  }
}
 8000c28:	bf00      	nop
 8000c2a:	bf00      	nop
 8000c2c:	3710      	adds	r7, #16
 8000c2e:	46bd      	mov	sp, r7
 8000c30:	bd80      	pop	{r7, pc}
 8000c32:	bf00      	nop
 8000c34:	20000008 	.word	0x20000008

08000c38 <__NVIC_SetPriorityGrouping>:
           In case of a conflict between priority grouping and available
           priority bits (__NVIC_PRIO_BITS), the smallest possible priority group is set.
  \param [in]      PriorityGroup  Priority grouping field.
 */
__STATIC_INLINE void __NVIC_SetPriorityGrouping(uint32_t PriorityGroup)
{
 8000c38:	b480      	push	{r7}
 8000c3a:	b085      	sub	sp, #20
 8000c3c:	af00      	add	r7, sp, #0
 8000c3e:	6078      	str	r0, [r7, #4]
  uint32_t reg_value;
  uint32_t PriorityGroupTmp = (PriorityGroup & (uint32_t)0x07UL);             /* only values 0..7 are used          */
 8000c40:	687b      	ldr	r3, [r7, #4]
 8000c42:	f003 0307 	and.w	r3, r3, #7
 8000c46:	60fb      	str	r3, [r7, #12]

  reg_value  =  SCB->AIRCR;                                                   /* read old register configuration    */
 8000c48:	4b0c      	ldr	r3, [pc, #48]	; (8000c7c <__NVIC_SetPriorityGrouping+0x44>)
 8000c4a:	68db      	ldr	r3, [r3, #12]
 8000c4c:	60bb      	str	r3, [r7, #8]
  reg_value &= ~((uint32_t)(SCB_AIRCR_VECTKEY_Msk | SCB_AIRCR_PRIGROUP_Msk)); /* clear bits to change               */
 8000c4e:	68ba      	ldr	r2, [r7, #8]
 8000c50:	f64f 03ff 	movw	r3, #63743	; 0xf8ff
 8000c54:	4013      	ands	r3, r2
 8000c56:	60bb      	str	r3, [r7, #8]
  reg_value  =  (reg_value                                   |
                ((uint32_t)0x5FAUL << SCB_AIRCR_VECTKEY_Pos) |
                (PriorityGroupTmp << SCB_AIRCR_PRIGROUP_Pos)  );              /* Insert write key and priority group */
 8000c58:	68fb      	ldr	r3, [r7, #12]
 8000c5a:	021a      	lsls	r2, r3, #8
                ((uint32_t)0x5FAUL << SCB_AIRCR_VECTKEY_Pos) |
 8000c5c:	68bb      	ldr	r3, [r7, #8]
 8000c5e:	4313      	orrs	r3, r2
  reg_value  =  (reg_value                                   |
 8000c60:	f043 63bf 	orr.w	r3, r3, #100139008	; 0x5f80000
 8000c64:	f443 3300 	orr.w	r3, r3, #131072	; 0x20000
 8000c68:	60bb      	str	r3, [r7, #8]
  SCB->AIRCR =  reg_value;
 8000c6a:	4a04      	ldr	r2, [pc, #16]	; (8000c7c <__NVIC_SetPriorityGrouping+0x44>)
 8000c6c:	68bb      	ldr	r3, [r7, #8]
 8000c6e:	60d3      	str	r3, [r2, #12]
}
 8000c70:	bf00      	nop
 8000c72:	3714      	adds	r7, #20
 8000c74:	46bd      	mov	sp, r7
 8000c76:	f85d 7b04 	ldr.w	r7, [sp], #4
 8000c7a:	4770      	bx	lr
 8000c7c:	e000ed00 	.word	0xe000ed00

08000c80 <__NVIC_GetPriorityGrouping>:
  \brief   Get Priority Grouping
  \details Reads the priority grouping field from the NVIC Interrupt Controller.
  \return                Priority grouping field (SCB->AIRCR [10:8] PRIGROUP field).
 */
__STATIC_INLINE uint32_t __NVIC_GetPriorityGrouping(void)
{
 8000c80:	b480      	push	{r7}
 8000c82:	af00      	add	r7, sp, #0
  return ((uint32_t)((SCB->AIRCR & SCB_AIRCR_PRIGROUP_Msk) >> SCB_AIRCR_PRIGROUP_Pos));
 8000c84:	4b04      	ldr	r3, [pc, #16]	; (8000c98 <__NVIC_GetPriorityGrouping+0x18>)
 8000c86:	68db      	ldr	r3, [r3, #12]
 8000c88:	0a1b      	lsrs	r3, r3, #8
 8000c8a:	f003 0307 	and.w	r3, r3, #7
}
 8000c8e:	4618      	mov	r0, r3
 8000c90:	46bd      	mov	sp, r7
 8000c92:	f85d 7b04 	ldr.w	r7, [sp], #4
 8000c96:	4770      	bx	lr
 8000c98:	e000ed00 	.word	0xe000ed00

08000c9c <__NVIC_SetPriority>:
  \param [in]      IRQn  Interrupt number.
  \param [in]  priority  Priority to set.
  \note    The priority cannot be set for every processor exception.
 */
__STATIC_INLINE void __NVIC_SetPriority(IRQn_Type IRQn, uint32_t priority)
{
 8000c9c:	b480      	push	{r7}
 8000c9e:	b083      	sub	sp, #12
 8000ca0:	af00      	add	r7, sp, #0
 8000ca2:	4603      	mov	r3, r0
 8000ca4:	6039      	str	r1, [r7, #0]
 8000ca6:	71fb      	strb	r3, [r7, #7]
  if ((int32_t)(IRQn) >= 0)
 8000ca8:	f997 3007 	ldrsb.w	r3, [r7, #7]
 8000cac:	2b00      	cmp	r3, #0
 8000cae:	db0a      	blt.n	8000cc6 <__NVIC_SetPriority+0x2a>
  {
    NVIC->IP[((uint32_t)IRQn)]               = (uint8_t)((priority << (8U - __NVIC_PRIO_BITS)) & (uint32_t)0xFFUL);
 8000cb0:	683b      	ldr	r3, [r7, #0]
 8000cb2:	b2da      	uxtb	r2, r3
 8000cb4:	490c      	ldr	r1, [pc, #48]	; (8000ce8 <__NVIC_SetPriority+0x4c>)
 8000cb6:	f997 3007 	ldrsb.w	r3, [r7, #7]
 8000cba:	0112      	lsls	r2, r2, #4
 8000cbc:	b2d2      	uxtb	r2, r2
 8000cbe:	440b      	add	r3, r1
 8000cc0:	f883 2300 	strb.w	r2, [r3, #768]	; 0x300
  }
  else
  {
    SCB->SHP[(((uint32_t)IRQn) & 0xFUL)-4UL] = (uint8_t)((priority << (8U - __NVIC_PRIO_BITS)) & (uint32_t)0xFFUL);
  }
}
 8000cc4:	e00a      	b.n	8000cdc <__NVIC_SetPriority+0x40>
    SCB->SHP[(((uint32_t)IRQn) & 0xFUL)-4UL] = (uint8_t)((priority << (8U - __NVIC_PRIO_BITS)) & (uint32_t)0xFFUL);
 8000cc6:	683b      	ldr	r3, [r7, #0]
 8000cc8:	b2da      	uxtb	r2, r3
 8000cca:	4908      	ldr	r1, [pc, #32]	; (8000cec <__NVIC_SetPriority+0x50>)
 8000ccc:	79fb      	ldrb	r3, [r7, #7]
 8000cce:	f003 030f 	and.w	r3, r3, #15
 8000cd2:	3b04      	subs	r3, #4
 8000cd4:	0112      	lsls	r2, r2, #4
 8000cd6:	b2d2      	uxtb	r2, r2
 8000cd8:	440b      	add	r3, r1
 8000cda:	761a      	strb	r2, [r3, #24]
}
 8000cdc:	bf00      	nop
 8000cde:	370c      	adds	r7, #12
 8000ce0:	46bd      	mov	sp, r7
 8000ce2:	f85d 7b04 	ldr.w	r7, [sp], #4
 8000ce6:	4770      	bx	lr
 8000ce8:	e000e100 	.word	0xe000e100
 8000cec:	e000ed00 	.word	0xe000ed00

08000cf0 <NVIC_EncodePriority>:
  \param [in]   PreemptPriority  Preemptive priority value (starting from 0).
  \param [in]       SubPriority  Subpriority value (starting from 0).
  \return                        Encoded priority. Value can be used in the function \ref NVIC_SetPriority().
 */
__STATIC_INLINE uint32_t NVIC_EncodePriority (uint32_t PriorityGroup, uint32_t PreemptPriority, uint32_t SubPriority)
{
 8000cf0:	b480      	push	{r7}
 8000cf2:	b089      	sub	sp, #36	; 0x24
 8000cf4:	af00      	add	r7, sp, #0
 8000cf6:	60f8      	str	r0, [r7, #12]
 8000cf8:	60b9      	str	r1, [r7, #8]
 8000cfa:	607a      	str	r2, [r7, #4]
  uint32_t PriorityGroupTmp = (PriorityGroup & (uint32_t)0x07UL);   /* only values 0..7 are used          */
 8000cfc:	68fb      	ldr	r3, [r7, #12]
 8000cfe:	f003 0307 	and.w	r3, r3, #7
 8000d02:	61fb      	str	r3, [r7, #28]
  uint32_t PreemptPriorityBits;
  uint32_t SubPriorityBits;

  PreemptPriorityBits = ((7UL - PriorityGroupTmp) > (uint32_t)(__NVIC_PRIO_BITS)) ? (uint32_t)(__NVIC_PRIO_BITS) : (uint32_t)(7UL - PriorityGroupTmp);
 8000d04:	69fb      	ldr	r3, [r7, #28]
 8000d06:	f1c3 0307 	rsb	r3, r3, #7
 8000d0a:	2b04      	cmp	r3, #4
 8000d0c:	bf28      	it	cs
 8000d0e:	2304      	movcs	r3, #4
 8000d10:	61bb      	str	r3, [r7, #24]
  SubPriorityBits     = ((PriorityGroupTmp + (uint32_t)(__NVIC_PRIO_BITS)) < (uint32_t)7UL) ? (uint32_t)0UL : (uint32_t)((PriorityGroupTmp - 7UL) + (uint32_t)(__NVIC_PRIO_BITS));
 8000d12:	69fb      	ldr	r3, [r7, #28]
 8000d14:	3304      	adds	r3, #4
 8000d16:	2b06      	cmp	r3, #6
 8000d18:	d902      	bls.n	8000d20 <NVIC_EncodePriority+0x30>
 8000d1a:	69fb      	ldr	r3, [r7, #28]
 8000d1c:	3b03      	subs	r3, #3
 8000d1e:	e000      	b.n	8000d22 <NVIC_EncodePriority+0x32>
 8000d20:	2300      	movs	r3, #0
 8000d22:	617b      	str	r3, [r7, #20]

  return (
           ((PreemptPriority & (uint32_t)((1UL << (PreemptPriorityBits)) - 1UL)) << SubPriorityBits) |
 8000d24:	f04f 32ff 	mov.w	r2, #4294967295
 8000d28:	69bb      	ldr	r3, [r7, #24]
 8000d2a:	fa02 f303 	lsl.w	r3, r2, r3
 8000d2e:	43da      	mvns	r2, r3
 8000d30:	68bb      	ldr	r3, [r7, #8]
 8000d32:	401a      	ands	r2, r3
 8000d34:	697b      	ldr	r3, [r7, #20]
 8000d36:	409a      	lsls	r2, r3
           ((SubPriority     & (uint32_t)((1UL << (SubPriorityBits    )) - 1UL)))
 8000d38:	f04f 31ff 	mov.w	r1, #4294967295
 8000d3c:	697b      	ldr	r3, [r7, #20]
 8000d3e:	fa01 f303 	lsl.w	r3, r1, r3
 8000d42:	43d9      	mvns	r1, r3
 8000d44:	687b      	ldr	r3, [r7, #4]
 8000d46:	400b      	ands	r3, r1
           ((PreemptPriority & (uint32_t)((1UL << (PreemptPriorityBits)) - 1UL)) << SubPriorityBits) |
 8000d48:	4313      	orrs	r3, r2
         );
}
 8000d4a:	4618      	mov	r0, r3
 8000d4c:	3724      	adds	r7, #36	; 0x24
 8000d4e:	46bd      	mov	sp, r7
 8000d50:	f85d 7b04 	ldr.w	r7, [sp], #4
 8000d54:	4770      	bx	lr
	...

08000d58 <SysTick_Config>:
  \note    When the variable <b>__Vendor_SysTickConfig</b> is set to 1, then the
           function <b>SysTick_Config</b> is not included. In this case, the file <b><i>device</i>.h</b>
           must contain a vendor-specific implementation of this function.
 */
__STATIC_INLINE uint32_t SysTick_Config(uint32_t ticks)
{
 8000d58:	b580      	push	{r7, lr}
 8000d5a:	b082      	sub	sp, #8
 8000d5c:	af00      	add	r7, sp, #0
 8000d5e:	6078      	str	r0, [r7, #4]
  if ((ticks - 1UL) > SysTick_LOAD_RELOAD_Msk)
 8000d60:	687b      	ldr	r3, [r7, #4]
 8000d62:	3b01      	subs	r3, #1
 8000d64:	f1b3 7f80 	cmp.w	r3, #16777216	; 0x1000000
 8000d68:	d301      	bcc.n	8000d6e <SysTick_Config+0x16>
  {
    return (1UL);                                                   /* Reload value impossible */
 8000d6a:	2301      	movs	r3, #1
 8000d6c:	e00f      	b.n	8000d8e <SysTick_Config+0x36>
  }

  SysTick->LOAD  = (uint32_t)(ticks - 1UL);                         /* set reload register */
 8000d6e:	4a0a      	ldr	r2, [pc, #40]	; (8000d98 <SysTick_Config+0x40>)
 8000d70:	687b      	ldr	r3, [r7, #4]
 8000d72:	3b01      	subs	r3, #1
 8000d74:	6053      	str	r3, [r2, #4]
  NVIC_SetPriority (SysTick_IRQn, (1UL << __NVIC_PRIO_BITS) - 1UL); /* set Priority for Systick Interrupt */
 8000d76:	210f      	movs	r1, #15
 8000d78:	f04f 30ff 	mov.w	r0, #4294967295
 8000d7c:	f7ff ff8e 	bl	8000c9c <__NVIC_SetPriority>
  SysTick->VAL   = 0UL;                                             /* Load the SysTick Counter Value */
 8000d80:	4b05      	ldr	r3, [pc, #20]	; (8000d98 <SysTick_Config+0x40>)
 8000d82:	2200      	movs	r2, #0
 8000d84:	609a      	str	r2, [r3, #8]
  SysTick->CTRL  = SysTick_CTRL_CLKSOURCE_Msk |
 8000d86:	4b04      	ldr	r3, [pc, #16]	; (8000d98 <SysTick_Config+0x40>)
 8000d88:	2207      	movs	r2, #7
 8000d8a:	601a      	str	r2, [r3, #0]
                   SysTick_CTRL_TICKINT_Msk   |
                   SysTick_CTRL_ENABLE_Msk;                         /* Enable SysTick IRQ and SysTick Timer */
  return (0UL);                                                     /* Function successful */
 8000d8c:	2300      	movs	r3, #0
}
 8000d8e:	4618      	mov	r0, r3
 8000d90:	3708      	adds	r7, #8
 8000d92:	46bd      	mov	sp, r7
 8000d94:	bd80      	pop	{r7, pc}
 8000d96:	bf00      	nop
 8000d98:	e000e010 	.word	0xe000e010

08000d9c <HAL_NVIC_SetPriorityGrouping>:
  * @note   When the NVIC_PriorityGroup_0 is selected, IRQ preemption is no more possible. 
  *         The pending IRQ priority will be managed only by the subpriority. 
  * @retval None
  */
void HAL_NVIC_SetPriorityGrouping(uint32_t PriorityGroup)
{
 8000d9c:	b580      	push	{r7, lr}
 8000d9e:	b082      	sub	sp, #8
 8000da0:	af00      	add	r7, sp, #0
 8000da2:	6078      	str	r0, [r7, #4]
  /* Check the parameters */
  assert_param(IS_NVIC_PRIORITY_GROUP(PriorityGroup));
  
  /* Set the PRIGROUP[10:8] bits according to the PriorityGroup parameter value */
  NVIC_SetPriorityGrouping(PriorityGroup);
 8000da4:	6878      	ldr	r0, [r7, #4]
 8000da6:	f7ff ff47 	bl	8000c38 <__NVIC_SetPriorityGrouping>
}
 8000daa:	bf00      	nop
 8000dac:	3708      	adds	r7, #8
 8000dae:	46bd      	mov	sp, r7
 8000db0:	bd80      	pop	{r7, pc}

08000db2 <HAL_NVIC_SetPriority>:
  *         This parameter can be a value between 0 and 15
  *         A lower priority value indicates a higher priority.          
  * @retval None
  */
void HAL_NVIC_SetPriority(IRQn_Type IRQn, uint32_t PreemptPriority, uint32_t SubPriority)
{ 
 8000db2:	b580      	push	{r7, lr}
 8000db4:	b086      	sub	sp, #24
 8000db6:	af00      	add	r7, sp, #0
 8000db8:	4603      	mov	r3, r0
 8000dba:	60b9      	str	r1, [r7, #8]
 8000dbc:	607a      	str	r2, [r7, #4]
 8000dbe:	73fb      	strb	r3, [r7, #15]
  uint32_t prioritygroup = 0x00U;
 8000dc0:	2300      	movs	r3, #0
 8000dc2:	617b      	str	r3, [r7, #20]
  
  /* Check the parameters */
  assert_param(IS_NVIC_SUB_PRIORITY(SubPriority));
  assert_param(IS_NVIC_PREEMPTION_PRIORITY(PreemptPriority));
  
  prioritygroup = NVIC_GetPriorityGrouping();
 8000dc4:	f7ff ff5c 	bl	8000c80 <__NVIC_GetPriorityGrouping>
 8000dc8:	6178      	str	r0, [r7, #20]
  
  NVIC_SetPriority(IRQn, NVIC_EncodePriority(prioritygroup, PreemptPriority, SubPriority));
 8000dca:	687a      	ldr	r2, [r7, #4]
 8000dcc:	68b9      	ldr	r1, [r7, #8]
 8000dce:	6978      	ldr	r0, [r7, #20]
 8000dd0:	f7ff ff8e 	bl	8000cf0 <NVIC_EncodePriority>
 8000dd4:	4602      	mov	r2, r0
 8000dd6:	f997 300f 	ldrsb.w	r3, [r7, #15]
 8000dda:	4611      	mov	r1, r2
 8000ddc:	4618      	mov	r0, r3
 8000dde:	f7ff ff5d 	bl	8000c9c <__NVIC_SetPriority>
}
 8000de2:	bf00      	nop
 8000de4:	3718      	adds	r7, #24
 8000de6:	46bd      	mov	sp, r7
 8000de8:	bd80      	pop	{r7, pc}

08000dea <HAL_SYSTICK_Config>:
  * @param  TicksNumb Specifies the ticks Number of ticks between two interrupts.
  * @retval status:  - 0  Function succeeded.
  *                  - 1  Function failed.
  */
uint32_t HAL_SYSTICK_Config(uint32_t TicksNumb)
{
 8000dea:	b580      	push	{r7, lr}
 8000dec:	b082      	sub	sp, #8
 8000dee:	af00      	add	r7, sp, #0
 8000df0:	6078      	str	r0, [r7, #4]
   return SysTick_Config(TicksNumb);
 8000df2:	6878      	ldr	r0, [r7, #4]
 8000df4:	f7ff ffb0 	bl	8000d58 <SysTick_Config>
 8000df8:	4603      	mov	r3, r0
}
 8000dfa:	4618      	mov	r0, r3
 8000dfc:	3708      	adds	r7, #8
 8000dfe:	46bd      	mov	sp, r7
 8000e00:	bd80      	pop	{r7, pc}
	...

08000e04 <HAL_GPIO_Init>:
  * @param  GPIO_Init pointer to a GPIO_InitTypeDef structure that contains
  *         the configuration information for the specified GPIO peripheral.
  * @retval None
  */
void HAL_GPIO_Init(GPIO_TypeDef  *GPIOx, GPIO_InitTypeDef *GPIO_Init)
{
 8000e04:	b480      	push	{r7}
 8000e06:	b089      	sub	sp, #36	; 0x24
 8000e08:	af00      	add	r7, sp, #0
 8000e0a:	6078      	str	r0, [r7, #4]
 8000e0c:	6039      	str	r1, [r7, #0]
  uint32_t position;
  uint32_t ioposition = 0x00U;
 8000e0e:	2300      	movs	r3, #0
 8000e10:	617b      	str	r3, [r7, #20]
  uint32_t iocurrent = 0x00U;
 8000e12:	2300      	movs	r3, #0
 8000e14:	613b      	str	r3, [r7, #16]
  uint32_t temp = 0x00U;
 8000e16:	2300      	movs	r3, #0
 8000e18:	61bb      	str	r3, [r7, #24]
  assert_param(IS_GPIO_ALL_INSTANCE(GPIOx));
  assert_param(IS_GPIO_PIN(GPIO_Init->Pin));
  assert_param(IS_GPIO_MODE(GPIO_Init->Mode));

  /* Configure the port pins */
  for(position = 0U; position < GPIO_NUMBER; position++)
 8000e1a:	2300      	movs	r3, #0
 8000e1c:	61fb      	str	r3, [r7, #28]
 8000e1e:	e177      	b.n	8001110 <HAL_GPIO_Init+0x30c>
  {
    /* Get the IO position */
    ioposition = 0x01U << position;
 8000e20:	2201      	movs	r2, #1
 8000e22:	69fb      	ldr	r3, [r7, #28]
 8000e24:	fa02 f303 	lsl.w	r3, r2, r3
 8000e28:	617b      	str	r3, [r7, #20]
    /* Get the current IO position */
    iocurrent = (uint32_t)(GPIO_Init->Pin) & ioposition;
 8000e2a:	683b      	ldr	r3, [r7, #0]
 8000e2c:	681b      	ldr	r3, [r3, #0]
 8000e2e:	697a      	ldr	r2, [r7, #20]
 8000e30:	4013      	ands	r3, r2
 8000e32:	613b      	str	r3, [r7, #16]

    if(iocurrent == ioposition)
 8000e34:	693a      	ldr	r2, [r7, #16]
 8000e36:	697b      	ldr	r3, [r7, #20]
 8000e38:	429a      	cmp	r2, r3
 8000e3a:	f040 8166 	bne.w	800110a <HAL_GPIO_Init+0x306>
    {
      /*--------------------- GPIO Mode Configuration ------------------------*/
      /* In case of Output or Alternate function mode selection */
      if(((GPIO_Init->Mode & GPIO_MODE) == MODE_OUTPUT) || \
 8000e3e:	683b      	ldr	r3, [r7, #0]
 8000e40:	685b      	ldr	r3, [r3, #4]
 8000e42:	f003 0303 	and.w	r3, r3, #3
 8000e46:	2b01      	cmp	r3, #1
 8000e48:	d005      	beq.n	8000e56 <HAL_GPIO_Init+0x52>
          (GPIO_Init->Mode & GPIO_MODE) == MODE_AF)
 8000e4a:	683b      	ldr	r3, [r7, #0]
 8000e4c:	685b      	ldr	r3, [r3, #4]
 8000e4e:	f003 0303 	and.w	r3, r3, #3
      if(((GPIO_Init->Mode & GPIO_MODE) == MODE_OUTPUT) || \
 8000e52:	2b02      	cmp	r3, #2
 8000e54:	d130      	bne.n	8000eb8 <HAL_GPIO_Init+0xb4>
      {
        /* Check the Speed parameter */
        assert_param(IS_GPIO_SPEED(GPIO_Init->Speed));
        /* Configure the IO Speed */
        temp = GPIOx->OSPEEDR; 
 8000e56:	687b      	ldr	r3, [r7, #4]
 8000e58:	689b      	ldr	r3, [r3, #8]
 8000e5a:	61bb      	str	r3, [r7, #24]
        temp &= ~(GPIO_OSPEEDER_OSPEEDR0 << (position * 2U));
 8000e5c:	69fb      	ldr	r3, [r7, #28]
 8000e5e:	005b      	lsls	r3, r3, #1
 8000e60:	2203      	movs	r2, #3
 8000e62:	fa02 f303 	lsl.w	r3, r2, r3
 8000e66:	43db      	mvns	r3, r3
 8000e68:	69ba      	ldr	r2, [r7, #24]
 8000e6a:	4013      	ands	r3, r2
 8000e6c:	61bb      	str	r3, [r7, #24]
        temp |= (GPIO_Init->Speed << (position * 2U));
 8000e6e:	683b      	ldr	r3, [r7, #0]
 8000e70:	68da      	ldr	r2, [r3, #12]
 8000e72:	69fb      	ldr	r3, [r7, #28]
 8000e74:	005b      	lsls	r3, r3, #1
 8000e76:	fa02 f303 	lsl.w	r3, r2, r3
 8000e7a:	69ba      	ldr	r2, [r7, #24]
 8000e7c:	4313      	orrs	r3, r2
 8000e7e:	61bb      	str	r3, [r7, #24]
        GPIOx->OSPEEDR = temp;
 8000e80:	687b      	ldr	r3, [r7, #4]
 8000e82:	69ba      	ldr	r2, [r7, #24]
 8000e84:	609a      	str	r2, [r3, #8]

        /* Configure the IO Output Type */
        temp = GPIOx->OTYPER;
 8000e86:	687b      	ldr	r3, [r7, #4]
 8000e88:	685b      	ldr	r3, [r3, #4]
 8000e8a:	61bb      	str	r3, [r7, #24]
        temp &= ~(GPIO_OTYPER_OT_0 << position) ;
 8000e8c:	2201      	movs	r2, #1
 8000e8e:	69fb      	ldr	r3, [r7, #28]
 8000e90:	fa02 f303 	lsl.w	r3, r2, r3
 8000e94:	43db      	mvns	r3, r3
 8000e96:	69ba      	ldr	r2, [r7, #24]
 8000e98:	4013      	ands	r3, r2
 8000e9a:	61bb      	str	r3, [r7, #24]
        temp |= (((GPIO_Init->Mode & OUTPUT_TYPE) >> OUTPUT_TYPE_Pos) << position);
 8000e9c:	683b      	ldr	r3, [r7, #0]
 8000e9e:	685b      	ldr	r3, [r3, #4]
 8000ea0:	091b      	lsrs	r3, r3, #4
 8000ea2:	f003 0201 	and.w	r2, r3, #1
 8000ea6:	69fb      	ldr	r3, [r7, #28]
 8000ea8:	fa02 f303 	lsl.w	r3, r2, r3
 8000eac:	69ba      	ldr	r2, [r7, #24]
 8000eae:	4313      	orrs	r3, r2
 8000eb0:	61bb      	str	r3, [r7, #24]
        GPIOx->OTYPER = temp;
 8000eb2:	687b      	ldr	r3, [r7, #4]
 8000eb4:	69ba      	ldr	r2, [r7, #24]
 8000eb6:	605a      	str	r2, [r3, #4]
       }

      if((GPIO_Init->Mode & GPIO_MODE) != MODE_ANALOG)
 8000eb8:	683b      	ldr	r3, [r7, #0]
 8000eba:	685b      	ldr	r3, [r3, #4]
 8000ebc:	f003 0303 	and.w	r3, r3, #3
 8000ec0:	2b03      	cmp	r3, #3
 8000ec2:	d017      	beq.n	8000ef4 <HAL_GPIO_Init+0xf0>
      {
        /* Check the parameters */
        assert_param(IS_GPIO_PULL(GPIO_Init->Pull));
        
        /* Activate the Pull-up or Pull down resistor for the current IO */
        temp = GPIOx->PUPDR;
 8000ec4:	687b      	ldr	r3, [r7, #4]
 8000ec6:	68db      	ldr	r3, [r3, #12]
 8000ec8:	61bb      	str	r3, [r7, #24]
        temp &= ~(GPIO_PUPDR_PUPDR0 << (position * 2U));
 8000eca:	69fb      	ldr	r3, [r7, #28]
 8000ecc:	005b      	lsls	r3, r3, #1
 8000ece:	2203      	movs	r2, #3
 8000ed0:	fa02 f303 	lsl.w	r3, r2, r3
 8000ed4:	43db      	mvns	r3, r3
 8000ed6:	69ba      	ldr	r2, [r7, #24]
 8000ed8:	4013      	ands	r3, r2
 8000eda:	61bb      	str	r3, [r7, #24]
        temp |= ((GPIO_Init->Pull) << (position * 2U));
 8000edc:	683b      	ldr	r3, [r7, #0]
 8000ede:	689a      	ldr	r2, [r3, #8]
 8000ee0:	69fb      	ldr	r3, [r7, #28]
 8000ee2:	005b      	lsls	r3, r3, #1
 8000ee4:	fa02 f303 	lsl.w	r3, r2, r3
 8000ee8:	69ba      	ldr	r2, [r7, #24]
 8000eea:	4313      	orrs	r3, r2
 8000eec:	61bb      	str	r3, [r7, #24]
        GPIOx->PUPDR = temp;
 8000eee:	687b      	ldr	r3, [r7, #4]
 8000ef0:	69ba      	ldr	r2, [r7, #24]
 8000ef2:	60da      	str	r2, [r3, #12]
      }

      /* In case of Alternate function mode selection */
      if((GPIO_Init->Mode & GPIO_MODE) == MODE_AF)
 8000ef4:	683b      	ldr	r3, [r7, #0]
 8000ef6:	685b      	ldr	r3, [r3, #4]
 8000ef8:	f003 0303 	and.w	r3, r3, #3
 8000efc:	2b02      	cmp	r3, #2
 8000efe:	d123      	bne.n	8000f48 <HAL_GPIO_Init+0x144>
      {
        /* Check the Alternate function parameter */
        assert_param(IS_GPIO_AF(GPIO_Init->Alternate));
        /* Configure Alternate function mapped with the current IO */
        temp = GPIOx->AFR[position >> 3U];
 8000f00:	69fb      	ldr	r3, [r7, #28]
 8000f02:	08da      	lsrs	r2, r3, #3
 8000f04:	687b      	ldr	r3, [r7, #4]
 8000f06:	3208      	adds	r2, #8
 8000f08:	f853 3022 	ldr.w	r3, [r3, r2, lsl #2]
 8000f0c:	61bb      	str	r3, [r7, #24]
        temp &= ~(0xFU << ((uint32_t)(position & 0x07U) * 4U)) ;
 8000f0e:	69fb      	ldr	r3, [r7, #28]
 8000f10:	f003 0307 	and.w	r3, r3, #7
 8000f14:	009b      	lsls	r3, r3, #2
 8000f16:	220f      	movs	r2, #15
 8000f18:	fa02 f303 	lsl.w	r3, r2, r3
 8000f1c:	43db      	mvns	r3, r3
 8000f1e:	69ba      	ldr	r2, [r7, #24]
 8000f20:	4013      	ands	r3, r2
 8000f22:	61bb      	str	r3, [r7, #24]
        temp |= ((uint32_t)(GPIO_Init->Alternate) << (((uint32_t)position & 0x07U) * 4U));
 8000f24:	683b      	ldr	r3, [r7, #0]
 8000f26:	691a      	ldr	r2, [r3, #16]
 8000f28:	69fb      	ldr	r3, [r7, #28]
 8000f2a:	f003 0307 	and.w	r3, r3, #7
 8000f2e:	009b      	lsls	r3, r3, #2
 8000f30:	fa02 f303 	lsl.w	r3, r2, r3
 8000f34:	69ba      	ldr	r2, [r7, #24]
 8000f36:	4313      	orrs	r3, r2
 8000f38:	61bb      	str	r3, [r7, #24]
        GPIOx->AFR[position >> 3U] = temp;
 8000f3a:	69fb      	ldr	r3, [r7, #28]
 8000f3c:	08da      	lsrs	r2, r3, #3
 8000f3e:	687b      	ldr	r3, [r7, #4]
 8000f40:	3208      	adds	r2, #8
 8000f42:	69b9      	ldr	r1, [r7, #24]
 8000f44:	f843 1022 	str.w	r1, [r3, r2, lsl #2]
      }

      /* Configure IO Direction mode (Input, Output, Alternate or Analog) */
      temp = GPIOx->MODER;
 8000f48:	687b      	ldr	r3, [r7, #4]
 8000f4a:	681b      	ldr	r3, [r3, #0]
 8000f4c:	61bb      	str	r3, [r7, #24]
      temp &= ~(GPIO_MODER_MODER0 << (position * 2U));
 8000f4e:	69fb      	ldr	r3, [r7, #28]
 8000f50:	005b      	lsls	r3, r3, #1
 8000f52:	2203      	movs	r2, #3
 8000f54:	fa02 f303 	lsl.w	r3, r2, r3
 8000f58:	43db      	mvns	r3, r3
 8000f5a:	69ba      	ldr	r2, [r7, #24]
 8000f5c:	4013      	ands	r3, r2
 8000f5e:	61bb      	str	r3, [r7, #24]
      temp |= ((GPIO_Init->Mode & GPIO_MODE) << (position * 2U));
 8000f60:	683b      	ldr	r3, [r7, #0]
 8000f62:	685b      	ldr	r3, [r3, #4]
 8000f64:	f003 0203 	and.w	r2, r3, #3
 8000f68:	69fb      	ldr	r3, [r7, #28]
 8000f6a:	005b      	lsls	r3, r3, #1
 8000f6c:	fa02 f303 	lsl.w	r3, r2, r3
 8000f70:	69ba      	ldr	r2, [r7, #24]
 8000f72:	4313      	orrs	r3, r2
 8000f74:	61bb      	str	r3, [r7, #24]
      GPIOx->MODER = temp;
 8000f76:	687b      	ldr	r3, [r7, #4]
 8000f78:	69ba      	ldr	r2, [r7, #24]
 8000f7a:	601a      	str	r2, [r3, #0]

      /*--------------------- EXTI Mode Configuration ------------------------*/
      /* Configure the External Interrupt or event for the current IO */
      if((GPIO_Init->Mode & EXTI_MODE) != 0x00U)
 8000f7c:	683b      	ldr	r3, [r7, #0]
 8000f7e:	685b      	ldr	r3, [r3, #4]
 8000f80:	f403 3340 	and.w	r3, r3, #196608	; 0x30000
 8000f84:	2b00      	cmp	r3, #0
 8000f86:	f000 80c0 	beq.w	800110a <HAL_GPIO_Init+0x306>
      {
        /* Enable SYSCFG Clock */
        __HAL_RCC_SYSCFG_CLK_ENABLE();
 8000f8a:	2300      	movs	r3, #0
 8000f8c:	60fb      	str	r3, [r7, #12]
 8000f8e:	4b66      	ldr	r3, [pc, #408]	; (8001128 <HAL_GPIO_Init+0x324>)
 8000f90:	6c5b      	ldr	r3, [r3, #68]	; 0x44
 8000f92:	4a65      	ldr	r2, [pc, #404]	; (8001128 <HAL_GPIO_Init+0x324>)
 8000f94:	f443 4380 	orr.w	r3, r3, #16384	; 0x4000
 8000f98:	6453      	str	r3, [r2, #68]	; 0x44
 8000f9a:	4b63      	ldr	r3, [pc, #396]	; (8001128 <HAL_GPIO_Init+0x324>)
 8000f9c:	6c5b      	ldr	r3, [r3, #68]	; 0x44
 8000f9e:	f403 4380 	and.w	r3, r3, #16384	; 0x4000
 8000fa2:	60fb      	str	r3, [r7, #12]
 8000fa4:	68fb      	ldr	r3, [r7, #12]

        temp = SYSCFG->EXTICR[position >> 2U];
 8000fa6:	4a61      	ldr	r2, [pc, #388]	; (800112c <HAL_GPIO_Init+0x328>)
 8000fa8:	69fb      	ldr	r3, [r7, #28]
 8000faa:	089b      	lsrs	r3, r3, #2
 8000fac:	3302      	adds	r3, #2
 8000fae:	f852 3023 	ldr.w	r3, [r2, r3, lsl #2]
 8000fb2:	61bb      	str	r3, [r7, #24]
        temp &= ~(0x0FU << (4U * (position & 0x03U)));
 8000fb4:	69fb      	ldr	r3, [r7, #28]
 8000fb6:	f003 0303 	and.w	r3, r3, #3
 8000fba:	009b      	lsls	r3, r3, #2
 8000fbc:	220f      	movs	r2, #15
 8000fbe:	fa02 f303 	lsl.w	r3, r2, r3
 8000fc2:	43db      	mvns	r3, r3
 8000fc4:	69ba      	ldr	r2, [r7, #24]
 8000fc6:	4013      	ands	r3, r2
 8000fc8:	61bb      	str	r3, [r7, #24]
        temp |= ((uint32_t)(GPIO_GET_INDEX(GPIOx)) << (4U * (position & 0x03U)));
 8000fca:	687b      	ldr	r3, [r7, #4]
 8000fcc:	4a58      	ldr	r2, [pc, #352]	; (8001130 <HAL_GPIO_Init+0x32c>)
 8000fce:	4293      	cmp	r3, r2
 8000fd0:	d037      	beq.n	8001042 <HAL_GPIO_Init+0x23e>
 8000fd2:	687b      	ldr	r3, [r7, #4]
 8000fd4:	4a57      	ldr	r2, [pc, #348]	; (8001134 <HAL_GPIO_Init+0x330>)
 8000fd6:	4293      	cmp	r3, r2
 8000fd8:	d031      	beq.n	800103e <HAL_GPIO_Init+0x23a>
 8000fda:	687b      	ldr	r3, [r7, #4]
 8000fdc:	4a56      	ldr	r2, [pc, #344]	; (8001138 <HAL_GPIO_Init+0x334>)
 8000fde:	4293      	cmp	r3, r2
 8000fe0:	d02b      	beq.n	800103a <HAL_GPIO_Init+0x236>
 8000fe2:	687b      	ldr	r3, [r7, #4]
 8000fe4:	4a55      	ldr	r2, [pc, #340]	; (800113c <HAL_GPIO_Init+0x338>)
 8000fe6:	4293      	cmp	r3, r2
 8000fe8:	d025      	beq.n	8001036 <HAL_GPIO_Init+0x232>
 8000fea:	687b      	ldr	r3, [r7, #4]
 8000fec:	4a54      	ldr	r2, [pc, #336]	; (8001140 <HAL_GPIO_Init+0x33c>)
 8000fee:	4293      	cmp	r3, r2
 8000ff0:	d01f      	beq.n	8001032 <HAL_GPIO_Init+0x22e>
 8000ff2:	687b      	ldr	r3, [r7, #4]
 8000ff4:	4a53      	ldr	r2, [pc, #332]	; (8001144 <HAL_GPIO_Init+0x340>)
 8000ff6:	4293      	cmp	r3, r2
 8000ff8:	d019      	beq.n	800102e <HAL_GPIO_Init+0x22a>
 8000ffa:	687b      	ldr	r3, [r7, #4]
 8000ffc:	4a52      	ldr	r2, [pc, #328]	; (8001148 <HAL_GPIO_Init+0x344>)
 8000ffe:	4293      	cmp	r3, r2
 8001000:	d013      	beq.n	800102a <HAL_GPIO_Init+0x226>
 8001002:	687b      	ldr	r3, [r7, #4]
 8001004:	4a51      	ldr	r2, [pc, #324]	; (800114c <HAL_GPIO_Init+0x348>)
 8001006:	4293      	cmp	r3, r2
 8001008:	d00d      	beq.n	8001026 <HAL_GPIO_Init+0x222>
 800100a:	687b      	ldr	r3, [r7, #4]
 800100c:	4a50      	ldr	r2, [pc, #320]	; (8001150 <HAL_GPIO_Init+0x34c>)
 800100e:	4293      	cmp	r3, r2
 8001010:	d007      	beq.n	8001022 <HAL_GPIO_Init+0x21e>
 8001012:	687b      	ldr	r3, [r7, #4]
 8001014:	4a4f      	ldr	r2, [pc, #316]	; (8001154 <HAL_GPIO_Init+0x350>)
 8001016:	4293      	cmp	r3, r2
 8001018:	d101      	bne.n	800101e <HAL_GPIO_Init+0x21a>
 800101a:	2309      	movs	r3, #9
 800101c:	e012      	b.n	8001044 <HAL_GPIO_Init+0x240>
 800101e:	230a      	movs	r3, #10
 8001020:	e010      	b.n	8001044 <HAL_GPIO_Init+0x240>
 8001022:	2308      	movs	r3, #8
 8001024:	e00e      	b.n	8001044 <HAL_GPIO_Init+0x240>
 8001026:	2307      	movs	r3, #7
 8001028:	e00c      	b.n	8001044 <HAL_GPIO_Init+0x240>
 800102a:	2306      	movs	r3, #6
 800102c:	e00a      	b.n	8001044 <HAL_GPIO_Init+0x240>
 800102e:	2305      	movs	r3, #5
 8001030:	e008      	b.n	8001044 <HAL_GPIO_Init+0x240>
 8001032:	2304      	movs	r3, #4
 8001034:	e006      	b.n	8001044 <HAL_GPIO_Init+0x240>
 8001036:	2303      	movs	r3, #3
 8001038:	e004      	b.n	8001044 <HAL_GPIO_Init+0x240>
 800103a:	2302      	movs	r3, #2
 800103c:	e002      	b.n	8001044 <HAL_GPIO_Init+0x240>
 800103e:	2301      	movs	r3, #1
 8001040:	e000      	b.n	8001044 <HAL_GPIO_Init+0x240>
 8001042:	2300      	movs	r3, #0
 8001044:	69fa      	ldr	r2, [r7, #28]
 8001046:	f002 0203 	and.w	r2, r2, #3
 800104a:	0092      	lsls	r2, r2, #2
 800104c:	4093      	lsls	r3, r2
 800104e:	69ba      	ldr	r2, [r7, #24]
 8001050:	4313      	orrs	r3, r2
 8001052:	61bb      	str	r3, [r7, #24]
        SYSCFG->EXTICR[position >> 2U] = temp;
 8001054:	4935      	ldr	r1, [pc, #212]	; (800112c <HAL_GPIO_Init+0x328>)
 8001056:	69fb      	ldr	r3, [r7, #28]
 8001058:	089b      	lsrs	r3, r3, #2
 800105a:	3302      	adds	r3, #2
 800105c:	69ba      	ldr	r2, [r7, #24]
 800105e:	f841 2023 	str.w	r2, [r1, r3, lsl #2]

        /* Clear Rising Falling edge configuration */
        temp = EXTI->RTSR;
 8001062:	4b3d      	ldr	r3, [pc, #244]	; (8001158 <HAL_GPIO_Init+0x354>)
 8001064:	689b      	ldr	r3, [r3, #8]
 8001066:	61bb      	str	r3, [r7, #24]
        temp &= ~((uint32_t)iocurrent);
 8001068:	693b      	ldr	r3, [r7, #16]
 800106a:	43db      	mvns	r3, r3
 800106c:	69ba      	ldr	r2, [r7, #24]
 800106e:	4013      	ands	r3, r2
 8001070:	61bb      	str	r3, [r7, #24]
        if((GPIO_Init->Mode & TRIGGER_RISING) != 0x00U)
 8001072:	683b      	ldr	r3, [r7, #0]
 8001074:	685b      	ldr	r3, [r3, #4]
 8001076:	f403 1380 	and.w	r3, r3, #1048576	; 0x100000
 800107a:	2b00      	cmp	r3, #0
 800107c:	d003      	beq.n	8001086 <HAL_GPIO_Init+0x282>
        {
          temp |= iocurrent;
 800107e:	69ba      	ldr	r2, [r7, #24]
 8001080:	693b      	ldr	r3, [r7, #16]
 8001082:	4313      	orrs	r3, r2
 8001084:	61bb      	str	r3, [r7, #24]
        }
        EXTI->RTSR = temp;
 8001086:	4a34      	ldr	r2, [pc, #208]	; (8001158 <HAL_GPIO_Init+0x354>)
 8001088:	69bb      	ldr	r3, [r7, #24]
 800108a:	6093      	str	r3, [r2, #8]

        temp = EXTI->FTSR;
 800108c:	4b32      	ldr	r3, [pc, #200]	; (8001158 <HAL_GPIO_Init+0x354>)
 800108e:	68db      	ldr	r3, [r3, #12]
 8001090:	61bb      	str	r3, [r7, #24]
        temp &= ~((uint32_t)iocurrent);
 8001092:	693b      	ldr	r3, [r7, #16]
 8001094:	43db      	mvns	r3, r3
 8001096:	69ba      	ldr	r2, [r7, #24]
 8001098:	4013      	ands	r3, r2
 800109a:	61bb      	str	r3, [r7, #24]
        if((GPIO_Init->Mode & TRIGGER_FALLING) != 0x00U)
 800109c:	683b      	ldr	r3, [r7, #0]
 800109e:	685b      	ldr	r3, [r3, #4]
 80010a0:	f403 1300 	and.w	r3, r3, #2097152	; 0x200000
 80010a4:	2b00      	cmp	r3, #0
 80010a6:	d003      	beq.n	80010b0 <HAL_GPIO_Init+0x2ac>
        {
          temp |= iocurrent;
 80010a8:	69ba      	ldr	r2, [r7, #24]
 80010aa:	693b      	ldr	r3, [r7, #16]
 80010ac:	4313      	orrs	r3, r2
 80010ae:	61bb      	str	r3, [r7, #24]
        }
        EXTI->FTSR = temp;
 80010b0:	4a29      	ldr	r2, [pc, #164]	; (8001158 <HAL_GPIO_Init+0x354>)
 80010b2:	69bb      	ldr	r3, [r7, #24]
 80010b4:	60d3      	str	r3, [r2, #12]

        temp = EXTI->EMR;
 80010b6:	4b28      	ldr	r3, [pc, #160]	; (8001158 <HAL_GPIO_Init+0x354>)
 80010b8:	685b      	ldr	r3, [r3, #4]
 80010ba:	61bb      	str	r3, [r7, #24]
        temp &= ~((uint32_t)iocurrent);
 80010bc:	693b      	ldr	r3, [r7, #16]
 80010be:	43db      	mvns	r3, r3
 80010c0:	69ba      	ldr	r2, [r7, #24]
 80010c2:	4013      	ands	r3, r2
 80010c4:	61bb      	str	r3, [r7, #24]
        if((GPIO_Init->Mode & EXTI_EVT) != 0x00U)
 80010c6:	683b      	ldr	r3, [r7, #0]
 80010c8:	685b      	ldr	r3, [r3, #4]
 80010ca:	f403 3300 	and.w	r3, r3, #131072	; 0x20000
 80010ce:	2b00      	cmp	r3, #0
 80010d0:	d003      	beq.n	80010da <HAL_GPIO_Init+0x2d6>
        {
          temp |= iocurrent;
 80010d2:	69ba      	ldr	r2, [r7, #24]
 80010d4:	693b      	ldr	r3, [r7, #16]
 80010d6:	4313      	orrs	r3, r2
 80010d8:	61bb      	str	r3, [r7, #24]
        }
        EXTI->EMR = temp;
 80010da:	4a1f      	ldr	r2, [pc, #124]	; (8001158 <HAL_GPIO_Init+0x354>)
 80010dc:	69bb      	ldr	r3, [r7, #24]
 80010de:	6053      	str	r3, [r2, #4]

        /* Clear EXTI line configuration */
        temp = EXTI->IMR;
 80010e0:	4b1d      	ldr	r3, [pc, #116]	; (8001158 <HAL_GPIO_Init+0x354>)
 80010e2:	681b      	ldr	r3, [r3, #0]
 80010e4:	61bb      	str	r3, [r7, #24]
        temp &= ~((uint32_t)iocurrent);
 80010e6:	693b      	ldr	r3, [r7, #16]
 80010e8:	43db      	mvns	r3, r3
 80010ea:	69ba      	ldr	r2, [r7, #24]
 80010ec:	4013      	ands	r3, r2
 80010ee:	61bb      	str	r3, [r7, #24]
        if((GPIO_Init->Mode & EXTI_IT) != 0x00U)
 80010f0:	683b      	ldr	r3, [r7, #0]
 80010f2:	685b      	ldr	r3, [r3, #4]
 80010f4:	f403 3380 	and.w	r3, r3, #65536	; 0x10000
 80010f8:	2b00      	cmp	r3, #0
 80010fa:	d003      	beq.n	8001104 <HAL_GPIO_Init+0x300>
        {
          temp |= iocurrent;
 80010fc:	69ba      	ldr	r2, [r7, #24]
 80010fe:	693b      	ldr	r3, [r7, #16]
 8001100:	4313      	orrs	r3, r2
 8001102:	61bb      	str	r3, [r7, #24]
        }
        EXTI->IMR = temp;
 8001104:	4a14      	ldr	r2, [pc, #80]	; (8001158 <HAL_GPIO_Init+0x354>)
 8001106:	69bb      	ldr	r3, [r7, #24]
 8001108:	6013      	str	r3, [r2, #0]
  for(position = 0U; position < GPIO_NUMBER; position++)
 800110a:	69fb      	ldr	r3, [r7, #28]
 800110c:	3301      	adds	r3, #1
 800110e:	61fb      	str	r3, [r7, #28]
 8001110:	69fb      	ldr	r3, [r7, #28]
 8001112:	2b0f      	cmp	r3, #15
 8001114:	f67f ae84 	bls.w	8000e20 <HAL_GPIO_Init+0x1c>
      }
    }
  }
}
 8001118:	bf00      	nop
 800111a:	bf00      	nop
 800111c:	3724      	adds	r7, #36	; 0x24
 800111e:	46bd      	mov	sp, r7
 8001120:	f85d 7b04 	ldr.w	r7, [sp], #4
 8001124:	4770      	bx	lr
 8001126:	bf00      	nop
 8001128:	40023800 	.word	0x40023800
 800112c:	40013800 	.word	0x40013800
 8001130:	40020000 	.word	0x40020000
 8001134:	40020400 	.word	0x40020400
 8001138:	40020800 	.word	0x40020800
 800113c:	40020c00 	.word	0x40020c00
 8001140:	40021000 	.word	0x40021000
 8001144:	40021400 	.word	0x40021400
 8001148:	40021800 	.word	0x40021800
 800114c:	40021c00 	.word	0x40021c00
 8001150:	40022000 	.word	0x40022000
 8001154:	40022400 	.word	0x40022400
 8001158:	40013c00 	.word	0x40013c00

0800115c <HAL_GPIO_ReadPin>:
  * @param  GPIO_Pin specifies the port bit to read.
  *         This parameter can be GPIO_PIN_x where x can be (0..15).
  * @retval The input port pin value.
  */
GPIO_PinState HAL_GPIO_ReadPin(GPIO_TypeDef* GPIOx, uint16_t GPIO_Pin)
{
 800115c:	b480      	push	{r7}
 800115e:	b085      	sub	sp, #20
 8001160:	af00      	add	r7, sp, #0
 8001162:	6078      	str	r0, [r7, #4]
 8001164:	460b      	mov	r3, r1
 8001166:	807b      	strh	r3, [r7, #2]
  GPIO_PinState bitstatus;

  /* Check the parameters */
  assert_param(IS_GPIO_PIN(GPIO_Pin));

  if((GPIOx->IDR & GPIO_Pin) != (uint32_t)GPIO_PIN_RESET)
 8001168:	687b      	ldr	r3, [r7, #4]
 800116a:	691a      	ldr	r2, [r3, #16]
 800116c:	887b      	ldrh	r3, [r7, #2]
 800116e:	4013      	ands	r3, r2
 8001170:	2b00      	cmp	r3, #0
 8001172:	d002      	beq.n	800117a <HAL_GPIO_ReadPin+0x1e>
  {
    bitstatus = GPIO_PIN_SET;
 8001174:	2301      	movs	r3, #1
 8001176:	73fb      	strb	r3, [r7, #15]
 8001178:	e001      	b.n	800117e <HAL_GPIO_ReadPin+0x22>
  }
  else
  {
    bitstatus = GPIO_PIN_RESET;
 800117a:	2300      	movs	r3, #0
 800117c:	73fb      	strb	r3, [r7, #15]
  }
  return bitstatus;
 800117e:	7bfb      	ldrb	r3, [r7, #15]
}
 8001180:	4618      	mov	r0, r3
 8001182:	3714      	adds	r7, #20
 8001184:	46bd      	mov	sp, r7
 8001186:	f85d 7b04 	ldr.w	r7, [sp], #4
 800118a:	4770      	bx	lr

0800118c <HAL_GPIO_WritePin>:
  *            @arg GPIO_PIN_RESET: to clear the port pin
  *            @arg GPIO_PIN_SET: to set the port pin
  * @retval None
  */
void HAL_GPIO_WritePin(GPIO_TypeDef* GPIOx, uint16_t GPIO_Pin, GPIO_PinState PinState)
{
 800118c:	b480      	push	{r7}
 800118e:	b083      	sub	sp, #12
 8001190:	af00      	add	r7, sp, #0
 8001192:	6078      	str	r0, [r7, #4]
 8001194:	460b      	mov	r3, r1
 8001196:	807b      	strh	r3, [r7, #2]
 8001198:	4613      	mov	r3, r2
 800119a:	707b      	strb	r3, [r7, #1]
  /* Check the parameters */
  assert_param(IS_GPIO_PIN(GPIO_Pin));
  assert_param(IS_GPIO_PIN_ACTION(PinState));

  if(PinState != GPIO_PIN_RESET)
 800119c:	787b      	ldrb	r3, [r7, #1]
 800119e:	2b00      	cmp	r3, #0
 80011a0:	d003      	beq.n	80011aa <HAL_GPIO_WritePin+0x1e>
  {
    GPIOx->BSRR = GPIO_Pin;
 80011a2:	887a      	ldrh	r2, [r7, #2]
 80011a4:	687b      	ldr	r3, [r7, #4]
 80011a6:	619a      	str	r2, [r3, #24]
  }
  else
  {
    GPIOx->BSRR = (uint32_t)GPIO_Pin << 16U;
  }
}
 80011a8:	e003      	b.n	80011b2 <HAL_GPIO_WritePin+0x26>
    GPIOx->BSRR = (uint32_t)GPIO_Pin << 16U;
 80011aa:	887b      	ldrh	r3, [r7, #2]
 80011ac:	041a      	lsls	r2, r3, #16
 80011ae:	687b      	ldr	r3, [r7, #4]
 80011b0:	619a      	str	r2, [r3, #24]
}
 80011b2:	bf00      	nop
 80011b4:	370c      	adds	r7, #12
 80011b6:	46bd      	mov	sp, r7
 80011b8:	f85d 7b04 	ldr.w	r7, [sp], #4
 80011bc:	4770      	bx	lr
	...

080011c0 <HAL_RCC_OscConfig>:
  *         supported by this API. User should request a transition to HSE Off
  *         first and then HSE On or HSE Bypass.
  * @retval HAL status
  */
__weak HAL_StatusTypeDef HAL_RCC_OscConfig(RCC_OscInitTypeDef  *RCC_OscInitStruct)
{
 80011c0:	b580      	push	{r7, lr}
 80011c2:	b086      	sub	sp, #24
 80011c4:	af00      	add	r7, sp, #0
 80011c6:	6078      	str	r0, [r7, #4]
  uint32_t tickstart, pll_config;

  /* Check Null pointer */
  if(RCC_OscInitStruct == NULL)
 80011c8:	687b      	ldr	r3, [r7, #4]
 80011ca:	2b00      	cmp	r3, #0
 80011cc:	d101      	bne.n	80011d2 <HAL_RCC_OscConfig+0x12>
  {
    return HAL_ERROR;
 80011ce:	2301      	movs	r3, #1
 80011d0:	e267      	b.n	80016a2 <HAL_RCC_OscConfig+0x4e2>
  }

  /* Check the parameters */
  assert_param(IS_RCC_OSCILLATORTYPE(RCC_OscInitStruct->OscillatorType));
  /*------------------------------- HSE Configuration ------------------------*/
  if(((RCC_OscInitStruct->OscillatorType) & RCC_OSCILLATORTYPE_HSE) == RCC_OSCILLATORTYPE_HSE)
 80011d2:	687b      	ldr	r3, [r7, #4]
 80011d4:	681b      	ldr	r3, [r3, #0]
 80011d6:	f003 0301 	and.w	r3, r3, #1
 80011da:	2b00      	cmp	r3, #0
 80011dc:	d075      	beq.n	80012ca <HAL_RCC_OscConfig+0x10a>
  {
    /* Check the parameters */
    assert_param(IS_RCC_HSE(RCC_OscInitStruct->HSEState));
    /* When the HSE is used as system clock or clock source for PLL in these cases HSE will not disabled */
    if((__HAL_RCC_GET_SYSCLK_SOURCE() == RCC_CFGR_SWS_HSE) ||\
 80011de:	4b88      	ldr	r3, [pc, #544]	; (8001400 <HAL_RCC_OscConfig+0x240>)
 80011e0:	689b      	ldr	r3, [r3, #8]
 80011e2:	f003 030c 	and.w	r3, r3, #12
 80011e6:	2b04      	cmp	r3, #4
 80011e8:	d00c      	beq.n	8001204 <HAL_RCC_OscConfig+0x44>
      ((__HAL_RCC_GET_SYSCLK_SOURCE() == RCC_CFGR_SWS_PLL) && ((RCC->PLLCFGR & RCC_PLLCFGR_PLLSRC) == RCC_PLLCFGR_PLLSRC_HSE)))
 80011ea:	4b85      	ldr	r3, [pc, #532]	; (8001400 <HAL_RCC_OscConfig+0x240>)
 80011ec:	689b      	ldr	r3, [r3, #8]
 80011ee:	f003 030c 	and.w	r3, r3, #12
    if((__HAL_RCC_GET_SYSCLK_SOURCE() == RCC_CFGR_SWS_HSE) ||\
 80011f2:	2b08      	cmp	r3, #8
 80011f4:	d112      	bne.n	800121c <HAL_RCC_OscConfig+0x5c>
      ((__HAL_RCC_GET_SYSCLK_SOURCE() == RCC_CFGR_SWS_PLL) && ((RCC->PLLCFGR & RCC_PLLCFGR_PLLSRC) == RCC_PLLCFGR_PLLSRC_HSE)))
 80011f6:	4b82      	ldr	r3, [pc, #520]	; (8001400 <HAL_RCC_OscConfig+0x240>)
 80011f8:	685b      	ldr	r3, [r3, #4]
 80011fa:	f403 0380 	and.w	r3, r3, #4194304	; 0x400000
 80011fe:	f5b3 0f80 	cmp.w	r3, #4194304	; 0x400000
 8001202:	d10b      	bne.n	800121c <HAL_RCC_OscConfig+0x5c>
    {
      if((__HAL_RCC_GET_FLAG(RCC_FLAG_HSERDY) != RESET) && (RCC_OscInitStruct->HSEState == RCC_HSE_OFF))
 8001204:	4b7e      	ldr	r3, [pc, #504]	; (8001400 <HAL_RCC_OscConfig+0x240>)
 8001206:	681b      	ldr	r3, [r3, #0]
 8001208:	f403 3300 	and.w	r3, r3, #131072	; 0x20000
 800120c:	2b00      	cmp	r3, #0
 800120e:	d05b      	beq.n	80012c8 <HAL_RCC_OscConfig+0x108>
 8001210:	687b      	ldr	r3, [r7, #4]
 8001212:	685b      	ldr	r3, [r3, #4]
 8001214:	2b00      	cmp	r3, #0
 8001216:	d157      	bne.n	80012c8 <HAL_RCC_OscConfig+0x108>
      {
        return HAL_ERROR;
 8001218:	2301      	movs	r3, #1
 800121a:	e242      	b.n	80016a2 <HAL_RCC_OscConfig+0x4e2>
      }
    }
    else
    {
      /* Set the new HSE configuration ---------------------------------------*/
      __HAL_RCC_HSE_CONFIG(RCC_OscInitStruct->HSEState);
 800121c:	687b      	ldr	r3, [r7, #4]
 800121e:	685b      	ldr	r3, [r3, #4]
 8001220:	f5b3 3f80 	cmp.w	r3, #65536	; 0x10000
 8001224:	d106      	bne.n	8001234 <HAL_RCC_OscConfig+0x74>
 8001226:	4b76      	ldr	r3, [pc, #472]	; (8001400 <HAL_RCC_OscConfig+0x240>)
 8001228:	681b      	ldr	r3, [r3, #0]
 800122a:	4a75      	ldr	r2, [pc, #468]	; (8001400 <HAL_RCC_OscConfig+0x240>)
 800122c:	f443 3380 	orr.w	r3, r3, #65536	; 0x10000
 8001230:	6013      	str	r3, [r2, #0]
 8001232:	e01d      	b.n	8001270 <HAL_RCC_OscConfig+0xb0>
 8001234:	687b      	ldr	r3, [r7, #4]
 8001236:	685b      	ldr	r3, [r3, #4]
 8001238:	f5b3 2fa0 	cmp.w	r3, #327680	; 0x50000
 800123c:	d10c      	bne.n	8001258 <HAL_RCC_OscConfig+0x98>
 800123e:	4b70      	ldr	r3, [pc, #448]	; (8001400 <HAL_RCC_OscConfig+0x240>)
 8001240:	681b      	ldr	r3, [r3, #0]
 8001242:	4a6f      	ldr	r2, [pc, #444]	; (8001400 <HAL_RCC_OscConfig+0x240>)
 8001244:	f443 2380 	orr.w	r3, r3, #262144	; 0x40000
 8001248:	6013      	str	r3, [r2, #0]
 800124a:	4b6d      	ldr	r3, [pc, #436]	; (8001400 <HAL_RCC_OscConfig+0x240>)
 800124c:	681b      	ldr	r3, [r3, #0]
 800124e:	4a6c      	ldr	r2, [pc, #432]	; (8001400 <HAL_RCC_OscConfig+0x240>)
 8001250:	f443 3380 	orr.w	r3, r3, #65536	; 0x10000
 8001254:	6013      	str	r3, [r2, #0]
 8001256:	e00b      	b.n	8001270 <HAL_RCC_OscConfig+0xb0>
 8001258:	4b69      	ldr	r3, [pc, #420]	; (8001400 <HAL_RCC_OscConfig+0x240>)
 800125a:	681b      	ldr	r3, [r3, #0]
 800125c:	4a68      	ldr	r2, [pc, #416]	; (8001400 <HAL_RCC_OscConfig+0x240>)
 800125e:	f423 3380 	bic.w	r3, r3, #65536	; 0x10000
 8001262:	6013      	str	r3, [r2, #0]
 8001264:	4b66      	ldr	r3, [pc, #408]	; (8001400 <HAL_RCC_OscConfig+0x240>)
 8001266:	681b      	ldr	r3, [r3, #0]
 8001268:	4a65      	ldr	r2, [pc, #404]	; (8001400 <HAL_RCC_OscConfig+0x240>)
 800126a:	f423 2380 	bic.w	r3, r3, #262144	; 0x40000
 800126e:	6013      	str	r3, [r2, #0]

      /* Check the HSE State */
      if((RCC_OscInitStruct->HSEState) != RCC_HSE_OFF)
 8001270:	687b      	ldr	r3, [r7, #4]
 8001272:	685b      	ldr	r3, [r3, #4]
 8001274:	2b00      	cmp	r3, #0
 8001276:	d013      	beq.n	80012a0 <HAL_RCC_OscConfig+0xe0>
      {
        /* Get Start Tick */
        tickstart = HAL_GetTick();
 8001278:	f7ff fcae 	bl	8000bd8 <HAL_GetTick>
 800127c:	6138      	str	r0, [r7, #16]

        /* Wait till HSE is ready */
        while(__HAL_RCC_GET_FLAG(RCC_FLAG_HSERDY) == RESET)
 800127e:	e008      	b.n	8001292 <HAL_RCC_OscConfig+0xd2>
        {
          if((HAL_GetTick() - tickstart ) > HSE_TIMEOUT_VALUE)
 8001280:	f7ff fcaa 	bl	8000bd8 <HAL_GetTick>
 8001284:	4602      	mov	r2, r0
 8001286:	693b      	ldr	r3, [r7, #16]
 8001288:	1ad3      	subs	r3, r2, r3
 800128a:	2b64      	cmp	r3, #100	; 0x64
 800128c:	d901      	bls.n	8001292 <HAL_RCC_OscConfig+0xd2>
          {
            return HAL_TIMEOUT;
 800128e:	2303      	movs	r3, #3
 8001290:	e207      	b.n	80016a2 <HAL_RCC_OscConfig+0x4e2>
        while(__HAL_RCC_GET_FLAG(RCC_FLAG_HSERDY) == RESET)
 8001292:	4b5b      	ldr	r3, [pc, #364]	; (8001400 <HAL_RCC_OscConfig+0x240>)
 8001294:	681b      	ldr	r3, [r3, #0]
 8001296:	f403 3300 	and.w	r3, r3, #131072	; 0x20000
 800129a:	2b00      	cmp	r3, #0
 800129c:	d0f0      	beq.n	8001280 <HAL_RCC_OscConfig+0xc0>
 800129e:	e014      	b.n	80012ca <HAL_RCC_OscConfig+0x10a>
        }
      }
      else
      {
        /* Get Start Tick */
        tickstart = HAL_GetTick();
 80012a0:	f7ff fc9a 	bl	8000bd8 <HAL_GetTick>
 80012a4:	6138      	str	r0, [r7, #16]

        /* Wait till HSE is bypassed or disabled */
        while(__HAL_RCC_GET_FLAG(RCC_FLAG_HSERDY) != RESET)
 80012a6:	e008      	b.n	80012ba <HAL_RCC_OscConfig+0xfa>
        {
          if((HAL_GetTick() - tickstart ) > HSE_TIMEOUT_VALUE)
 80012a8:	f7ff fc96 	bl	8000bd8 <HAL_GetTick>
 80012ac:	4602      	mov	r2, r0
 80012ae:	693b      	ldr	r3, [r7, #16]
 80012b0:	1ad3      	subs	r3, r2, r3
 80012b2:	2b64      	cmp	r3, #100	; 0x64
 80012b4:	d901      	bls.n	80012ba <HAL_RCC_OscConfig+0xfa>
          {
            return HAL_TIMEOUT;
 80012b6:	2303      	movs	r3, #3
 80012b8:	e1f3      	b.n	80016a2 <HAL_RCC_OscConfig+0x4e2>
        while(__HAL_RCC_GET_FLAG(RCC_FLAG_HSERDY) != RESET)
 80012ba:	4b51      	ldr	r3, [pc, #324]	; (8001400 <HAL_RCC_OscConfig+0x240>)
 80012bc:	681b      	ldr	r3, [r3, #0]
 80012be:	f403 3300 	and.w	r3, r3, #131072	; 0x20000
 80012c2:	2b00      	cmp	r3, #0
 80012c4:	d1f0      	bne.n	80012a8 <HAL_RCC_OscConfig+0xe8>
 80012c6:	e000      	b.n	80012ca <HAL_RCC_OscConfig+0x10a>
      if((__HAL_RCC_GET_FLAG(RCC_FLAG_HSERDY) != RESET) && (RCC_OscInitStruct->HSEState == RCC_HSE_OFF))
 80012c8:	bf00      	nop
        }
      }
    }
  }
  /*----------------------------- HSI Configuration --------------------------*/
  if(((RCC_OscInitStruct->OscillatorType) & RCC_OSCILLATORTYPE_HSI) == RCC_OSCILLATORTYPE_HSI)
 80012ca:	687b      	ldr	r3, [r7, #4]
 80012cc:	681b      	ldr	r3, [r3, #0]
 80012ce:	f003 0302 	and.w	r3, r3, #2
 80012d2:	2b00      	cmp	r3, #0
 80012d4:	d063      	beq.n	800139e <HAL_RCC_OscConfig+0x1de>
    /* Check the parameters */
    assert_param(IS_RCC_HSI(RCC_OscInitStruct->HSIState));
    assert_param(IS_RCC_CALIBRATION_VALUE(RCC_OscInitStruct->HSICalibrationValue));

    /* Check if HSI is used as system clock or as PLL source when PLL is selected as system clock */
    if((__HAL_RCC_GET_SYSCLK_SOURCE() == RCC_CFGR_SWS_HSI) ||\
 80012d6:	4b4a      	ldr	r3, [pc, #296]	; (8001400 <HAL_RCC_OscConfig+0x240>)
 80012d8:	689b      	ldr	r3, [r3, #8]
 80012da:	f003 030c 	and.w	r3, r3, #12
 80012de:	2b00      	cmp	r3, #0
 80012e0:	d00b      	beq.n	80012fa <HAL_RCC_OscConfig+0x13a>
      ((__HAL_RCC_GET_SYSCLK_SOURCE() == RCC_CFGR_SWS_PLL) && ((RCC->PLLCFGR & RCC_PLLCFGR_PLLSRC) == RCC_PLLCFGR_PLLSRC_HSI)))
 80012e2:	4b47      	ldr	r3, [pc, #284]	; (8001400 <HAL_RCC_OscConfig+0x240>)
 80012e4:	689b      	ldr	r3, [r3, #8]
 80012e6:	f003 030c 	and.w	r3, r3, #12
    if((__HAL_RCC_GET_SYSCLK_SOURCE() == RCC_CFGR_SWS_HSI) ||\
 80012ea:	2b08      	cmp	r3, #8
 80012ec:	d11c      	bne.n	8001328 <HAL_RCC_OscConfig+0x168>
      ((__HAL_RCC_GET_SYSCLK_SOURCE() == RCC_CFGR_SWS_PLL) && ((RCC->PLLCFGR & RCC_PLLCFGR_PLLSRC) == RCC_PLLCFGR_PLLSRC_HSI)))
 80012ee:	4b44      	ldr	r3, [pc, #272]	; (8001400 <HAL_RCC_OscConfig+0x240>)
 80012f0:	685b      	ldr	r3, [r3, #4]
 80012f2:	f403 0380 	and.w	r3, r3, #4194304	; 0x400000
 80012f6:	2b00      	cmp	r3, #0
 80012f8:	d116      	bne.n	8001328 <HAL_RCC_OscConfig+0x168>
    {
      /* When HSI is used as system clock it will not disabled */
      if((__HAL_RCC_GET_FLAG(RCC_FLAG_HSIRDY) != RESET) && (RCC_OscInitStruct->HSIState != RCC_HSI_ON))
 80012fa:	4b41      	ldr	r3, [pc, #260]	; (8001400 <HAL_RCC_OscConfig+0x240>)
 80012fc:	681b      	ldr	r3, [r3, #0]
 80012fe:	f003 0302 	and.w	r3, r3, #2
 8001302:	2b00      	cmp	r3, #0
 8001304:	d005      	beq.n	8001312 <HAL_RCC_OscConfig+0x152>
 8001306:	687b      	ldr	r3, [r7, #4]
 8001308:	68db      	ldr	r3, [r3, #12]
 800130a:	2b01      	cmp	r3, #1
 800130c:	d001      	beq.n	8001312 <HAL_RCC_OscConfig+0x152>
      {
        return HAL_ERROR;
 800130e:	2301      	movs	r3, #1
 8001310:	e1c7      	b.n	80016a2 <HAL_RCC_OscConfig+0x4e2>
      }
      /* Otherwise, just the calibration is allowed */
      else
      {
        /* Adjusts the Internal High Speed oscillator (HSI) calibration value.*/
        __HAL_RCC_HSI_CALIBRATIONVALUE_ADJUST(RCC_OscInitStruct->HSICalibrationValue);
 8001312:	4b3b      	ldr	r3, [pc, #236]	; (8001400 <HAL_RCC_OscConfig+0x240>)
 8001314:	681b      	ldr	r3, [r3, #0]
 8001316:	f023 02f8 	bic.w	r2, r3, #248	; 0xf8
 800131a:	687b      	ldr	r3, [r7, #4]
 800131c:	691b      	ldr	r3, [r3, #16]
 800131e:	00db      	lsls	r3, r3, #3
 8001320:	4937      	ldr	r1, [pc, #220]	; (8001400 <HAL_RCC_OscConfig+0x240>)
 8001322:	4313      	orrs	r3, r2
 8001324:	600b      	str	r3, [r1, #0]
      if((__HAL_RCC_GET_FLAG(RCC_FLAG_HSIRDY) != RESET) && (RCC_OscInitStruct->HSIState != RCC_HSI_ON))
 8001326:	e03a      	b.n	800139e <HAL_RCC_OscConfig+0x1de>
      }
    }
    else
    {
      /* Check the HSI State */
      if((RCC_OscInitStruct->HSIState)!= RCC_HSI_OFF)
 8001328:	687b      	ldr	r3, [r7, #4]
 800132a:	68db      	ldr	r3, [r3, #12]
 800132c:	2b00      	cmp	r3, #0
 800132e:	d020      	beq.n	8001372 <HAL_RCC_OscConfig+0x1b2>
      {
        /* Enable the Internal High Speed oscillator (HSI). */
        __HAL_RCC_HSI_ENABLE();
 8001330:	4b34      	ldr	r3, [pc, #208]	; (8001404 <HAL_RCC_OscConfig+0x244>)
 8001332:	2201      	movs	r2, #1
 8001334:	601a      	str	r2, [r3, #0]

        /* Get Start Tick*/
        tickstart = HAL_GetTick();
 8001336:	f7ff fc4f 	bl	8000bd8 <HAL_GetTick>
 800133a:	6138      	str	r0, [r7, #16]

        /* Wait till HSI is ready */
        while(__HAL_RCC_GET_FLAG(RCC_FLAG_HSIRDY) == RESET)
 800133c:	e008      	b.n	8001350 <HAL_RCC_OscConfig+0x190>
        {
          if((HAL_GetTick() - tickstart ) > HSI_TIMEOUT_VALUE)
 800133e:	f7ff fc4b 	bl	8000bd8 <HAL_GetTick>
 8001342:	4602      	mov	r2, r0
 8001344:	693b      	ldr	r3, [r7, #16]
 8001346:	1ad3      	subs	r3, r2, r3
 8001348:	2b02      	cmp	r3, #2
 800134a:	d901      	bls.n	8001350 <HAL_RCC_OscConfig+0x190>
          {
            return HAL_TIMEOUT;
 800134c:	2303      	movs	r3, #3
 800134e:	e1a8      	b.n	80016a2 <HAL_RCC_OscConfig+0x4e2>
        while(__HAL_RCC_GET_FLAG(RCC_FLAG_HSIRDY) == RESET)
 8001350:	4b2b      	ldr	r3, [pc, #172]	; (8001400 <HAL_RCC_OscConfig+0x240>)
 8001352:	681b      	ldr	r3, [r3, #0]
 8001354:	f003 0302 	and.w	r3, r3, #2
 8001358:	2b00      	cmp	r3, #0
 800135a:	d0f0      	beq.n	800133e <HAL_RCC_OscConfig+0x17e>
          }
        }

        /* Adjusts the Internal High Speed oscillator (HSI) calibration value. */
        __HAL_RCC_HSI_CALIBRATIONVALUE_ADJUST(RCC_OscInitStruct->HSICalibrationValue);
 800135c:	4b28      	ldr	r3, [pc, #160]	; (8001400 <HAL_RCC_OscConfig+0x240>)
 800135e:	681b      	ldr	r3, [r3, #0]
 8001360:	f023 02f8 	bic.w	r2, r3, #248	; 0xf8
 8001364:	687b      	ldr	r3, [r7, #4]
 8001366:	691b      	ldr	r3, [r3, #16]
 8001368:	00db      	lsls	r3, r3, #3
 800136a:	4925      	ldr	r1, [pc, #148]	; (8001400 <HAL_RCC_OscConfig+0x240>)
 800136c:	4313      	orrs	r3, r2
 800136e:	600b      	str	r3, [r1, #0]
 8001370:	e015      	b.n	800139e <HAL_RCC_OscConfig+0x1de>
      }
      else
      {
        /* Disable the Internal High Speed oscillator (HSI). */
        __HAL_RCC_HSI_DISABLE();
 8001372:	4b24      	ldr	r3, [pc, #144]	; (8001404 <HAL_RCC_OscConfig+0x244>)
 8001374:	2200      	movs	r2, #0
 8001376:	601a      	str	r2, [r3, #0]

        /* Get Start Tick*/
        tickstart = HAL_GetTick();
 8001378:	f7ff fc2e 	bl	8000bd8 <HAL_GetTick>
 800137c:	6138      	str	r0, [r7, #16]

        /* Wait till HSI is ready */
        while(__HAL_RCC_GET_FLAG(RCC_FLAG_HSIRDY) != RESET)
 800137e:	e008      	b.n	8001392 <HAL_RCC_OscConfig+0x1d2>
        {
          if((HAL_GetTick() - tickstart ) > HSI_TIMEOUT_VALUE)
 8001380:	f7ff fc2a 	bl	8000bd8 <HAL_GetTick>
 8001384:	4602      	mov	r2, r0
 8001386:	693b      	ldr	r3, [r7, #16]
 8001388:	1ad3      	subs	r3, r2, r3
 800138a:	2b02      	cmp	r3, #2
 800138c:	d901      	bls.n	8001392 <HAL_RCC_OscConfig+0x1d2>
          {
            return HAL_TIMEOUT;
 800138e:	2303      	movs	r3, #3
 8001390:	e187      	b.n	80016a2 <HAL_RCC_OscConfig+0x4e2>
        while(__HAL_RCC_GET_FLAG(RCC_FLAG_HSIRDY) != RESET)
 8001392:	4b1b      	ldr	r3, [pc, #108]	; (8001400 <HAL_RCC_OscConfig+0x240>)
 8001394:	681b      	ldr	r3, [r3, #0]
 8001396:	f003 0302 	and.w	r3, r3, #2
 800139a:	2b00      	cmp	r3, #0
 800139c:	d1f0      	bne.n	8001380 <HAL_RCC_OscConfig+0x1c0>
        }
      }
    }
  }
  /*------------------------------ LSI Configuration -------------------------*/
  if(((RCC_OscInitStruct->OscillatorType) & RCC_OSCILLATORTYPE_LSI) == RCC_OSCILLATORTYPE_LSI)
 800139e:	687b      	ldr	r3, [r7, #4]
 80013a0:	681b      	ldr	r3, [r3, #0]
 80013a2:	f003 0308 	and.w	r3, r3, #8
 80013a6:	2b00      	cmp	r3, #0
 80013a8:	d036      	beq.n	8001418 <HAL_RCC_OscConfig+0x258>
  {
    /* Check the parameters */
    assert_param(IS_RCC_LSI(RCC_OscInitStruct->LSIState));

    /* Check the LSI State */
    if((RCC_OscInitStruct->LSIState)!= RCC_LSI_OFF)
 80013aa:	687b      	ldr	r3, [r7, #4]
 80013ac:	695b      	ldr	r3, [r3, #20]
 80013ae:	2b00      	cmp	r3, #0
 80013b0:	d016      	beq.n	80013e0 <HAL_RCC_OscConfig+0x220>
    {
      /* Enable the Internal Low Speed oscillator (LSI). */
      __HAL_RCC_LSI_ENABLE();
 80013b2:	4b15      	ldr	r3, [pc, #84]	; (8001408 <HAL_RCC_OscConfig+0x248>)
 80013b4:	2201      	movs	r2, #1
 80013b6:	601a      	str	r2, [r3, #0]

      /* Get Start Tick*/
      tickstart = HAL_GetTick();
 80013b8:	f7ff fc0e 	bl	8000bd8 <HAL_GetTick>
 80013bc:	6138      	str	r0, [r7, #16]

      /* Wait till LSI is ready */
      while(__HAL_RCC_GET_FLAG(RCC_FLAG_LSIRDY) == RESET)
 80013be:	e008      	b.n	80013d2 <HAL_RCC_OscConfig+0x212>
      {
        if((HAL_GetTick() - tickstart ) > LSI_TIMEOUT_VALUE)
 80013c0:	f7ff fc0a 	bl	8000bd8 <HAL_GetTick>
 80013c4:	4602      	mov	r2, r0
 80013c6:	693b      	ldr	r3, [r7, #16]
 80013c8:	1ad3      	subs	r3, r2, r3
 80013ca:	2b02      	cmp	r3, #2
 80013cc:	d901      	bls.n	80013d2 <HAL_RCC_OscConfig+0x212>
        {
          return HAL_TIMEOUT;
 80013ce:	2303      	movs	r3, #3
 80013d0:	e167      	b.n	80016a2 <HAL_RCC_OscConfig+0x4e2>
      while(__HAL_RCC_GET_FLAG(RCC_FLAG_LSIRDY) == RESET)
 80013d2:	4b0b      	ldr	r3, [pc, #44]	; (8001400 <HAL_RCC_OscConfig+0x240>)
 80013d4:	6f5b      	ldr	r3, [r3, #116]	; 0x74
 80013d6:	f003 0302 	and.w	r3, r3, #2
 80013da:	2b00      	cmp	r3, #0
 80013dc:	d0f0      	beq.n	80013c0 <HAL_RCC_OscConfig+0x200>
 80013de:	e01b      	b.n	8001418 <HAL_RCC_OscConfig+0x258>
      }
    }
    else
    {
      /* Disable the Internal Low Speed oscillator (LSI). */
      __HAL_RCC_LSI_DISABLE();
 80013e0:	4b09      	ldr	r3, [pc, #36]	; (8001408 <HAL_RCC_OscConfig+0x248>)
 80013e2:	2200      	movs	r2, #0
 80013e4:	601a      	str	r2, [r3, #0]

      /* Get Start Tick */
      tickstart = HAL_GetTick();
 80013e6:	f7ff fbf7 	bl	8000bd8 <HAL_GetTick>
 80013ea:	6138      	str	r0, [r7, #16]

      /* Wait till LSI is ready */
      while(__HAL_RCC_GET_FLAG(RCC_FLAG_LSIRDY) != RESET)
 80013ec:	e00e      	b.n	800140c <HAL_RCC_OscConfig+0x24c>
      {
        if((HAL_GetTick() - tickstart ) > LSI_TIMEOUT_VALUE)
 80013ee:	f7ff fbf3 	bl	8000bd8 <HAL_GetTick>
 80013f2:	4602      	mov	r2, r0
 80013f4:	693b      	ldr	r3, [r7, #16]
 80013f6:	1ad3      	subs	r3, r2, r3
 80013f8:	2b02      	cmp	r3, #2
 80013fa:	d907      	bls.n	800140c <HAL_RCC_OscConfig+0x24c>
        {
          return HAL_TIMEOUT;
 80013fc:	2303      	movs	r3, #3
 80013fe:	e150      	b.n	80016a2 <HAL_RCC_OscConfig+0x4e2>
 8001400:	40023800 	.word	0x40023800
 8001404:	42470000 	.word	0x42470000
 8001408:	42470e80 	.word	0x42470e80
      while(__HAL_RCC_GET_FLAG(RCC_FLAG_LSIRDY) != RESET)
 800140c:	4b88      	ldr	r3, [pc, #544]	; (8001630 <HAL_RCC_OscConfig+0x470>)
 800140e:	6f5b      	ldr	r3, [r3, #116]	; 0x74
 8001410:	f003 0302 	and.w	r3, r3, #2
 8001414:	2b00      	cmp	r3, #0
 8001416:	d1ea      	bne.n	80013ee <HAL_RCC_OscConfig+0x22e>
        }
      }
    }
  }
  /*------------------------------ LSE Configuration -------------------------*/
  if(((RCC_OscInitStruct->OscillatorType) & RCC_OSCILLATORTYPE_LSE) == RCC_OSCILLATORTYPE_LSE)
 8001418:	687b      	ldr	r3, [r7, #4]
 800141a:	681b      	ldr	r3, [r3, #0]
 800141c:	f003 0304 	and.w	r3, r3, #4
 8001420:	2b00      	cmp	r3, #0
 8001422:	f000 8097 	beq.w	8001554 <HAL_RCC_OscConfig+0x394>
  {
    FlagStatus       pwrclkchanged = RESET;
 8001426:	2300      	movs	r3, #0
 8001428:	75fb      	strb	r3, [r7, #23]
    /* Check the parameters */
    assert_param(IS_RCC_LSE(RCC_OscInitStruct->LSEState));

    /* Update LSE configuration in Backup Domain control register    */
    /* Requires to enable write access to Backup Domain of necessary */
    if(__HAL_RCC_PWR_IS_CLK_DISABLED())
 800142a:	4b81      	ldr	r3, [pc, #516]	; (8001630 <HAL_RCC_OscConfig+0x470>)
 800142c:	6c1b      	ldr	r3, [r3, #64]	; 0x40
 800142e:	f003 5380 	and.w	r3, r3, #268435456	; 0x10000000
 8001432:	2b00      	cmp	r3, #0
 8001434:	d10f      	bne.n	8001456 <HAL_RCC_OscConfig+0x296>
    {
      __HAL_RCC_PWR_CLK_ENABLE();
 8001436:	2300      	movs	r3, #0
 8001438:	60bb      	str	r3, [r7, #8]
 800143a:	4b7d      	ldr	r3, [pc, #500]	; (8001630 <HAL_RCC_OscConfig+0x470>)
 800143c:	6c1b      	ldr	r3, [r3, #64]	; 0x40
 800143e:	4a7c      	ldr	r2, [pc, #496]	; (8001630 <HAL_RCC_OscConfig+0x470>)
 8001440:	f043 5380 	orr.w	r3, r3, #268435456	; 0x10000000
 8001444:	6413      	str	r3, [r2, #64]	; 0x40
 8001446:	4b7a      	ldr	r3, [pc, #488]	; (8001630 <HAL_RCC_OscConfig+0x470>)
 8001448:	6c1b      	ldr	r3, [r3, #64]	; 0x40
 800144a:	f003 5380 	and.w	r3, r3, #268435456	; 0x10000000
 800144e:	60bb      	str	r3, [r7, #8]
 8001450:	68bb      	ldr	r3, [r7, #8]
      pwrclkchanged = SET;
 8001452:	2301      	movs	r3, #1
 8001454:	75fb      	strb	r3, [r7, #23]
    }

    if(HAL_IS_BIT_CLR(PWR->CR, PWR_CR_DBP))
 8001456:	4b77      	ldr	r3, [pc, #476]	; (8001634 <HAL_RCC_OscConfig+0x474>)
 8001458:	681b      	ldr	r3, [r3, #0]
 800145a:	f403 7380 	and.w	r3, r3, #256	; 0x100
 800145e:	2b00      	cmp	r3, #0
 8001460:	d118      	bne.n	8001494 <HAL_RCC_OscConfig+0x2d4>
    {
      /* Enable write access to Backup domain */
      SET_BIT(PWR->CR, PWR_CR_DBP);
 8001462:	4b74      	ldr	r3, [pc, #464]	; (8001634 <HAL_RCC_OscConfig+0x474>)
 8001464:	681b      	ldr	r3, [r3, #0]
 8001466:	4a73      	ldr	r2, [pc, #460]	; (8001634 <HAL_RCC_OscConfig+0x474>)
 8001468:	f443 7380 	orr.w	r3, r3, #256	; 0x100
 800146c:	6013      	str	r3, [r2, #0]

      /* Wait for Backup domain Write protection disable */
      tickstart = HAL_GetTick();
 800146e:	f7ff fbb3 	bl	8000bd8 <HAL_GetTick>
 8001472:	6138      	str	r0, [r7, #16]

      while(HAL_IS_BIT_CLR(PWR->CR, PWR_CR_DBP))
 8001474:	e008      	b.n	8001488 <HAL_RCC_OscConfig+0x2c8>
      {
        if((HAL_GetTick() - tickstart) > RCC_DBP_TIMEOUT_VALUE)
 8001476:	f7ff fbaf 	bl	8000bd8 <HAL_GetTick>
 800147a:	4602      	mov	r2, r0
 800147c:	693b      	ldr	r3, [r7, #16]
 800147e:	1ad3      	subs	r3, r2, r3
 8001480:	2b02      	cmp	r3, #2
 8001482:	d901      	bls.n	8001488 <HAL_RCC_OscConfig+0x2c8>
        {
          return HAL_TIMEOUT;
 8001484:	2303      	movs	r3, #3
 8001486:	e10c      	b.n	80016a2 <HAL_RCC_OscConfig+0x4e2>
      while(HAL_IS_BIT_CLR(PWR->CR, PWR_CR_DBP))
 8001488:	4b6a      	ldr	r3, [pc, #424]	; (8001634 <HAL_RCC_OscConfig+0x474>)
 800148a:	681b      	ldr	r3, [r3, #0]
 800148c:	f403 7380 	and.w	r3, r3, #256	; 0x100
 8001490:	2b00      	cmp	r3, #0
 8001492:	d0f0      	beq.n	8001476 <HAL_RCC_OscConfig+0x2b6>
        }
      }
    }

    /* Set the new LSE configuration -----------------------------------------*/
    __HAL_RCC_LSE_CONFIG(RCC_OscInitStruct->LSEState);
 8001494:	687b      	ldr	r3, [r7, #4]
 8001496:	689b      	ldr	r3, [r3, #8]
 8001498:	2b01      	cmp	r3, #1
 800149a:	d106      	bne.n	80014aa <HAL_RCC_OscConfig+0x2ea>
 800149c:	4b64      	ldr	r3, [pc, #400]	; (8001630 <HAL_RCC_OscConfig+0x470>)
 800149e:	6f1b      	ldr	r3, [r3, #112]	; 0x70
 80014a0:	4a63      	ldr	r2, [pc, #396]	; (8001630 <HAL_RCC_OscConfig+0x470>)
 80014a2:	f043 0301 	orr.w	r3, r3, #1
 80014a6:	6713      	str	r3, [r2, #112]	; 0x70
 80014a8:	e01c      	b.n	80014e4 <HAL_RCC_OscConfig+0x324>
 80014aa:	687b      	ldr	r3, [r7, #4]
 80014ac:	689b      	ldr	r3, [r3, #8]
 80014ae:	2b05      	cmp	r3, #5
 80014b0:	d10c      	bne.n	80014cc <HAL_RCC_OscConfig+0x30c>
 80014b2:	4b5f      	ldr	r3, [pc, #380]	; (8001630 <HAL_RCC_OscConfig+0x470>)
 80014b4:	6f1b      	ldr	r3, [r3, #112]	; 0x70
 80014b6:	4a5e      	ldr	r2, [pc, #376]	; (8001630 <HAL_RCC_OscConfig+0x470>)
 80014b8:	f043 0304 	orr.w	r3, r3, #4
 80014bc:	6713      	str	r3, [r2, #112]	; 0x70
 80014be:	4b5c      	ldr	r3, [pc, #368]	; (8001630 <HAL_RCC_OscConfig+0x470>)
 80014c0:	6f1b      	ldr	r3, [r3, #112]	; 0x70
 80014c2:	4a5b      	ldr	r2, [pc, #364]	; (8001630 <HAL_RCC_OscConfig+0x470>)
 80014c4:	f043 0301 	orr.w	r3, r3, #1
 80014c8:	6713      	str	r3, [r2, #112]	; 0x70
 80014ca:	e00b      	b.n	80014e4 <HAL_RCC_OscConfig+0x324>
 80014cc:	4b58      	ldr	r3, [pc, #352]	; (8001630 <HAL_RCC_OscConfig+0x470>)
 80014ce:	6f1b      	ldr	r3, [r3, #112]	; 0x70
 80014d0:	4a57      	ldr	r2, [pc, #348]	; (8001630 <HAL_RCC_OscConfig+0x470>)
 80014d2:	f023 0301 	bic.w	r3, r3, #1
 80014d6:	6713      	str	r3, [r2, #112]	; 0x70
 80014d8:	4b55      	ldr	r3, [pc, #340]	; (8001630 <HAL_RCC_OscConfig+0x470>)
 80014da:	6f1b      	ldr	r3, [r3, #112]	; 0x70
 80014dc:	4a54      	ldr	r2, [pc, #336]	; (8001630 <HAL_RCC_OscConfig+0x470>)
 80014de:	f023 0304 	bic.w	r3, r3, #4
 80014e2:	6713      	str	r3, [r2, #112]	; 0x70
    /* Check the LSE State */
    if((RCC_OscInitStruct->LSEState) != RCC_LSE_OFF)
 80014e4:	687b      	ldr	r3, [r7, #4]
 80014e6:	689b      	ldr	r3, [r3, #8]
 80014e8:	2b00      	cmp	r3, #0
 80014ea:	d015      	beq.n	8001518 <HAL_RCC_OscConfig+0x358>
    {
      /* Get Start Tick*/
      tickstart = HAL_GetTick();
 80014ec:	f7ff fb74 	bl	8000bd8 <HAL_GetTick>
 80014f0:	6138      	str	r0, [r7, #16]

      /* Wait till LSE is ready */
      while(__HAL_RCC_GET_FLAG(RCC_FLAG_LSERDY) == RESET)
 80014f2:	e00a      	b.n	800150a <HAL_RCC_OscConfig+0x34a>
      {
        if((HAL_GetTick() - tickstart ) > RCC_LSE_TIMEOUT_VALUE)
 80014f4:	f7ff fb70 	bl	8000bd8 <HAL_GetTick>
 80014f8:	4602      	mov	r2, r0
 80014fa:	693b      	ldr	r3, [r7, #16]
 80014fc:	1ad3      	subs	r3, r2, r3
 80014fe:	f241 3288 	movw	r2, #5000	; 0x1388
 8001502:	4293      	cmp	r3, r2
 8001504:	d901      	bls.n	800150a <HAL_RCC_OscConfig+0x34a>
        {
          return HAL_TIMEOUT;
 8001506:	2303      	movs	r3, #3
 8001508:	e0cb      	b.n	80016a2 <HAL_RCC_OscConfig+0x4e2>
      while(__HAL_RCC_GET_FLAG(RCC_FLAG_LSERDY) == RESET)
 800150a:	4b49      	ldr	r3, [pc, #292]	; (8001630 <HAL_RCC_OscConfig+0x470>)
 800150c:	6f1b      	ldr	r3, [r3, #112]	; 0x70
 800150e:	f003 0302 	and.w	r3, r3, #2
 8001512:	2b00      	cmp	r3, #0
 8001514:	d0ee      	beq.n	80014f4 <HAL_RCC_OscConfig+0x334>
 8001516:	e014      	b.n	8001542 <HAL_RCC_OscConfig+0x382>
      }
    }
    else
    {
      /* Get Start Tick */
      tickstart = HAL_GetTick();
 8001518:	f7ff fb5e 	bl	8000bd8 <HAL_GetTick>
 800151c:	6138      	str	r0, [r7, #16]

      /* Wait till LSE is ready */
      while(__HAL_RCC_GET_FLAG(RCC_FLAG_LSERDY) != RESET)
 800151e:	e00a      	b.n	8001536 <HAL_RCC_OscConfig+0x376>
      {
        if((HAL_GetTick() - tickstart ) > RCC_LSE_TIMEOUT_VALUE)
 8001520:	f7ff fb5a 	bl	8000bd8 <HAL_GetTick>
 8001524:	4602      	mov	r2, r0
 8001526:	693b      	ldr	r3, [r7, #16]
 8001528:	1ad3      	subs	r3, r2, r3
 800152a:	f241 3288 	movw	r2, #5000	; 0x1388
 800152e:	4293      	cmp	r3, r2
 8001530:	d901      	bls.n	8001536 <HAL_RCC_OscConfig+0x376>
        {
          return HAL_TIMEOUT;
 8001532:	2303      	movs	r3, #3
 8001534:	e0b5      	b.n	80016a2 <HAL_RCC_OscConfig+0x4e2>
      while(__HAL_RCC_GET_FLAG(RCC_FLAG_LSERDY) != RESET)
 8001536:	4b3e      	ldr	r3, [pc, #248]	; (8001630 <HAL_RCC_OscConfig+0x470>)
 8001538:	6f1b      	ldr	r3, [r3, #112]	; 0x70
 800153a:	f003 0302 	and.w	r3, r3, #2
 800153e:	2b00      	cmp	r3, #0
 8001540:	d1ee      	bne.n	8001520 <HAL_RCC_OscConfig+0x360>
        }
      }
    }

    /* Restore clock configuration if changed */
    if(pwrclkchanged == SET)
 8001542:	7dfb      	ldrb	r3, [r7, #23]
 8001544:	2b01      	cmp	r3, #1
 8001546:	d105      	bne.n	8001554 <HAL_RCC_OscConfig+0x394>
    {
      __HAL_RCC_PWR_CLK_DISABLE();
 8001548:	4b39      	ldr	r3, [pc, #228]	; (8001630 <HAL_RCC_OscConfig+0x470>)
 800154a:	6c1b      	ldr	r3, [r3, #64]	; 0x40
 800154c:	4a38      	ldr	r2, [pc, #224]	; (8001630 <HAL_RCC_OscConfig+0x470>)
 800154e:	f023 5380 	bic.w	r3, r3, #268435456	; 0x10000000
 8001552:	6413      	str	r3, [r2, #64]	; 0x40
    }
  }
  /*-------------------------------- PLL Configuration -----------------------*/
  /* Check the parameters */
  assert_param(IS_RCC_PLL(RCC_OscInitStruct->PLL.PLLState));
  if ((RCC_OscInitStruct->PLL.PLLState) != RCC_PLL_NONE)
 8001554:	687b      	ldr	r3, [r7, #4]
 8001556:	699b      	ldr	r3, [r3, #24]
 8001558:	2b00      	cmp	r3, #0
 800155a:	f000 80a1 	beq.w	80016a0 <HAL_RCC_OscConfig+0x4e0>
  {
    /* Check if the PLL is used as system clock or not */
    if(__HAL_RCC_GET_SYSCLK_SOURCE() != RCC_CFGR_SWS_PLL)
 800155e:	4b34      	ldr	r3, [pc, #208]	; (8001630 <HAL_RCC_OscConfig+0x470>)
 8001560:	689b      	ldr	r3, [r3, #8]
 8001562:	f003 030c 	and.w	r3, r3, #12
 8001566:	2b08      	cmp	r3, #8
 8001568:	d05c      	beq.n	8001624 <HAL_RCC_OscConfig+0x464>
    {
      if((RCC_OscInitStruct->PLL.PLLState) == RCC_PLL_ON)
 800156a:	687b      	ldr	r3, [r7, #4]
 800156c:	699b      	ldr	r3, [r3, #24]
 800156e:	2b02      	cmp	r3, #2
 8001570:	d141      	bne.n	80015f6 <HAL_RCC_OscConfig+0x436>
        assert_param(IS_RCC_PLLN_VALUE(RCC_OscInitStruct->PLL.PLLN));
        assert_param(IS_RCC_PLLP_VALUE(RCC_OscInitStruct->PLL.PLLP));
        assert_param(IS_RCC_PLLQ_VALUE(RCC_OscInitStruct->PLL.PLLQ));

        /* Disable the main PLL. */
        __HAL_RCC_PLL_DISABLE();
 8001572:	4b31      	ldr	r3, [pc, #196]	; (8001638 <HAL_RCC_OscConfig+0x478>)
 8001574:	2200      	movs	r2, #0
 8001576:	601a      	str	r2, [r3, #0]

        /* Get Start Tick */
        tickstart = HAL_GetTick();
 8001578:	f7ff fb2e 	bl	8000bd8 <HAL_GetTick>
 800157c:	6138      	str	r0, [r7, #16]

        /* Wait till PLL is ready */
        while(__HAL_RCC_GET_FLAG(RCC_FLAG_PLLRDY) != RESET)
 800157e:	e008      	b.n	8001592 <HAL_RCC_OscConfig+0x3d2>
        {
          if((HAL_GetTick() - tickstart ) > PLL_TIMEOUT_VALUE)
 8001580:	f7ff fb2a 	bl	8000bd8 <HAL_GetTick>
 8001584:	4602      	mov	r2, r0
 8001586:	693b      	ldr	r3, [r7, #16]
 8001588:	1ad3      	subs	r3, r2, r3
 800158a:	2b02      	cmp	r3, #2
 800158c:	d901      	bls.n	8001592 <HAL_RCC_OscConfig+0x3d2>
          {
            return HAL_TIMEOUT;
 800158e:	2303      	movs	r3, #3
 8001590:	e087      	b.n	80016a2 <HAL_RCC_OscConfig+0x4e2>
        while(__HAL_RCC_GET_FLAG(RCC_FLAG_PLLRDY) != RESET)
 8001592:	4b27      	ldr	r3, [pc, #156]	; (8001630 <HAL_RCC_OscConfig+0x470>)
 8001594:	681b      	ldr	r3, [r3, #0]
 8001596:	f003 7300 	and.w	r3, r3, #33554432	; 0x2000000
 800159a:	2b00      	cmp	r3, #0
 800159c:	d1f0      	bne.n	8001580 <HAL_RCC_OscConfig+0x3c0>
          }
        }

        /* Configure the main PLL clock source, multiplication and division factors. */
        WRITE_REG(RCC->PLLCFGR, (RCC_OscInitStruct->PLL.PLLSource                                            | \
 800159e:	687b      	ldr	r3, [r7, #4]
 80015a0:	69da      	ldr	r2, [r3, #28]
 80015a2:	687b      	ldr	r3, [r7, #4]
 80015a4:	6a1b      	ldr	r3, [r3, #32]
 80015a6:	431a      	orrs	r2, r3
 80015a8:	687b      	ldr	r3, [r7, #4]
 80015aa:	6a5b      	ldr	r3, [r3, #36]	; 0x24
 80015ac:	019b      	lsls	r3, r3, #6
 80015ae:	431a      	orrs	r2, r3
 80015b0:	687b      	ldr	r3, [r7, #4]
 80015b2:	6a9b      	ldr	r3, [r3, #40]	; 0x28
 80015b4:	085b      	lsrs	r3, r3, #1
 80015b6:	3b01      	subs	r3, #1
 80015b8:	041b      	lsls	r3, r3, #16
 80015ba:	431a      	orrs	r2, r3
 80015bc:	687b      	ldr	r3, [r7, #4]
 80015be:	6adb      	ldr	r3, [r3, #44]	; 0x2c
 80015c0:	061b      	lsls	r3, r3, #24
 80015c2:	491b      	ldr	r1, [pc, #108]	; (8001630 <HAL_RCC_OscConfig+0x470>)
 80015c4:	4313      	orrs	r3, r2
 80015c6:	604b      	str	r3, [r1, #4]
                                 RCC_OscInitStruct->PLL.PLLM                                                 | \
                                 (RCC_OscInitStruct->PLL.PLLN << RCC_PLLCFGR_PLLN_Pos)             | \
                                 (((RCC_OscInitStruct->PLL.PLLP >> 1U) - 1U) << RCC_PLLCFGR_PLLP_Pos) | \
                                 (RCC_OscInitStruct->PLL.PLLQ << RCC_PLLCFGR_PLLQ_Pos)));
        /* Enable the main PLL. */
        __HAL_RCC_PLL_ENABLE();
 80015c8:	4b1b      	ldr	r3, [pc, #108]	; (8001638 <HAL_RCC_OscConfig+0x478>)
 80015ca:	2201      	movs	r2, #1
 80015cc:	601a      	str	r2, [r3, #0]

        /* Get Start Tick */
        tickstart = HAL_GetTick();
 80015ce:	f7ff fb03 	bl	8000bd8 <HAL_GetTick>
 80015d2:	6138      	str	r0, [r7, #16]

        /* Wait till PLL is ready */
        while(__HAL_RCC_GET_FLAG(RCC_FLAG_PLLRDY) == RESET)
 80015d4:	e008      	b.n	80015e8 <HAL_RCC_OscConfig+0x428>
        {
          if((HAL_GetTick() - tickstart ) > PLL_TIMEOUT_VALUE)
 80015d6:	f7ff faff 	bl	8000bd8 <HAL_GetTick>
 80015da:	4602      	mov	r2, r0
 80015dc:	693b      	ldr	r3, [r7, #16]
 80015de:	1ad3      	subs	r3, r2, r3
 80015e0:	2b02      	cmp	r3, #2
 80015e2:	d901      	bls.n	80015e8 <HAL_RCC_OscConfig+0x428>
          {
            return HAL_TIMEOUT;
 80015e4:	2303      	movs	r3, #3
 80015e6:	e05c      	b.n	80016a2 <HAL_RCC_OscConfig+0x4e2>
        while(__HAL_RCC_GET_FLAG(RCC_FLAG_PLLRDY) == RESET)
 80015e8:	4b11      	ldr	r3, [pc, #68]	; (8001630 <HAL_RCC_OscConfig+0x470>)
 80015ea:	681b      	ldr	r3, [r3, #0]
 80015ec:	f003 7300 	and.w	r3, r3, #33554432	; 0x2000000
 80015f0:	2b00      	cmp	r3, #0
 80015f2:	d0f0      	beq.n	80015d6 <HAL_RCC_OscConfig+0x416>
 80015f4:	e054      	b.n	80016a0 <HAL_RCC_OscConfig+0x4e0>
        }
      }
      else
      {
        /* Disable the main PLL. */
        __HAL_RCC_PLL_DISABLE();
 80015f6:	4b10      	ldr	r3, [pc, #64]	; (8001638 <HAL_RCC_OscConfig+0x478>)
 80015f8:	2200      	movs	r2, #0
 80015fa:	601a      	str	r2, [r3, #0]

        /* Get Start Tick */
        tickstart = HAL_GetTick();
 80015fc:	f7ff faec 	bl	8000bd8 <HAL_GetTick>
 8001600:	6138      	str	r0, [r7, #16]

        /* Wait till PLL is ready */
        while(__HAL_RCC_GET_FLAG(RCC_FLAG_PLLRDY) != RESET)
 8001602:	e008      	b.n	8001616 <HAL_RCC_OscConfig+0x456>
        {
          if((HAL_GetTick() - tickstart ) > PLL_TIMEOUT_VALUE)
 8001604:	f7ff fae8 	bl	8000bd8 <HAL_GetTick>
 8001608:	4602      	mov	r2, r0
 800160a:	693b      	ldr	r3, [r7, #16]
 800160c:	1ad3      	subs	r3, r2, r3
 800160e:	2b02      	cmp	r3, #2
 8001610:	d901      	bls.n	8001616 <HAL_RCC_OscConfig+0x456>
          {
            return HAL_TIMEOUT;
 8001612:	2303      	movs	r3, #3
 8001614:	e045      	b.n	80016a2 <HAL_RCC_OscConfig+0x4e2>
        while(__HAL_RCC_GET_FLAG(RCC_FLAG_PLLRDY) != RESET)
 8001616:	4b06      	ldr	r3, [pc, #24]	; (8001630 <HAL_RCC_OscConfig+0x470>)
 8001618:	681b      	ldr	r3, [r3, #0]
 800161a:	f003 7300 	and.w	r3, r3, #33554432	; 0x2000000
 800161e:	2b00      	cmp	r3, #0
 8001620:	d1f0      	bne.n	8001604 <HAL_RCC_OscConfig+0x444>
 8001622:	e03d      	b.n	80016a0 <HAL_RCC_OscConfig+0x4e0>
      }
    }
    else
    {
      /* Check if there is a request to disable the PLL used as System clock source */
      if((RCC_OscInitStruct->PLL.PLLState) == RCC_PLL_OFF)
 8001624:	687b      	ldr	r3, [r7, #4]
 8001626:	699b      	ldr	r3, [r3, #24]
 8001628:	2b01      	cmp	r3, #1
 800162a:	d107      	bne.n	800163c <HAL_RCC_OscConfig+0x47c>
      {
        return HAL_ERROR;
 800162c:	2301      	movs	r3, #1
 800162e:	e038      	b.n	80016a2 <HAL_RCC_OscConfig+0x4e2>
 8001630:	40023800 	.word	0x40023800
 8001634:	40007000 	.word	0x40007000
 8001638:	42470060 	.word	0x42470060
      }
      else
      {
        /* Do not return HAL_ERROR if request repeats the current configuration */
        pll_config = RCC->PLLCFGR;
 800163c:	4b1b      	ldr	r3, [pc, #108]	; (80016ac <HAL_RCC_OscConfig+0x4ec>)
 800163e:	685b      	ldr	r3, [r3, #4]
 8001640:	60fb      	str	r3, [r7, #12]
            (READ_BIT(pll_config, RCC_PLLCFGR_PLLN) != (RCC_OscInitStruct->PLL.PLLN) << RCC_PLLCFGR_PLLN_Pos) ||
            (READ_BIT(pll_config, RCC_PLLCFGR_PLLP) != (((RCC_OscInitStruct->PLL.PLLP >> 1U) - 1U)) << RCC_PLLCFGR_PLLP_Pos) ||
            (READ_BIT(pll_config, RCC_PLLCFGR_PLLQ) != (RCC_OscInitStruct->PLL.PLLQ << RCC_PLLCFGR_PLLQ_Pos)) ||
            (READ_BIT(pll_config, RCC_PLLCFGR_PLLR) != (RCC_OscInitStruct->PLL.PLLR << RCC_PLLCFGR_PLLR_Pos)))
#else
        if (((RCC_OscInitStruct->PLL.PLLState) == RCC_PLL_OFF) ||
 8001642:	687b      	ldr	r3, [r7, #4]
 8001644:	699b      	ldr	r3, [r3, #24]
 8001646:	2b01      	cmp	r3, #1
 8001648:	d028      	beq.n	800169c <HAL_RCC_OscConfig+0x4dc>
            (READ_BIT(pll_config, RCC_PLLCFGR_PLLSRC) != RCC_OscInitStruct->PLL.PLLSource) ||
 800164a:	68fb      	ldr	r3, [r7, #12]
 800164c:	f403 0280 	and.w	r2, r3, #4194304	; 0x400000
 8001650:	687b      	ldr	r3, [r7, #4]
 8001652:	69db      	ldr	r3, [r3, #28]
        if (((RCC_OscInitStruct->PLL.PLLState) == RCC_PLL_OFF) ||
 8001654:	429a      	cmp	r2, r3
 8001656:	d121      	bne.n	800169c <HAL_RCC_OscConfig+0x4dc>
            (READ_BIT(pll_config, RCC_PLLCFGR_PLLM) != (RCC_OscInitStruct->PLL.PLLM) << RCC_PLLCFGR_PLLM_Pos) ||
 8001658:	68fb      	ldr	r3, [r7, #12]
 800165a:	f003 023f 	and.w	r2, r3, #63	; 0x3f
 800165e:	687b      	ldr	r3, [r7, #4]
 8001660:	6a1b      	ldr	r3, [r3, #32]
            (READ_BIT(pll_config, RCC_PLLCFGR_PLLSRC) != RCC_OscInitStruct->PLL.PLLSource) ||
 8001662:	429a      	cmp	r2, r3
 8001664:	d11a      	bne.n	800169c <HAL_RCC_OscConfig+0x4dc>
            (READ_BIT(pll_config, RCC_PLLCFGR_PLLN) != (RCC_OscInitStruct->PLL.PLLN) << RCC_PLLCFGR_PLLN_Pos) ||
 8001666:	68fa      	ldr	r2, [r7, #12]
 8001668:	f647 73c0 	movw	r3, #32704	; 0x7fc0
 800166c:	4013      	ands	r3, r2
 800166e:	687a      	ldr	r2, [r7, #4]
 8001670:	6a52      	ldr	r2, [r2, #36]	; 0x24
 8001672:	0192      	lsls	r2, r2, #6
            (READ_BIT(pll_config, RCC_PLLCFGR_PLLM) != (RCC_OscInitStruct->PLL.PLLM) << RCC_PLLCFGR_PLLM_Pos) ||
 8001674:	4293      	cmp	r3, r2
 8001676:	d111      	bne.n	800169c <HAL_RCC_OscConfig+0x4dc>
            (READ_BIT(pll_config, RCC_PLLCFGR_PLLP) != (((RCC_OscInitStruct->PLL.PLLP >> 1U) - 1U)) << RCC_PLLCFGR_PLLP_Pos) ||
 8001678:	68fb      	ldr	r3, [r7, #12]
 800167a:	f403 3240 	and.w	r2, r3, #196608	; 0x30000
 800167e:	687b      	ldr	r3, [r7, #4]
 8001680:	6a9b      	ldr	r3, [r3, #40]	; 0x28
 8001682:	085b      	lsrs	r3, r3, #1
 8001684:	3b01      	subs	r3, #1
 8001686:	041b      	lsls	r3, r3, #16
            (READ_BIT(pll_config, RCC_PLLCFGR_PLLN) != (RCC_OscInitStruct->PLL.PLLN) << RCC_PLLCFGR_PLLN_Pos) ||
 8001688:	429a      	cmp	r2, r3
 800168a:	d107      	bne.n	800169c <HAL_RCC_OscConfig+0x4dc>
            (READ_BIT(pll_config, RCC_PLLCFGR_PLLQ) != (RCC_OscInitStruct->PLL.PLLQ << RCC_PLLCFGR_PLLQ_Pos)))
 800168c:	68fb      	ldr	r3, [r7, #12]
 800168e:	f003 6270 	and.w	r2, r3, #251658240	; 0xf000000
 8001692:	687b      	ldr	r3, [r7, #4]
 8001694:	6adb      	ldr	r3, [r3, #44]	; 0x2c
 8001696:	061b      	lsls	r3, r3, #24
            (READ_BIT(pll_config, RCC_PLLCFGR_PLLP) != (((RCC_OscInitStruct->PLL.PLLP >> 1U) - 1U)) << RCC_PLLCFGR_PLLP_Pos) ||
 8001698:	429a      	cmp	r2, r3
 800169a:	d001      	beq.n	80016a0 <HAL_RCC_OscConfig+0x4e0>
#endif
        {
          return HAL_ERROR;
 800169c:	2301      	movs	r3, #1
 800169e:	e000      	b.n	80016a2 <HAL_RCC_OscConfig+0x4e2>
        }
      }
    }
  }
  return HAL_OK;
 80016a0:	2300      	movs	r3, #0
}
 80016a2:	4618      	mov	r0, r3
 80016a4:	3718      	adds	r7, #24
 80016a6:	46bd      	mov	sp, r7
 80016a8:	bd80      	pop	{r7, pc}
 80016aa:	bf00      	nop
 80016ac:	40023800 	.word	0x40023800

080016b0 <HAL_RCC_ClockConfig>:
  *         HPRE[3:0] bits to ensure that HCLK not exceed the maximum allowed frequency
  *         (for more details refer to section above "Initialization/de-initialization functions")
  * @retval None
  */
HAL_StatusTypeDef HAL_RCC_ClockConfig(RCC_ClkInitTypeDef  *RCC_ClkInitStruct, uint32_t FLatency)
{
 80016b0:	b580      	push	{r7, lr}
 80016b2:	b084      	sub	sp, #16
 80016b4:	af00      	add	r7, sp, #0
 80016b6:	6078      	str	r0, [r7, #4]
 80016b8:	6039      	str	r1, [r7, #0]
  uint32_t tickstart;

  /* Check Null pointer */
  if(RCC_ClkInitStruct == NULL)
 80016ba:	687b      	ldr	r3, [r7, #4]
 80016bc:	2b00      	cmp	r3, #0
 80016be:	d101      	bne.n	80016c4 <HAL_RCC_ClockConfig+0x14>
  {
    return HAL_ERROR;
 80016c0:	2301      	movs	r3, #1
 80016c2:	e0cc      	b.n	800185e <HAL_RCC_ClockConfig+0x1ae>
  /* To correctly read data from FLASH memory, the number of wait states (LATENCY)
    must be correctly programmed according to the frequency of the CPU clock
    (HCLK) and the supply voltage of the device. */

  /* Increasing the number of wait states because of higher CPU frequency */
  if(FLatency > __HAL_FLASH_GET_LATENCY())
 80016c4:	4b68      	ldr	r3, [pc, #416]	; (8001868 <HAL_RCC_ClockConfig+0x1b8>)
 80016c6:	681b      	ldr	r3, [r3, #0]
 80016c8:	f003 030f 	and.w	r3, r3, #15
 80016cc:	683a      	ldr	r2, [r7, #0]
 80016ce:	429a      	cmp	r2, r3
 80016d0:	d90c      	bls.n	80016ec <HAL_RCC_ClockConfig+0x3c>
  {
    /* Program the new number of wait states to the LATENCY bits in the FLASH_ACR register */
    __HAL_FLASH_SET_LATENCY(FLatency);
 80016d2:	4b65      	ldr	r3, [pc, #404]	; (8001868 <HAL_RCC_ClockConfig+0x1b8>)
 80016d4:	683a      	ldr	r2, [r7, #0]
 80016d6:	b2d2      	uxtb	r2, r2
 80016d8:	701a      	strb	r2, [r3, #0]

    /* Check that the new number of wait states is taken into account to access the Flash
    memory by reading the FLASH_ACR register */
    if(__HAL_FLASH_GET_LATENCY() != FLatency)
 80016da:	4b63      	ldr	r3, [pc, #396]	; (8001868 <HAL_RCC_ClockConfig+0x1b8>)
 80016dc:	681b      	ldr	r3, [r3, #0]
 80016de:	f003 030f 	and.w	r3, r3, #15
 80016e2:	683a      	ldr	r2, [r7, #0]
 80016e4:	429a      	cmp	r2, r3
 80016e6:	d001      	beq.n	80016ec <HAL_RCC_ClockConfig+0x3c>
    {
      return HAL_ERROR;
 80016e8:	2301      	movs	r3, #1
 80016ea:	e0b8      	b.n	800185e <HAL_RCC_ClockConfig+0x1ae>
    }
  }

  /*-------------------------- HCLK Configuration --------------------------*/
  if(((RCC_ClkInitStruct->ClockType) & RCC_CLOCKTYPE_HCLK) == RCC_CLOCKTYPE_HCLK)
 80016ec:	687b      	ldr	r3, [r7, #4]
 80016ee:	681b      	ldr	r3, [r3, #0]
 80016f0:	f003 0302 	and.w	r3, r3, #2
 80016f4:	2b00      	cmp	r3, #0
 80016f6:	d020      	beq.n	800173a <HAL_RCC_ClockConfig+0x8a>
  {
    /* Set the highest APBx dividers in order to ensure that we do not go through
       a non-spec phase whatever we decrease or increase HCLK. */
    if(((RCC_ClkInitStruct->ClockType) & RCC_CLOCKTYPE_PCLK1) == RCC_CLOCKTYPE_PCLK1)
 80016f8:	687b      	ldr	r3, [r7, #4]
 80016fa:	681b      	ldr	r3, [r3, #0]
 80016fc:	f003 0304 	and.w	r3, r3, #4
 8001700:	2b00      	cmp	r3, #0
 8001702:	d005      	beq.n	8001710 <HAL_RCC_ClockConfig+0x60>
    {
      MODIFY_REG(RCC->CFGR, RCC_CFGR_PPRE1, RCC_HCLK_DIV16);
 8001704:	4b59      	ldr	r3, [pc, #356]	; (800186c <HAL_RCC_ClockConfig+0x1bc>)
 8001706:	689b      	ldr	r3, [r3, #8]
 8001708:	4a58      	ldr	r2, [pc, #352]	; (800186c <HAL_RCC_ClockConfig+0x1bc>)
 800170a:	f443 53e0 	orr.w	r3, r3, #7168	; 0x1c00
 800170e:	6093      	str	r3, [r2, #8]
    }

    if(((RCC_ClkInitStruct->ClockType) & RCC_CLOCKTYPE_PCLK2) == RCC_CLOCKTYPE_PCLK2)
 8001710:	687b      	ldr	r3, [r7, #4]
 8001712:	681b      	ldr	r3, [r3, #0]
 8001714:	f003 0308 	and.w	r3, r3, #8
 8001718:	2b00      	cmp	r3, #0
 800171a:	d005      	beq.n	8001728 <HAL_RCC_ClockConfig+0x78>
    {
      MODIFY_REG(RCC->CFGR, RCC_CFGR_PPRE2, (RCC_HCLK_DIV16 << 3));
 800171c:	4b53      	ldr	r3, [pc, #332]	; (800186c <HAL_RCC_ClockConfig+0x1bc>)
 800171e:	689b      	ldr	r3, [r3, #8]
 8001720:	4a52      	ldr	r2, [pc, #328]	; (800186c <HAL_RCC_ClockConfig+0x1bc>)
 8001722:	f443 4360 	orr.w	r3, r3, #57344	; 0xe000
 8001726:	6093      	str	r3, [r2, #8]
    }

    assert_param(IS_RCC_HCLK(RCC_ClkInitStruct->AHBCLKDivider));
    MODIFY_REG(RCC->CFGR, RCC_CFGR_HPRE, RCC_ClkInitStruct->AHBCLKDivider);
 8001728:	4b50      	ldr	r3, [pc, #320]	; (800186c <HAL_RCC_ClockConfig+0x1bc>)
 800172a:	689b      	ldr	r3, [r3, #8]
 800172c:	f023 02f0 	bic.w	r2, r3, #240	; 0xf0
 8001730:	687b      	ldr	r3, [r7, #4]
 8001732:	689b      	ldr	r3, [r3, #8]
 8001734:	494d      	ldr	r1, [pc, #308]	; (800186c <HAL_RCC_ClockConfig+0x1bc>)
 8001736:	4313      	orrs	r3, r2
 8001738:	608b      	str	r3, [r1, #8]
  }

  /*------------------------- SYSCLK Configuration ---------------------------*/
  if(((RCC_ClkInitStruct->ClockType) & RCC_CLOCKTYPE_SYSCLK) == RCC_CLOCKTYPE_SYSCLK)
 800173a:	687b      	ldr	r3, [r7, #4]
 800173c:	681b      	ldr	r3, [r3, #0]
 800173e:	f003 0301 	and.w	r3, r3, #1
 8001742:	2b00      	cmp	r3, #0
 8001744:	d044      	beq.n	80017d0 <HAL_RCC_ClockConfig+0x120>
  {
    assert_param(IS_RCC_SYSCLKSOURCE(RCC_ClkInitStruct->SYSCLKSource));

    /* HSE is selected as System Clock Source */
    if(RCC_ClkInitStruct->SYSCLKSource == RCC_SYSCLKSOURCE_HSE)
 8001746:	687b      	ldr	r3, [r7, #4]
 8001748:	685b      	ldr	r3, [r3, #4]
 800174a:	2b01      	cmp	r3, #1
 800174c:	d107      	bne.n	800175e <HAL_RCC_ClockConfig+0xae>
    {
      /* Check the HSE ready flag */
      if(__HAL_RCC_GET_FLAG(RCC_FLAG_HSERDY) == RESET)
 800174e:	4b47      	ldr	r3, [pc, #284]	; (800186c <HAL_RCC_ClockConfig+0x1bc>)
 8001750:	681b      	ldr	r3, [r3, #0]
 8001752:	f403 3300 	and.w	r3, r3, #131072	; 0x20000
 8001756:	2b00      	cmp	r3, #0
 8001758:	d119      	bne.n	800178e <HAL_RCC_ClockConfig+0xde>
      {
        return HAL_ERROR;
 800175a:	2301      	movs	r3, #1
 800175c:	e07f      	b.n	800185e <HAL_RCC_ClockConfig+0x1ae>
      }
    }
    /* PLL is selected as System Clock Source */
    else if((RCC_ClkInitStruct->SYSCLKSource == RCC_SYSCLKSOURCE_PLLCLK)   ||
 800175e:	687b      	ldr	r3, [r7, #4]
 8001760:	685b      	ldr	r3, [r3, #4]
 8001762:	2b02      	cmp	r3, #2
 8001764:	d003      	beq.n	800176e <HAL_RCC_ClockConfig+0xbe>
            (RCC_ClkInitStruct->SYSCLKSource == RCC_SYSCLKSOURCE_PLLRCLK))
 8001766:	687b      	ldr	r3, [r7, #4]
 8001768:	685b      	ldr	r3, [r3, #4]
    else if((RCC_ClkInitStruct->SYSCLKSource == RCC_SYSCLKSOURCE_PLLCLK)   ||
 800176a:	2b03      	cmp	r3, #3
 800176c:	d107      	bne.n	800177e <HAL_RCC_ClockConfig+0xce>
    {
      /* Check the PLL ready flag */
      if(__HAL_RCC_GET_FLAG(RCC_FLAG_PLLRDY) == RESET)
 800176e:	4b3f      	ldr	r3, [pc, #252]	; (800186c <HAL_RCC_ClockConfig+0x1bc>)
 8001770:	681b      	ldr	r3, [r3, #0]
 8001772:	f003 7300 	and.w	r3, r3, #33554432	; 0x2000000
 8001776:	2b00      	cmp	r3, #0
 8001778:	d109      	bne.n	800178e <HAL_RCC_ClockConfig+0xde>
      {
        return HAL_ERROR;
 800177a:	2301      	movs	r3, #1
 800177c:	e06f      	b.n	800185e <HAL_RCC_ClockConfig+0x1ae>
    }
    /* HSI is selected as System Clock Source */
    else
    {
      /* Check the HSI ready flag */
      if(__HAL_RCC_GET_FLAG(RCC_FLAG_HSIRDY) == RESET)
 800177e:	4b3b      	ldr	r3, [pc, #236]	; (800186c <HAL_RCC_ClockConfig+0x1bc>)
 8001780:	681b      	ldr	r3, [r3, #0]
 8001782:	f003 0302 	and.w	r3, r3, #2
 8001786:	2b00      	cmp	r3, #0
 8001788:	d101      	bne.n	800178e <HAL_RCC_ClockConfig+0xde>
      {
        return HAL_ERROR;
 800178a:	2301      	movs	r3, #1
 800178c:	e067      	b.n	800185e <HAL_RCC_ClockConfig+0x1ae>
      }
    }

    __HAL_RCC_SYSCLK_CONFIG(RCC_ClkInitStruct->SYSCLKSource);
 800178e:	4b37      	ldr	r3, [pc, #220]	; (800186c <HAL_RCC_ClockConfig+0x1bc>)
 8001790:	689b      	ldr	r3, [r3, #8]
 8001792:	f023 0203 	bic.w	r2, r3, #3
 8001796:	687b      	ldr	r3, [r7, #4]
 8001798:	685b      	ldr	r3, [r3, #4]
 800179a:	4934      	ldr	r1, [pc, #208]	; (800186c <HAL_RCC_ClockConfig+0x1bc>)
 800179c:	4313      	orrs	r3, r2
 800179e:	608b      	str	r3, [r1, #8]

    /* Get Start Tick */
    tickstart = HAL_GetTick();
 80017a0:	f7ff fa1a 	bl	8000bd8 <HAL_GetTick>
 80017a4:	60f8      	str	r0, [r7, #12]

    while (__HAL_RCC_GET_SYSCLK_SOURCE() != (RCC_ClkInitStruct->SYSCLKSource << RCC_CFGR_SWS_Pos))
 80017a6:	e00a      	b.n	80017be <HAL_RCC_ClockConfig+0x10e>
    {
      if ((HAL_GetTick() - tickstart) > CLOCKSWITCH_TIMEOUT_VALUE)
 80017a8:	f7ff fa16 	bl	8000bd8 <HAL_GetTick>
 80017ac:	4602      	mov	r2, r0
 80017ae:	68fb      	ldr	r3, [r7, #12]
 80017b0:	1ad3      	subs	r3, r2, r3
 80017b2:	f241 3288 	movw	r2, #5000	; 0x1388
 80017b6:	4293      	cmp	r3, r2
 80017b8:	d901      	bls.n	80017be <HAL_RCC_ClockConfig+0x10e>
      {
        return HAL_TIMEOUT;
 80017ba:	2303      	movs	r3, #3
 80017bc:	e04f      	b.n	800185e <HAL_RCC_ClockConfig+0x1ae>
    while (__HAL_RCC_GET_SYSCLK_SOURCE() != (RCC_ClkInitStruct->SYSCLKSource << RCC_CFGR_SWS_Pos))
 80017be:	4b2b      	ldr	r3, [pc, #172]	; (800186c <HAL_RCC_ClockConfig+0x1bc>)
 80017c0:	689b      	ldr	r3, [r3, #8]
 80017c2:	f003 020c 	and.w	r2, r3, #12
 80017c6:	687b      	ldr	r3, [r7, #4]
 80017c8:	685b      	ldr	r3, [r3, #4]
 80017ca:	009b      	lsls	r3, r3, #2
 80017cc:	429a      	cmp	r2, r3
 80017ce:	d1eb      	bne.n	80017a8 <HAL_RCC_ClockConfig+0xf8>
      }
    }
  }

  /* Decreasing the number of wait states because of lower CPU frequency */
  if(FLatency < __HAL_FLASH_GET_LATENCY())
 80017d0:	4b25      	ldr	r3, [pc, #148]	; (8001868 <HAL_RCC_ClockConfig+0x1b8>)
 80017d2:	681b      	ldr	r3, [r3, #0]
 80017d4:	f003 030f 	and.w	r3, r3, #15
 80017d8:	683a      	ldr	r2, [r7, #0]
 80017da:	429a      	cmp	r2, r3
 80017dc:	d20c      	bcs.n	80017f8 <HAL_RCC_ClockConfig+0x148>
  {
     /* Program the new number of wait states to the LATENCY bits in the FLASH_ACR register */
    __HAL_FLASH_SET_LATENCY(FLatency);
 80017de:	4b22      	ldr	r3, [pc, #136]	; (8001868 <HAL_RCC_ClockConfig+0x1b8>)
 80017e0:	683a      	ldr	r2, [r7, #0]
 80017e2:	b2d2      	uxtb	r2, r2
 80017e4:	701a      	strb	r2, [r3, #0]

    /* Check that the new number of wait states is taken into account to access the Flash
    memory by reading the FLASH_ACR register */
    if(__HAL_FLASH_GET_LATENCY() != FLatency)
 80017e6:	4b20      	ldr	r3, [pc, #128]	; (8001868 <HAL_RCC_ClockConfig+0x1b8>)
 80017e8:	681b      	ldr	r3, [r3, #0]
 80017ea:	f003 030f 	and.w	r3, r3, #15
 80017ee:	683a      	ldr	r2, [r7, #0]
 80017f0:	429a      	cmp	r2, r3
 80017f2:	d001      	beq.n	80017f8 <HAL_RCC_ClockConfig+0x148>
    {
      return HAL_ERROR;
 80017f4:	2301      	movs	r3, #1
 80017f6:	e032      	b.n	800185e <HAL_RCC_ClockConfig+0x1ae>
    }
  }

  /*-------------------------- PCLK1 Configuration ---------------------------*/
  if(((RCC_ClkInitStruct->ClockType) & RCC_CLOCKTYPE_PCLK1) == RCC_CLOCKTYPE_PCLK1)
 80017f8:	687b      	ldr	r3, [r7, #4]
 80017fa:	681b      	ldr	r3, [r3, #0]
 80017fc:	f003 0304 	and.w	r3, r3, #4
 8001800:	2b00      	cmp	r3, #0
 8001802:	d008      	beq.n	8001816 <HAL_RCC_ClockConfig+0x166>
  {
    assert_param(IS_RCC_PCLK(RCC_ClkInitStruct->APB1CLKDivider));
    MODIFY_REG(RCC->CFGR, RCC_CFGR_PPRE1, RCC_ClkInitStruct->APB1CLKDivider);
 8001804:	4b19      	ldr	r3, [pc, #100]	; (800186c <HAL_RCC_ClockConfig+0x1bc>)
 8001806:	689b      	ldr	r3, [r3, #8]
 8001808:	f423 52e0 	bic.w	r2, r3, #7168	; 0x1c00
 800180c:	687b      	ldr	r3, [r7, #4]
 800180e:	68db      	ldr	r3, [r3, #12]
 8001810:	4916      	ldr	r1, [pc, #88]	; (800186c <HAL_RCC_ClockConfig+0x1bc>)
 8001812:	4313      	orrs	r3, r2
 8001814:	608b      	str	r3, [r1, #8]
  }

  /*-------------------------- PCLK2 Configuration ---------------------------*/
  if(((RCC_ClkInitStruct->ClockType) & RCC_CLOCKTYPE_PCLK2) == RCC_CLOCKTYPE_PCLK2)
 8001816:	687b      	ldr	r3, [r7, #4]
 8001818:	681b      	ldr	r3, [r3, #0]
 800181a:	f003 0308 	and.w	r3, r3, #8
 800181e:	2b00      	cmp	r3, #0
 8001820:	d009      	beq.n	8001836 <HAL_RCC_ClockConfig+0x186>
  {
    assert_param(IS_RCC_PCLK(RCC_ClkInitStruct->APB2CLKDivider));
    MODIFY_REG(RCC->CFGR, RCC_CFGR_PPRE2, ((RCC_ClkInitStruct->APB2CLKDivider) << 3U));
 8001822:	4b12      	ldr	r3, [pc, #72]	; (800186c <HAL_RCC_ClockConfig+0x1bc>)
 8001824:	689b      	ldr	r3, [r3, #8]
 8001826:	f423 4260 	bic.w	r2, r3, #57344	; 0xe000
 800182a:	687b      	ldr	r3, [r7, #4]
 800182c:	691b      	ldr	r3, [r3, #16]
 800182e:	00db      	lsls	r3, r3, #3
 8001830:	490e      	ldr	r1, [pc, #56]	; (800186c <HAL_RCC_ClockConfig+0x1bc>)
 8001832:	4313      	orrs	r3, r2
 8001834:	608b      	str	r3, [r1, #8]
  }

  /* Update the SystemCoreClock global variable */
  SystemCoreClock = HAL_RCC_GetSysClockFreq() >> AHBPrescTable[(RCC->CFGR & RCC_CFGR_HPRE)>> RCC_CFGR_HPRE_Pos];
 8001836:	f000 f821 	bl	800187c <HAL_RCC_GetSysClockFreq>
 800183a:	4602      	mov	r2, r0
 800183c:	4b0b      	ldr	r3, [pc, #44]	; (800186c <HAL_RCC_ClockConfig+0x1bc>)
 800183e:	689b      	ldr	r3, [r3, #8]
 8001840:	091b      	lsrs	r3, r3, #4
 8001842:	f003 030f 	and.w	r3, r3, #15
 8001846:	490a      	ldr	r1, [pc, #40]	; (8001870 <HAL_RCC_ClockConfig+0x1c0>)
 8001848:	5ccb      	ldrb	r3, [r1, r3]
 800184a:	fa22 f303 	lsr.w	r3, r2, r3
 800184e:	4a09      	ldr	r2, [pc, #36]	; (8001874 <HAL_RCC_ClockConfig+0x1c4>)
 8001850:	6013      	str	r3, [r2, #0]

  /* Configure the source of time base considering new system clocks settings */
  HAL_InitTick (uwTickPrio);
 8001852:	4b09      	ldr	r3, [pc, #36]	; (8001878 <HAL_RCC_ClockConfig+0x1c8>)
 8001854:	681b      	ldr	r3, [r3, #0]
 8001856:	4618      	mov	r0, r3
 8001858:	f7ff f97a 	bl	8000b50 <HAL_InitTick>

  return HAL_OK;
 800185c:	2300      	movs	r3, #0
}
 800185e:	4618      	mov	r0, r3
 8001860:	3710      	adds	r7, #16
 8001862:	46bd      	mov	sp, r7
 8001864:	bd80      	pop	{r7, pc}
 8001866:	bf00      	nop
 8001868:	40023c00 	.word	0x40023c00
 800186c:	40023800 	.word	0x40023800
 8001870:	08001af8 	.word	0x08001af8
 8001874:	20000000 	.word	0x20000000
 8001878:	20000004 	.word	0x20000004

0800187c <HAL_RCC_GetSysClockFreq>:
  *
  *
  * @retval SYSCLK frequency
  */
__weak uint32_t HAL_RCC_GetSysClockFreq(void)
{
 800187c:	e92d 4fb0 	stmdb	sp!, {r4, r5, r7, r8, r9, sl, fp, lr}
 8001880:	b094      	sub	sp, #80	; 0x50
 8001882:	af00      	add	r7, sp, #0
  uint32_t pllm = 0U, pllvco = 0U, pllp = 0U;
 8001884:	2300      	movs	r3, #0
 8001886:	647b      	str	r3, [r7, #68]	; 0x44
 8001888:	2300      	movs	r3, #0
 800188a:	64fb      	str	r3, [r7, #76]	; 0x4c
 800188c:	2300      	movs	r3, #0
 800188e:	643b      	str	r3, [r7, #64]	; 0x40
  uint32_t sysclockfreq = 0U;
 8001890:	2300      	movs	r3, #0
 8001892:	64bb      	str	r3, [r7, #72]	; 0x48

  /* Get SYSCLK source -------------------------------------------------------*/
  switch (RCC->CFGR & RCC_CFGR_SWS)
 8001894:	4b79      	ldr	r3, [pc, #484]	; (8001a7c <HAL_RCC_GetSysClockFreq+0x200>)
 8001896:	689b      	ldr	r3, [r3, #8]
 8001898:	f003 030c 	and.w	r3, r3, #12
 800189c:	2b08      	cmp	r3, #8
 800189e:	d00d      	beq.n	80018bc <HAL_RCC_GetSysClockFreq+0x40>
 80018a0:	2b08      	cmp	r3, #8
 80018a2:	f200 80e1 	bhi.w	8001a68 <HAL_RCC_GetSysClockFreq+0x1ec>
 80018a6:	2b00      	cmp	r3, #0
 80018a8:	d002      	beq.n	80018b0 <HAL_RCC_GetSysClockFreq+0x34>
 80018aa:	2b04      	cmp	r3, #4
 80018ac:	d003      	beq.n	80018b6 <HAL_RCC_GetSysClockFreq+0x3a>
 80018ae:	e0db      	b.n	8001a68 <HAL_RCC_GetSysClockFreq+0x1ec>
  {
    case RCC_CFGR_SWS_HSI:  /* HSI used as system clock source */
    {
      sysclockfreq = HSI_VALUE;
 80018b0:	4b73      	ldr	r3, [pc, #460]	; (8001a80 <HAL_RCC_GetSysClockFreq+0x204>)
 80018b2:	64bb      	str	r3, [r7, #72]	; 0x48
       break;
 80018b4:	e0db      	b.n	8001a6e <HAL_RCC_GetSysClockFreq+0x1f2>
    }
    case RCC_CFGR_SWS_HSE:  /* HSE used as system clock  source */
    {
      sysclockfreq = HSE_VALUE;
 80018b6:	4b73      	ldr	r3, [pc, #460]	; (8001a84 <HAL_RCC_GetSysClockFreq+0x208>)
 80018b8:	64bb      	str	r3, [r7, #72]	; 0x48
      break;
 80018ba:	e0d8      	b.n	8001a6e <HAL_RCC_GetSysClockFreq+0x1f2>
    }
    case RCC_CFGR_SWS_PLL:  /* PLL used as system clock  source */
    {
      /* PLL_VCO = (HSE_VALUE or HSI_VALUE / PLLM) * PLLN
      SYSCLK = PLL_VCO / PLLP */
      pllm = RCC->PLLCFGR & RCC_PLLCFGR_PLLM;
 80018bc:	4b6f      	ldr	r3, [pc, #444]	; (8001a7c <HAL_RCC_GetSysClockFreq+0x200>)
 80018be:	685b      	ldr	r3, [r3, #4]
 80018c0:	f003 033f 	and.w	r3, r3, #63	; 0x3f
 80018c4:	647b      	str	r3, [r7, #68]	; 0x44
      if(__HAL_RCC_GET_PLL_OSCSOURCE() != RCC_PLLSOURCE_HSI)
 80018c6:	4b6d      	ldr	r3, [pc, #436]	; (8001a7c <HAL_RCC_GetSysClockFreq+0x200>)
 80018c8:	685b      	ldr	r3, [r3, #4]
 80018ca:	f403 0380 	and.w	r3, r3, #4194304	; 0x400000
 80018ce:	2b00      	cmp	r3, #0
 80018d0:	d063      	beq.n	800199a <HAL_RCC_GetSysClockFreq+0x11e>
      {
        /* HSE used as PLL clock source */
        pllvco = (uint32_t) ((((uint64_t) HSE_VALUE * ((uint64_t) ((RCC->PLLCFGR & RCC_PLLCFGR_PLLN) >> RCC_PLLCFGR_PLLN_Pos)))) / (uint64_t)pllm);
 80018d2:	4b6a      	ldr	r3, [pc, #424]	; (8001a7c <HAL_RCC_GetSysClockFreq+0x200>)
 80018d4:	685b      	ldr	r3, [r3, #4]
 80018d6:	099b      	lsrs	r3, r3, #6
 80018d8:	2200      	movs	r2, #0
 80018da:	63bb      	str	r3, [r7, #56]	; 0x38
 80018dc:	63fa      	str	r2, [r7, #60]	; 0x3c
 80018de:	6bbb      	ldr	r3, [r7, #56]	; 0x38
 80018e0:	f3c3 0308 	ubfx	r3, r3, #0, #9
 80018e4:	633b      	str	r3, [r7, #48]	; 0x30
 80018e6:	2300      	movs	r3, #0
 80018e8:	637b      	str	r3, [r7, #52]	; 0x34
 80018ea:	e9d7 450c 	ldrd	r4, r5, [r7, #48]	; 0x30
 80018ee:	4622      	mov	r2, r4
 80018f0:	462b      	mov	r3, r5
 80018f2:	f04f 0000 	mov.w	r0, #0
 80018f6:	f04f 0100 	mov.w	r1, #0
 80018fa:	0159      	lsls	r1, r3, #5
 80018fc:	ea41 61d2 	orr.w	r1, r1, r2, lsr #27
 8001900:	0150      	lsls	r0, r2, #5
 8001902:	4602      	mov	r2, r0
 8001904:	460b      	mov	r3, r1
 8001906:	4621      	mov	r1, r4
 8001908:	1a51      	subs	r1, r2, r1
 800190a:	6139      	str	r1, [r7, #16]
 800190c:	4629      	mov	r1, r5
 800190e:	eb63 0301 	sbc.w	r3, r3, r1
 8001912:	617b      	str	r3, [r7, #20]
 8001914:	f04f 0200 	mov.w	r2, #0
 8001918:	f04f 0300 	mov.w	r3, #0
 800191c:	e9d7 ab04 	ldrd	sl, fp, [r7, #16]
 8001920:	4659      	mov	r1, fp
 8001922:	018b      	lsls	r3, r1, #6
 8001924:	4651      	mov	r1, sl
 8001926:	ea43 6391 	orr.w	r3, r3, r1, lsr #26
 800192a:	4651      	mov	r1, sl
 800192c:	018a      	lsls	r2, r1, #6
 800192e:	4651      	mov	r1, sl
 8001930:	ebb2 0801 	subs.w	r8, r2, r1
 8001934:	4659      	mov	r1, fp
 8001936:	eb63 0901 	sbc.w	r9, r3, r1
 800193a:	f04f 0200 	mov.w	r2, #0
 800193e:	f04f 0300 	mov.w	r3, #0
 8001942:	ea4f 03c9 	mov.w	r3, r9, lsl #3
 8001946:	ea43 7358 	orr.w	r3, r3, r8, lsr #29
 800194a:	ea4f 02c8 	mov.w	r2, r8, lsl #3
 800194e:	4690      	mov	r8, r2
 8001950:	4699      	mov	r9, r3
 8001952:	4623      	mov	r3, r4
 8001954:	eb18 0303 	adds.w	r3, r8, r3
 8001958:	60bb      	str	r3, [r7, #8]
 800195a:	462b      	mov	r3, r5
 800195c:	eb49 0303 	adc.w	r3, r9, r3
 8001960:	60fb      	str	r3, [r7, #12]
 8001962:	f04f 0200 	mov.w	r2, #0
 8001966:	f04f 0300 	mov.w	r3, #0
 800196a:	e9d7 4502 	ldrd	r4, r5, [r7, #8]
 800196e:	4629      	mov	r1, r5
 8001970:	024b      	lsls	r3, r1, #9
 8001972:	4621      	mov	r1, r4
 8001974:	ea43 53d1 	orr.w	r3, r3, r1, lsr #23
 8001978:	4621      	mov	r1, r4
 800197a:	024a      	lsls	r2, r1, #9
 800197c:	4610      	mov	r0, r2
 800197e:	4619      	mov	r1, r3
 8001980:	6c7b      	ldr	r3, [r7, #68]	; 0x44
 8001982:	2200      	movs	r2, #0
 8001984:	62bb      	str	r3, [r7, #40]	; 0x28
 8001986:	62fa      	str	r2, [r7, #44]	; 0x2c
 8001988:	e9d7 230a 	ldrd	r2, r3, [r7, #40]	; 0x28
 800198c:	f7fe fc2e 	bl	80001ec <__aeabi_uldivmod>
 8001990:	4602      	mov	r2, r0
 8001992:	460b      	mov	r3, r1
 8001994:	4613      	mov	r3, r2
 8001996:	64fb      	str	r3, [r7, #76]	; 0x4c
 8001998:	e058      	b.n	8001a4c <HAL_RCC_GetSysClockFreq+0x1d0>
      }
      else
      {
        /* HSI used as PLL clock source */
        pllvco = (uint32_t) ((((uint64_t) HSI_VALUE * ((uint64_t) ((RCC->PLLCFGR & RCC_PLLCFGR_PLLN) >> RCC_PLLCFGR_PLLN_Pos)))) / (uint64_t)pllm);
 800199a:	4b38      	ldr	r3, [pc, #224]	; (8001a7c <HAL_RCC_GetSysClockFreq+0x200>)
 800199c:	685b      	ldr	r3, [r3, #4]
 800199e:	099b      	lsrs	r3, r3, #6
 80019a0:	2200      	movs	r2, #0
 80019a2:	4618      	mov	r0, r3
 80019a4:	4611      	mov	r1, r2
 80019a6:	f3c0 0308 	ubfx	r3, r0, #0, #9
 80019aa:	623b      	str	r3, [r7, #32]
 80019ac:	2300      	movs	r3, #0
 80019ae:	627b      	str	r3, [r7, #36]	; 0x24
 80019b0:	e9d7 8908 	ldrd	r8, r9, [r7, #32]
 80019b4:	4642      	mov	r2, r8
 80019b6:	464b      	mov	r3, r9
 80019b8:	f04f 0000 	mov.w	r0, #0
 80019bc:	f04f 0100 	mov.w	r1, #0
 80019c0:	0159      	lsls	r1, r3, #5
 80019c2:	ea41 61d2 	orr.w	r1, r1, r2, lsr #27
 80019c6:	0150      	lsls	r0, r2, #5
 80019c8:	4602      	mov	r2, r0
 80019ca:	460b      	mov	r3, r1
 80019cc:	4641      	mov	r1, r8
 80019ce:	ebb2 0a01 	subs.w	sl, r2, r1
 80019d2:	4649      	mov	r1, r9
 80019d4:	eb63 0b01 	sbc.w	fp, r3, r1
 80019d8:	f04f 0200 	mov.w	r2, #0
 80019dc:	f04f 0300 	mov.w	r3, #0
 80019e0:	ea4f 138b 	mov.w	r3, fp, lsl #6
 80019e4:	ea43 639a 	orr.w	r3, r3, sl, lsr #26
 80019e8:	ea4f 128a 	mov.w	r2, sl, lsl #6
 80019ec:	ebb2 040a 	subs.w	r4, r2, sl
 80019f0:	eb63 050b 	sbc.w	r5, r3, fp
 80019f4:	f04f 0200 	mov.w	r2, #0
 80019f8:	f04f 0300 	mov.w	r3, #0
 80019fc:	00eb      	lsls	r3, r5, #3
 80019fe:	ea43 7354 	orr.w	r3, r3, r4, lsr #29
 8001a02:	00e2      	lsls	r2, r4, #3
 8001a04:	4614      	mov	r4, r2
 8001a06:	461d      	mov	r5, r3
 8001a08:	4643      	mov	r3, r8
 8001a0a:	18e3      	adds	r3, r4, r3
 8001a0c:	603b      	str	r3, [r7, #0]
 8001a0e:	464b      	mov	r3, r9
 8001a10:	eb45 0303 	adc.w	r3, r5, r3
 8001a14:	607b      	str	r3, [r7, #4]
 8001a16:	f04f 0200 	mov.w	r2, #0
 8001a1a:	f04f 0300 	mov.w	r3, #0
 8001a1e:	e9d7 4500 	ldrd	r4, r5, [r7]
 8001a22:	4629      	mov	r1, r5
 8001a24:	028b      	lsls	r3, r1, #10
 8001a26:	4621      	mov	r1, r4
 8001a28:	ea43 5391 	orr.w	r3, r3, r1, lsr #22
 8001a2c:	4621      	mov	r1, r4
 8001a2e:	028a      	lsls	r2, r1, #10
 8001a30:	4610      	mov	r0, r2
 8001a32:	4619      	mov	r1, r3
 8001a34:	6c7b      	ldr	r3, [r7, #68]	; 0x44
 8001a36:	2200      	movs	r2, #0
 8001a38:	61bb      	str	r3, [r7, #24]
 8001a3a:	61fa      	str	r2, [r7, #28]
 8001a3c:	e9d7 2306 	ldrd	r2, r3, [r7, #24]
 8001a40:	f7fe fbd4 	bl	80001ec <__aeabi_uldivmod>
 8001a44:	4602      	mov	r2, r0
 8001a46:	460b      	mov	r3, r1
 8001a48:	4613      	mov	r3, r2
 8001a4a:	64fb      	str	r3, [r7, #76]	; 0x4c
      }
      pllp = ((((RCC->PLLCFGR & RCC_PLLCFGR_PLLP) >> RCC_PLLCFGR_PLLP_Pos) + 1U) *2U);
 8001a4c:	4b0b      	ldr	r3, [pc, #44]	; (8001a7c <HAL_RCC_GetSysClockFreq+0x200>)
 8001a4e:	685b      	ldr	r3, [r3, #4]
 8001a50:	0c1b      	lsrs	r3, r3, #16
 8001a52:	f003 0303 	and.w	r3, r3, #3
 8001a56:	3301      	adds	r3, #1
 8001a58:	005b      	lsls	r3, r3, #1
 8001a5a:	643b      	str	r3, [r7, #64]	; 0x40

      sysclockfreq = pllvco/pllp;
 8001a5c:	6cfa      	ldr	r2, [r7, #76]	; 0x4c
 8001a5e:	6c3b      	ldr	r3, [r7, #64]	; 0x40
 8001a60:	fbb2 f3f3 	udiv	r3, r2, r3
 8001a64:	64bb      	str	r3, [r7, #72]	; 0x48
      break;
 8001a66:	e002      	b.n	8001a6e <HAL_RCC_GetSysClockFreq+0x1f2>
    }
    default:
    {
      sysclockfreq = HSI_VALUE;
 8001a68:	4b05      	ldr	r3, [pc, #20]	; (8001a80 <HAL_RCC_GetSysClockFreq+0x204>)
 8001a6a:	64bb      	str	r3, [r7, #72]	; 0x48
      break;
 8001a6c:	bf00      	nop
    }
  }
  return sysclockfreq;
 8001a6e:	6cbb      	ldr	r3, [r7, #72]	; 0x48
}
 8001a70:	4618      	mov	r0, r3
 8001a72:	3750      	adds	r7, #80	; 0x50
 8001a74:	46bd      	mov	sp, r7
 8001a76:	e8bd 8fb0 	ldmia.w	sp!, {r4, r5, r7, r8, r9, sl, fp, pc}
 8001a7a:	bf00      	nop
 8001a7c:	40023800 	.word	0x40023800
 8001a80:	00f42400 	.word	0x00f42400
 8001a84:	007a1200 	.word	0x007a1200

08001a88 <__libc_init_array>:
 8001a88:	b570      	push	{r4, r5, r6, lr}
 8001a8a:	4d0d      	ldr	r5, [pc, #52]	; (8001ac0 <__libc_init_array+0x38>)
 8001a8c:	4c0d      	ldr	r4, [pc, #52]	; (8001ac4 <__libc_init_array+0x3c>)
 8001a8e:	1b64      	subs	r4, r4, r5
 8001a90:	10a4      	asrs	r4, r4, #2
 8001a92:	2600      	movs	r6, #0
 8001a94:	42a6      	cmp	r6, r4
 8001a96:	d109      	bne.n	8001aac <__libc_init_array+0x24>
 8001a98:	4d0b      	ldr	r5, [pc, #44]	; (8001ac8 <__libc_init_array+0x40>)
 8001a9a:	4c0c      	ldr	r4, [pc, #48]	; (8001acc <__libc_init_array+0x44>)
 8001a9c:	f000 f820 	bl	8001ae0 <_init>
 8001aa0:	1b64      	subs	r4, r4, r5
 8001aa2:	10a4      	asrs	r4, r4, #2
 8001aa4:	2600      	movs	r6, #0
 8001aa6:	42a6      	cmp	r6, r4
 8001aa8:	d105      	bne.n	8001ab6 <__libc_init_array+0x2e>
 8001aaa:	bd70      	pop	{r4, r5, r6, pc}
 8001aac:	f855 3b04 	ldr.w	r3, [r5], #4
 8001ab0:	4798      	blx	r3
 8001ab2:	3601      	adds	r6, #1
 8001ab4:	e7ee      	b.n	8001a94 <__libc_init_array+0xc>
 8001ab6:	f855 3b04 	ldr.w	r3, [r5], #4
 8001aba:	4798      	blx	r3
 8001abc:	3601      	adds	r6, #1
 8001abe:	e7f2      	b.n	8001aa6 <__libc_init_array+0x1e>
 8001ac0:	08001b10 	.word	0x08001b10
 8001ac4:	08001b10 	.word	0x08001b10
 8001ac8:	08001b10 	.word	0x08001b10
 8001acc:	08001b14 	.word	0x08001b14

08001ad0 <memset>:
 8001ad0:	4402      	add	r2, r0
 8001ad2:	4603      	mov	r3, r0
 8001ad4:	4293      	cmp	r3, r2
 8001ad6:	d100      	bne.n	8001ada <memset+0xa>
 8001ad8:	4770      	bx	lr
 8001ada:	f803 1b01 	strb.w	r1, [r3], #1
 8001ade:	e7f9      	b.n	8001ad4 <memset+0x4>

08001ae0 <_init>:
 8001ae0:	b5f8      	push	{r3, r4, r5, r6, r7, lr}
 8001ae2:	bf00      	nop
 8001ae4:	bcf8      	pop	{r3, r4, r5, r6, r7}
 8001ae6:	bc08      	pop	{r3}
 8001ae8:	469e      	mov	lr, r3
 8001aea:	4770      	bx	lr

08001aec <_fini>:
 8001aec:	b5f8      	push	{r3, r4, r5, r6, r7, lr}
 8001aee:	bf00      	nop
 8001af0:	bcf8      	pop	{r3, r4, r5, r6, r7}
 8001af2:	bc08      	pop	{r3}
 8001af4:	469e      	mov	lr, r3
 8001af6:	4770      	bx	lr
